:100000000C9488750C94B9750C94B9750C94B975E9
:100010000C94B9750C94B9750C94B9750C94B975A8
:100020000C94B9750C94B9750C94B9750C94B97598
:100030000C94B9750D94FA660C94B9750C94B97555
:100040000C94B9750D947A2C0C94B9750C94B975FF
:100050000C94B9750C94B9750D9480240D94B84521
:100060000C94B9750D9438610C94B9750C94B975EC
:100070000C94B9750C94B9750C94B9750C94B97548
:100080000C94B9750C94B9750C94B9750C94B97538
:100090000C94B9750C94B9750C94B9750C94B97528
:1000A0000C94B9750C94B9750C94B9750C94B97518
:1000B0000C94B9750C94B9750C94B9750C94B97508
:1000C0000C94B9750C94B9750C94B9750C94B975F8
:1000D0000C94B9750C94B9750D940F610C94B975A5
:1000E0000C94B975DCC8C5C8C8C8CBC8CEC8D7C8B9
:1000F000E1C8EBC8D1C8D4C825DB28DB17DB1BDB84
:1001000021DB5FDB2CDB30DB36DB3ADB3EDB44DB49
:1001100048DB4CDB5FDB52DB56DB5ADBF700F700DA
:100120005101510151015701570157015F01F3007E
:10013000F300F300D6E66DEA6DEA6DEA6DEA6DEA6A
:100140006DEA6DEA6DEA6DEA6DEA6DEA6DEA6DEAF7
:100150006DEA6DEA6DEA4AEA5FE86DEA30E75CE76E
:10016000D9E9FDE8B8E996E9FAE91BEA6DEA6DEA32
:1001700022E96DEA6DEA6DEACDE8BAE794E76DEA47
:1001800028E8FEE679E92D016B015D01FD004B01D8
:10019000EF0011013F01FF00070133016701EB0090
:1001A00049012B015501ED001D01470153011301C8
:1001B000EB000D016101450105A84CCDB2D44EB94B
:1001C0003836A9020C50B9918688083CA6AAAA2AFA
:1001D000BE000000803F0D946B450D9416450D94B4
:1001E00049440D947A2A0D947C6C0D94F0460D943C
:1001F000676C0D9427250D9462190D948C440D9411
:10020000D9440D9433440D94002C0D94892A0D94F7
:10021000DE440D94B51D0D943A6A0D944D450D9430
:1002200082190D949A440D9443450D94AB1D0D9481
:1002300069420D9466190D941D480D9420450D9446
:100240003B2A0D945E190D942F270D94BF1D0D941C
:10025000171C0D9485700D9404450D944B440D941A
:10026000E4650D944C320D94E8440D941C420D94B9
:100270006A190D94401B0D94AB1F0D9491190D94A8
:10028000D4440D940D430D9487190D9461450D943C
:100290002A450D94FC440D9491440D948C190D94B1
:1002A000C91D0D946E6C0D9439450D940C450D943B
:1002B000756C0D94E4160D94E7330D947F440D9402
:1002C000826C0D9457450D94431B0D9457650D9406
:1002D000F2440D949B4F0D947D440D94C1164E41F4
:1002E0004E494E495459494E46CDCCCC3D0AD723B0
:1002F0003C17B7D13877CC2B329595E6241FB14FF8
:100300000A000020410000C84200401C4620BCBE3C
:100310004CCA1B0E5AAEC59D7400407A10F35A00A9
:10032000A0724E18090010A5D4E80000E87648171E
:100330000000E40B54020000CA9A3B000000E1F503
:1003400005000080969800000040420F000000A0C9
:100350008601000000102700000000E803000000F4
:10036000006400000000000A00000000000100001E
:100370000000002C76D888DC674F0823DFC1DFAE91
:1003800059E1B1B796E5E3E453C63AE6519976965A
:10039000E8E6C28426EB898C9B62ED407C6FFCEF23
:1003A000BC9C9F40F2BAA56FA5F490055A2AF75C51
:1003B000936B6CF9676DC11BFCE0E40D47FEF52003
:1003C000E6B500D0ED902E030094357705008084CB
:1003D0001E080000204E0A000000C80C33333333DF
:1003E0000F986E12831141EF8D2114893BE655164B
:1003F000CFFEE6DB18D1844B381BF77C1D901DA483
:10040000BBE424203284725E228100C9F124ECA175
:10041000E53D274C4556454C494E4700434F4D4D11
:10042000554E49434154494F4E0044525952554E3E
:10043000004552524F525300494E464F00454348E3
:100440004F00536C6565702E2E2E003C3C3C2047BF
:1004500032380A005261697365205A202862656645
:100460006F726520686F6D696E672920746F200058
:100470003E20656E6473746F70732E656E61626C7E
:10048000652874727565290A003C3C3C2047323867
:100490000A003E20686F6D696E67206E6F74206E73
:1004A00065656465642C20736B69700A003E3E3E8E
:1004B000204732380A00205A3A200020593A2000BA
:1004C00042656420583A20005761697420666F7253
:1004D00020757365722E2E2E004E6F206D6F76651F
:1004E0002E00456E642066696C65206C6973740A21
:1004F00000426567696E2066696C65206C6973747B
:100500000A002F2F616374696F6E3A73746172749D
:100510000A004D3132350043757272656E74206683
:10052000696C653A20005072696E742074696D655B
:100530003A20003D04380431042A041C0413046FDB
:1005400066660044454255473A004B494C4C454489
:100550002E20004D3131332053006F6B0054494E33
:100560004132204F66662E002C20002C2000464988
:10057000524D574152455F4E414D453A4D61726C67
:10058000696E204649524D574152455F5645525378
:10059000494F4E3A322E31352E322048415244577F
:1005A0004152455F56455253494F4E3A312E3920FC
:1005B0004D414348494E455F545950453A54494E80
:1005C00041322045585452554445525F434F554E91
:1005D000543A310A002F2F20004D31343520533C3E
:1005E000696E6465783E206F7574206F6620726155
:1005F0006E67652028302D31290A002054002052D2
:1006000000416363656C65726174696F6E3A205076
:100610000020466C6F773A200000011A1C18FF0278
:10062000FFFFFF3C3D3828FFFFFFFF2E303E121337
:10063000FFFFFFFFFF0C0804FFFFFF363726FFFF19
:10064000FF08440A094350726F6265205A204F66C2
:10065000667365743A200020643A0020693A0020ED
:10066000703A00496E76616C6964206578747275C1
:100670006465720A0043290A0061626C656420287F
:100680006D696E2074656D702000436F6C64206529
:10069000787472756465732061726520004E6F20F6
:1006A00063617365206C696768740A004265642041
:1006B0004C6576656C696E6720004661696C65649F
:1006C00020746F20656E61626C6520426564204C09
:1006D0006576656C696E670A00426564204C6576D4
:1006E000656C20436F7272656374696F6E204D6133
:1006F000747269783A00454550524F4D204F4B0A6D
:10070000003A200050726F6265205A204F6666736F
:100710006574003F5A206F7574206F662072616E99
:10072000676520282D323020746F203230290A006E
:100730004163746976652045787472756465723AB0
:100740002000496E76616C69642065787472756406
:1007500065720A003C3C3C2067636F64655F540A25
:1007600000203A2041465445520A00202063757209
:1007700072656E745F706F736974696F6E3D00208F
:100780003A204245464F52450A0020206375727256
:10079000656E745F706F736974696F6E3D003E3E85
:1007A0003E2067636F64655F5428004572726F7204
:1007B0002077726974696E6720746F2045455052C6
:1007C0004F4D210A00454550524F4D2064617461E0
:1007D00073697A65206572726F722E0A00290A00A9
:1007E0002062797465733B206372632000536574E3
:1007F00074696E67732053746F72656420280029D2
:100800000A002062797465733B20637263200020C4
:1008100073746F7265642073657474696E67732096
:1008200072657472696576656420280020286361AA
:100830006C63756C6174656429210A0020213D2078
:1008400000454550524F4D20435243206D69736D12
:1008500061746368202D202873746F726564292089
:10086000002053697A653A2000496E6465783A2021
:1008700000204D61726C696E3D563536290A00289C
:10088000454550524F4D3D00454550524F4D207605
:10089000657273696F6E206D69736D617463682032
:1008A000002C20002C2000203A2073796E635F70AA
:1008B0006C616E5F706F736974696F6E0A002020DF
:1008C00063757272656E745F706F736974696F6E51
:1008D0003D00656E7175657565696E672022004B18
:1008E000494C4C45442E200053544F505045442E03
:1008F00020005072696E7465722073746F70706539
:10090000642064756520746F206572726F72732E37
:100910002046697820746865206572726F72206164
:100920006E6420757365204D39393920746F2072DB
:100930006573746172742E202854656D70657261E0
:10094000747572652069732072657365742E205307
:1009500065742069742061667465722072657374B1
:10096000617274696E67290A004E6F20436865637F
:100970006B73756D2077697468206C696E65206E85
:10098000756D6265722C204C617374204C696E65C4
:100990003A20004E6F20436865636B73756D207756
:1009A000697468206C696E65206E756D6265722C65
:1009B000204C617374204C696E653A200063686551
:1009C000636B73756D206D69736D617463682C2042
:1009D0004C617374204C696E653A20004C696E65F9
:1009E000204E756D626572206973206E6F74204CA5
:1009F000617374204C696E65204E756D6265722B53
:100A0000312C204C617374204C696E653A20004D86
:100A1000313130004D3331002F2F616374696F6EB7
:100A20003A66696E6973680A0053442072656164AE
:100A3000206572726F720A00446F6E652070726971
:100A40006E74696E672066696C650A0020496E766F
:100A5000616C696420657874727564657220000049
:100A600000000000000000000000000000D2420072
:100A700000F0420000C8420A20736F66745F656E22
:100A80006473746F705F6D6178203D20000A20737D
:100A90006F66745F656E6473746F705F6D696E20EE
:100AA0003D20000A20706F736974696F6E5F736810
:100AB000696674203D200020617869733A0A2068D5
:100AC0006F6D655F6F6666736574203D2000466FCD
:100AD0007220003C3C3C20646F5F626C6F636B690A
:100AE0006E675F6D6F76655F746F0A003E3E3E20F5
:100AF000646F5F626C6F636B696E675F6D6F766565
:100B00005F746F00203A2073657475705F666F7252
:100B10005F656E6473746F705F6F725F70726F6227
:100B2000655F6D6F76650A00202063757272656E71
:100B3000745F706F736974696F6E3D00203A206353
:100B40006C65616E5F75705F61667465725F656E1E
:100B50006473746F705F6F725F70726F62655F6DE8
:100B60006F76650A00202063757272656E745F701F
:100B70006F736974696F6E3D00646F5F70726F624E
:100B8000655F726169736528006465706C6F793A9E
:100B90002000203A207365745F70726F62655F6435
:100BA00065706C6F7965640A0020206375727265E8
:100BB0006E745F706F736974696F6E3D00203A20C8
:100BC0003C3C3C20646F5F70726F62655F6D6F7656
:100BD000650A00202063757272656E745F706F73B2
:100BE0006974696F6E3D00203A203E3E3E20646F7E
:100BF0005F70726F62655F6D6F76650A00202063BB
:100C0000757272656E745F706F736974696F6E3D33
:100C10000072657365745F6265645F6C6576656CB0
:100C20000A00486F6D696E67206661696C656400D3
:100C30000000000000000000BBBCBD9F9E00000043
:100C400000000000000000000000000000004572ED
:100C500072657572206465207265746F757200002C
:100C600000000000486F6D696E67206765736368F8
:100C700065697465727400000000686F6D696E6765
:100C80002066616C6C6F0000000000000000000036
:100C9000486F6D652066616C6C69746F00000000C0
:100CA000000000000000486F6D696E672066616992
:100CB0006C6564000000000000000000486F6D6972
:100CC0006E672066616C686F7500000000000000B0
:100CD0000000486F6D696E67206973206D69736CE1
:100CE000756B740000000000486F6D696E672062CC
:100CF000617361726973697A206F6C6475008FE546
:100D000020D0D1EC20BEF500000000000000000063
:100D100000000000D0BDD0B520D183D0B4D0B0D079
:100D2000BBD0BED181D18C0000003C3C3C20646F24
:100D30005F686F6D696E675F6D6F766528005B0039
:100D4000290A002C20002C20003E3E3E20646F5FCC
:100D5000686F6D696E675F6D6F766528004D6F76A1
:100D6000696E672E2E2E00000000000000000000BB
:100D70000000C1B22E2E2E00000000000000000076
:100D8000000000000000004465706C6163656D65E3
:100D90006E742E2E2E00000000000000496E2042CE
:100DA00065776567756E672E2E2E000000000000C7
:100DB000004D6F7669656E646F2E2E2E0000000068
:100DC000000000000000496E206D6F76696D656E51
:100DD000746F2E2E2E000000000000B2C4DEB3C1DE
:100DE000ADB30000000000000000000000000000A3
:100DF0004D6F7665722D7365202E2E2E000000003B
:100E00000000000000566572706C61617473656E5D
:100E10002E2E2E000000000000004B6F6E756D6CD2
:100E2000616E69796F722E2E2E000000000000D4D2
:100E3000972E2E2E00000000000000000000000091
:100E400000000000D094D0B2D0B8D0B6D0B5D0BC9D
:100E5000D181D18F2E2E2E00002020202020200096
:100E60005A005900202020200058002003000320B1
:100E70000009200000000000000000000000000049
:100E80007FFFE00000000FE7CC10203C0000007066
:100E900000E000000001010A105042000000630C55
:100EA00060000000010109105002000000470E2000
:100EB0000000000101089088020000004F0F200090
:100EC000000001010890880C0000005F0FA00000E6
:100ED000000101089104300000005E07A07F80003F
:100EE00001010851FC40000000406020FFC00001EB
:100EF000010832024000000040F020FFC00001075E
:100F0000C812027E00000040F020FFC00000000078
:100F10000000000000004060207F80000000000012
:100F200000000000005E07A07F8000E3878F1C891F
:100F3000F3E780005F0FA0FFC00012444888C8425A
:100F40000440004F0F20FFC00012244888A842042C
:100F50004000470E20FFC00062278F08A843E780AB
:100F600000630C603F000012240A08A8420500003C
:100F70007000E01E00001244090898420480007FBF
:100F8000FFE00C0000E384089C8843E4400000007C
:100F9000000000000000000000000000007FFFE0F3
:100FA0000000000FE7CC10203C0000007000E000C3
:100FB000000001010A10504200000061F8600000CA
:100FC0000001010910500200000041F8200000005B
:100FD00001010890880200000040F020000000019C
:100FE000010890880C000000406020000000010112
:100FF000089104300000005801A07F800001010822
:1010000051FC400000005C63A0FFC00001010832F9
:1010100002400000005EF7A0FFC0000107C81202F6
:101020007E0000005EF7A0FFC0000000000000008E
:101030000000005C63A07F80000000000000000052
:1010400000005801A07F8000E3878F1C89F3E780B0
:1010500000406020FFC00012444888C8420440009D
:1010600040F020FFC00012244888A84204400041FC
:10107000F820FFC00062278F08A843E7800061F8CE
:10108000603F000012240A08A8420500007000E03A
:101090001E00001244090898420480007FFFE00C03
:1010A0000000E384089C8843E44000000000205ACC
:1010B0000020590041424C2041646A7573746D658B
:1010C0006E742058002028656E61626C6564290A80
:1010D00000202864697361626C6564290A003350DA
:1010E0004F494E54004175746F20426564204C6531
:1010F00076656C696E673A2000204E6F7A7A6C656F
:10110000290A0020262041626F76650020262053A0
:10111000616D65205A2061730020262042656C6F46
:1011200077002028416C69676E6564205769746890
:1011300000205A3A0020593A0050726F6265204FE1
:10114000666673657420583A004649585F4D4F559E
:101150004E5445445F50524F42450A0050726F62F0
:10116000653A200043617274657369616E0A004DCF
:10117000616368696E6520547970653A20003C3C73
:101180003C204732390A00203A2047323920636F29
:10119000727265637465642058595A0A002020638E
:1011A000757272656E745F706F736974696F6E3D8E
:1011B00000202044697363726570616E63793A0040
:1011C00020204D61747269783A005A2066726F6D02
:1011D0002050726F62653A00203A204732392075FC
:1011E0006E636F727265637465642058595A0A00A1
:1011F000202063757272656E745F706F73697469B5
:101200006F6E3D000A0A426564204C6576656C206D
:10121000436F7272656374696F6E204D6174726999
:10122000783A00203A203E2070726F62696E672023
:10123000636F6D706C6574650A002020637572724F
:10124000656E745F706F736974696F6E3D003E20E8
:10125000332D706F696E74204C6576656C696E67AE
:101260000A00202844525952554E2900473239204D
:101270004175746F20426564204C6576656C696EBB
:1012800067003F2856296572626F7365206C65762A
:10129000656C20697320696D706C61757369626C2F
:1012A000652028302D34292E0A003C3C3C20473252
:1012B000390A003E204175746F2D6C6576656C208F
:1012C0006E6F74206E65656465642C20736B697045
:1012D0000A00203A203E3E3E204732390A002020B4
:1012E00063757272656E745F706F736974696F6E27
:1012F0003D00486F74656E6420746F6F20636F6C7F
:10130000640A004D31303420543020533231300DD6
:101310000A4D3730312054300D0A4D3130342053CE
:10132000300D0A573130320053544550313A4C4F4A
:1013300041442046494C414D454E540000000000B8
:10134000000000000090203120B720E4AB92940010
:10135000000000000000000000000000000000008D
:101360000000312043686172676572206C652066F9
:10137000696C616D656E7400000000000000003152
:101380002046494C414D454E54204C4144454E0069
:101390000000000000000000000000003120636138
:1013A000726761722066696C616D656E746F0000B2
:1013B000000000000000000000312046494C414D73
:1013C000454E544F2044492043415249434F000069
:1013D00000000000000053544550313A4C4F414446
:1013E0002046494C414D454E54000000000000008D
:1013F000000000312046696C616D656E746F206479
:101400006520436172676100000000000000000079
:1014100031204C4141442046494C414D454E5400F9
:101420000000000000000000000000000031205912
:10143000554B2046494C414D454E54490000000053
:10144000000000000000000000003120FF883A206A
:10145000F79CA0F2209F9B0000000000000000000D
:10146000000000000000003120D09DD090D093D02B
:10147000A0D0A3D097D09AD0902046494C414D455A
:101480004E5400004E65787400000000000000001B
:101490000000000000000000F4F500000000000063
:1014A000000000000000000000000000436F6E74A8
:1014B000696E756572000000000000000000000009
:1014C000466F72747365747A656E000000000000E8
:1014D00000000000436F6E74696E75617200000059
:1014E0000000000000000000436F6E74696E7561BB
:1014F0000000000000000000000000004E6578744D
:1015000000000000000000000000000000000000DB
:1015100050726F78696D6F000000000000000000DD
:1015200000000000566F6C67656E64650000000087
:101530000000000000000000536F6E72616B6900D4
:1015400000000000000000000000000092EFBBBFA0
:10155000D3000000000000000000000000000000B8
:10156000D181D0BBD0B5D0B4D183D18ED189D0B800
:10157000D0B9000053544550323A494E5345525465
:10158000205344204341524400000000000000006A
:1015900000000000000090203220B720AAAB534486
:1015A000A800000000000000000000000000000093
:1015B00000000000000000003220494E5345525404
:1015C00020434152544520534400000000000000D5
:1015D00000000000000000000000322045524B4196
:1015E0004E4E542053442D4B4152544500000000B0
:1015F0000000000000000000000000003220496EE2
:10160000736572746172207461726A6574612053CB
:101610004400000000000000000000000000322034
:10162000494E53455249544120534420434152446A
:1016300000000000000000000000000000000000AA
:1016400053544550323A494E534552542053442046
:101650004341524400000000000000000000000070
:1016600000003220496E7365726972206361727482
:10167000616F2053440000000000000000000000E3
:10168000000000003220504C414154532053442D5F
:101690004B414152540000000000000000000000D7
:1016A0000000000000003220494E534552542053A0
:1016B00044204B4152540000000000000000000094
:1016C00000000000000000003220FF883A20534450
:1016D000ED9920B3D80000000000000000000000D9
:1016E000000000000000000000003220D092D181F4
:1016F000D182D0B0D0B2D18CD182D0B52053442D7C
:10170000D0BAD0B0D180D182D18300005072696E3E
:10171000742066726F6D20534400000000000000CA
:1017200000000000000000000000005344A8EEEF9D
:1017300000000000000000000000000000000000A9
:1017400000000000000000000000496D7072696D2B
:101750006572206465205344000000000000000012
:1017600000000000000000000053442D4B61727423
:101770006500000000000000000000000000000004
:101780000000000000000000496D7072696D697210
:10179000206465736465205344000000000000006D
:1017A000000000000000005374616D7061206461EE
:1017B0002053440000000000000000000000000072
:1017C0000000000000005344B6B0C4DEB6D7CCDF42
:1017D000D8DDC40000000000000000000000000090
:1017E0000000000000496D7072696D697220646FBD
:1017F0002053440000000000000000000000000032
:10180000000000005072696E742076616E205344AF
:1018100000000000000000000000000000000000C8
:1018200000000053442064656E2059617A64697237
:1018300000000000000000000000000000000000A8
:1018400000005344ED9920EB9E00000000000000D2
:101850000000000000000000000000000000000088
:1018600000D09FD0B5D187D0B0D182D18C20D1818A
:1018700020534420D0BAD0B0D180D182D18B000087
:1018800053544550333A43484F4943452046494C09
:1018900045000000000000000090203320B720CA5F
:1018A000F35344A88B8C00000000000000000000EF
:1018B0000000332043484F49582046494348494592
:1018C0005200000000000000000000332057414893
:1018D0004C44415445490000000000000000000055
:1018E0000000000033204172636869766F206465F0
:1018F00020656C656363696F6E00000000332046ED
:10190000494C45204449205343454C544100000074
:1019100000000000000053544550333A43484F49FB
:1019200043452046494C45000000000000000033BC
:10193000204172717569766F206465206573636FED
:101940006C6861000000000033204B45555A454249
:10195000455354414E4400000000000000000000C8
:10196000003320534543494D20444F535941534977
:10197000000000000000000000003320EFBBBFFFAC
:10198000883A20F4D720B5EF0000000000000000E6
:101990000000003320D092D0ABD091D09ED0A020B8
:1019A000D0A4D090D099D09BD0900000636C696394
:1019B0006B20746F2072657475726E006174207490
:1019C00068652073616D652074696D650034206DF4
:1019D0006F746F72732072756E6E696E67004D6FF3
:1019E000746F722054657374004D31380047312094
:1019F000582D313020592D3130205A202D313020B2
:101A0000452D3130204635303000473120583130B7
:101A100020593130205A3130204531302046353080
:101A20003000473120582D313020592D3130205A87
:101A3000202D313020452D313020463530300047C3
:101A4000312058313020593130205A313020453141
:101A50003020463530300047393220583020593058
:101A6000205A3020453020004D3330322050310094
:101A70005731303500576966690044697361626C9B
:101A800065204D656E75004D6F746F7200434C4F4D
:101A900055443A200049503A2000534E3A2000560F
:101AA000657273696F6E3A2000000000000000004C
:101AB00000000095963A20000000000000000000A1
:101AC0000000000000000056657273696F6E3A20D6
:101AD0000000000000000000000000417573667502
:101AE0006872756E673A2000000000000000005622
:101AF000657273696F6E3A200000000000000000FC
:101B000000000056657273696F6E653A2000000030
:101B10000000000000000056657273696F6E3A2085
:101B200000000000000000000000005665727361B4
:101B30006F3A200000000000000000000000005686
:101B400065727369653A2000000000000000000023
:101B5000000000537572756D3A200000000000000F
:101B600000000000000000AADF3A20000000000092
:101B70000000000000000000000000D092D0B5D1AD
:101B800080D181D0B8D18F3A200000000000004DF4
:101B9000616368696E6520496E666F000000000031
:101BA000000000BEA5ECED20202020200000000059
:101BB00000000000000000496E666F000000000099
:101BC00000000000000000000000004D6173636829
:101BD000696E656E696E666F000000000000004966
:101BE0006E666F726D6163696F6E000000000000C9
:101BF000000000496E666F726D617A696F6E6500F4
:101C0000000000000000004D616368696E652049B6
:101C10006E666F0000000000000000456D20666FDA
:101C2000726D6163616F0000000000000000004DF4
:101C3000616368696E652D696E666F000000000063
:101C40000000004D616B696E652042696C676973C5
:101C500069000000000000DCEC20E0AF00000000A4
:101C60000000000000000000000000D092D0B5D1BC
:101C700080D181D0B8D18F00000000000000004466
:101C80006F776E6C6F6164696E673A0000000000E8
:101C90000000000000828384E42020202020200017
:101CA000000000000000000000000054656C656347
:101CB00068617267656D656E743A0000000000002F
:101CC000005769726420686572756E746572676525
:101CD0006C6164656E3A0044657363617267616E3E
:101CE000646F3A00000000000000000000446F77BD
:101CF0006E6C6F61643A000000000000000000009C
:101D0000000000446F776E6C6F6164696E673A0023
:101D100000000000000000000042616978616E640C
:101D20006F3A0000000000000000000000000044C6
:101D30006F776E6C6F6164656E3A000000000000A2
:101D40000000000000496E64697269796F723A00A0
:101D5000000000000000000000000092CF9F9920CA
:101D6000E43A000000000000000000000000000055
:101D700000D097D0B0D0B3D180D183D0B7D0BAD073
:101D8000B03A00000000002000446F776E6C6F6175
:101D900064204661696C00000000000000000084BF
:101DA000E49F9E2020202020202000000000000032
:101DB000000000000054656C6563686172676572BD
:101DC000204661696C00000000000053636865698B
:101DD0007465726E0000000000000000000000004A
:101DE000004572726F72206465206465736361726E
:101DF00067610000000000536361726963612046FF
:101E000061696C00000000000000000000446F7772
:101E10006E6C6F6164204661696C00000000000018
:101E200000000046616C6861206E6F20646F776E01
:101E30006C6F61640000000000446F776E6C6F612E
:101E400064656E206D69736C756B740000000049E9
:101E50006E64697269796F723A00000000000000D8
:101E6000000000000092CF9F9920BEF50000000006
:101E70000000000000000000000000D0A1D0BAD097
:101E8000B0D187D0B0D182D18C204661696C00007E
:101E90000020005475726B69736800000000000038
:101EA000000000000000005475726B697368000048
:101EB0000000000000000000000000547572630084
:101EC00000000000000000000000000000000054BE
:101ED00075726B6973636800000000000000000009
:101EE000000000547572636F0000000000000000E5
:101EF00000000000000000547572636F00000000D5
:101F000000000000000000000000005475726B69C2
:101F10007368000000000000000000000000005492
:101F20007572636F000000000000000000000000F8
:101F30000000005475726B73000000000000000088
:101F4000000000000000005475726B0000000000EB
:101F500000000000000000000000005475726B6972
:101F6000736800000000000000000000000000D1C5
:101F700082D183D180D0B5D186D0BAD0B8D0B900C3
:101F80000000004475746368000000000000000059
:101F90000000000000000000000000447574636849
:101FA0000000000000000000000000000000000031
:101FB0000000004E6565726C616E646169730000BB
:101FC00000000000000000000000004E696564652C
:101FD000726C616E64697363680000000000000049
:101FE000000000486F6C616E6465730000000000C3
:101FF00000000000000000000000004F6C616E64F3
:102000006573650000000000000000000000000093
:1020100000000044757463680000000000000000C8
:102020000000000000000000000000486F6C616EBE
:102030006465730000000000000000000000000064
:102040000000004E656465726C616E647300000090
:102050000000000000000000000000466C656D6597
:102060006E6B6365000000000000000000000000CF
:102070000000004475746368000000000000000068
:102080000000000000000000000000D093D0BED08F
:10209000BBD0BBD0B0D0BDD0B4D181D0BAD0B8D035
:1020A000B90000506F72747567616C000000000029
:1020B000000000000000000000506F72747567613E
:1020C0006C00000000000000000000000000004C58
:1020D0006520506F72747567616C0000000000002D
:1020E0000000000000506F72747567616C000000A2
:1020F0000000000000000000000000506F727475C6
:10210000677565730000000000000000000000001B
:1021100000506F72746F67616C6C6F00000000009C
:1021200000000000000000506F72747567616C0061
:1021300000000000000000000000000000506F726E
:10214000747567616C000000000000000000000072
:10215000000000506F72747567616C000000000031
:10216000000000000000000000506F7274656B6991
:102170007A00000000000000000000000000005095
:102180006F72747567616C00000000000000000051
:102190000000000000D09FD0BED180D182D183D07A
:1021A000B3D0B0D0BBD0B8D18F00004A6170616E9F
:1021B0006573650000000000000000000000004A98
:1021C0006170616E65736500000000000000000032
:1021D0000000004A61706F6E6169730000000000CA
:1021E000000000000000004A6170616E697363685E
:1021F00000000000000000000000004A61706F6EE7
:10220000657361000000000000000000000000474E
:10221000696170706F6E65736500000000000000FA
:102220000000004A6170616E657365000000000087
:10223000000000000000004A61706F6E65730000CE
:1022400000000000000000000000004A6170616EA4
:102250007300000000000000000000000000004AC1
:1022600061706F6E636100000000000000000000FC
:102270000000004A6170616E657365000000000037
:1022800000000000000000D0AFD0BFD0BED0BDD154
:1022900081D0BAD0B8D0B9000000004B6F72656130
:1022A0006E00000000000000000000000000004B75
:1022B0006F7265616E000000000000000000000009
:1022C000000000436F7265656E00000000000000B2
:1022D000000000000000004B6F7265616E6973635F
:1022E0006800000000000000000000436F7265619C
:1022F0006E6F0000000000000000000000000043BE
:102300006F7265616E6F0000000000000000000049
:102310000000004B6F7265616E000000000000005D
:1023200000000000000000436F7265616E6F0000E6
:1023300000000000000000000000004B6F726561AB
:10234000616E730000000000000000000000004B00
:102350006F72656C69000000000000000000000062
:102360000000004B6F7265616E000000000000000D
:1023700000000000000000D09AD0BED180D0B5D0BF
:10238000B9D181D0BAD0B8D0B900004974616C69B4
:10239000616E000000000000000000000000004925
:1023A00074616C69616E00000000000000000000B4
:1023B0000000004974616C69656E6E650000000084
:1023C000000000000000004974616C69656E69736B
:1023D00063680000000000000000004974616C693F
:1023E000616E6F0000000000000000000000004966
:1023F00074616C69616E6100000000000000000003
:102400000000004974616C69616E0000000000000A
:10241000000000000000004974616C69616E6F008B
:1024200000000000000000000000004974616C69B9
:1024300061616E73000000000000000000000049B0
:1024400074616C79616E0000000000000000000003
:102450000000004974616C69616E000000000000BA
:1024600000000000000000D0B8D182D0B0D0BBD1B5
:102470008CD18FD0BDD0B5D18600005370616E690C
:10248000736800000000000000000000000000531E
:1024900070616E69736800000000000000000000B9
:1024A00000000045737061676E6F6C0000000000F3
:1024B000000000000000005370616E6973636800E3
:1024C0000000000000000000000000457370616E15
:1024D0006F6C0000000000000000000000000053CE
:1024E0007061676E6F6C610000000000000000000A
:1024F0000000005370616E69736800000000000006
:1025000000000000000000457370616E686F6C0091
:102510000000000000000000000000537061616EC8
:1025200073000000000000000000000000000049EF
:102530007370616E796F6C00000000000000000095
:102540000000005370616E697368000000000000B5
:1025500000000000000000D0B8D181D0BFD0B0D0C2
:10256000BDD181D0BAD0B8D0B900004765726D61D5
:102570006E000000000000000000000000000047A6
:1025800065726D616E000000000000000000000038
:10259000000000416C6C656D616E6400000000001D
:1025A00000000000000000446575747363686500F6
:1025B0000000000000000000000000416C656D613B
:1025C0006E00000000000000000000000000005449
:1025D0006564657363610000000000000000000096
:1025E0000000004765726D616E0000000000000091
:1025F00000000000000000416C656D616F0000008C
:1026000000000000000000000000004475697473C1
:102610000000000000000000000000000000004179
:102620006C6D616E6361000000000000000000003E
:102630000000004765726D616E0000000000000040
:1026400000000000000000D09DD0B5D0BCD0B5D1B6
:1026500086D0BAD0B8D0B9000000004672656E636B
:102660006800000000000000000000000000000002
:102670000000004672656E63680000000000000004
:1026800000000000000000000000004672616E6360
:1026900061697300000000000000000000000000FD
:1026A0000000004672616E7A6F73697363680000A0
:1026B00000000000000000000000004672616E6330
:1026C0006573000000000000000000000000000032
:1026D0000000004672616E636573650000000000D3
:1026E00000000000000000000000004672656E63FC
:1026F0006800000000000000000000000000000072
:102700000000004672616E63657300000000000007
:1027100000000000000000000000004672616E73BF
:1027200000000000000000000000000000000000A9
:102730000000004672616E73C4B17A6361000000EC
:1027400000000000000000000000004672656E639B
:102750006800000000000000000000000000000011
:10276000000000D0A4D180D0B0D0BDD186D183D01C
:10277000B7D181D0BAD0B8D0B9000052757373699F
:10278000616E000000000000000000000000005228
:1027900075737369616E00000000000000000000A6
:1027A0000000005275737365000000000000000017
:1027B00000000000000000527573736973636800C5
:1027C00000000000000000000000005275736F0060
:1027D00000000000000000000000000000000052A7
:1027E0007573736F0000000000000000000000001F
:1027F0000000005275737369616E000000000000F4
:1028000000000000000000527573736F00000000AC
:1028100000000000000000000000005275737369A2
:102820007363680000000000000000000000005218
:1028300075736361000000000000000000000000EC
:102840000000005275737369616E000000000000A3
:1028500000000000000000D180D183D181D181D05F
:10286000BAD0B8D0B90000000000004368696E65B6
:10287000736500000000000000000000000000433D
:1028800068696E65736500000000000000000000CC
:102890000000004368696E6F697365000000000006
:1028A000000000000000004368696E65736973638F
:1028B00068000000000000000000004368696E6FBF
:1028C00000000000000000000000000000000043C5
:1028D000696E6573650000000000000000000000E4
:1028E0000000004368696E65736500000000000029
:1028F000000000000000004368696E65730000007E
:1029000000000000000000000000004368696E65E0
:10291000736500000000000000000000000000439C
:10292000696E636500000000000000000000000008
:102930000000004368696E657365000000000000D8
:1029400000000000000000D09AD0B8D182D0B0D0F2
:10295000B9D181D0BAD0B8D0B90000456E676C69E2
:10296000736800000000000000000000000000008C
:1029700000456E676C69736800000000000000008D
:1029800000000000000000416E676C616973000088
:1029900000000000000000000000000000456E671D
:1029A0006C69736368000000000000000000000014
:1029B000000000496E676C657300000000000000B5
:1029C000000000000000000000496E676C65736540
:1029D00000000000000000000000000000000045B2
:1029E0006E676C6973680000000000000000000062
:1029F0000000000000496E676C6573000000000075
:102A00000000000000000000000000456E67656CDB
:102A10007300000000000000000000000000000043
:102A200000496E67696C697A636500000000000008
:102A300000000000000000456E676C6973680000CC
:102A400000000000000000000000000000D0B0D036
:102A5000BDD0B3D0BBD0B8D0B9D181D0BAD0B8D066
:102A6000B90000436F6E74726F6C000000000000CC
:102A700000000000000000D8D9EEEF0000000000C8
:102A80000000000000000000000000436F6E747240
:102A90006F6C6500000000000000000000000045B1
:102AA000696E7374656C6C756E67656E000000000E
:102AB000000000436F6E74726F6C00000000000035
:102AC00000000000000000436F6E74726F6C6C6F4A
:102AD0000000000000000000000000BADDC4DBB010
:102AE000D9000000000000000000000000000043CA
:102AF0006F6E74726F6C6F000000000000000000C9
:102B0000000000436F6E74726F6C000000000000E4
:102B1000000000000000004B6F6E74726F6C0000CC
:102B20000000000000000000000000E1C200000002
:102B3000000000000000000000000000000000D0C5
:102B40009DD0B0D181D182D180D0BED0B9D0BAD001
:102B5000B80000526573746F7265206465666175B4
:102B60006C74000000000000000000000000000085
:102B7000000000000000000000E7E8ADE9BEBF0073
:102B80000000000000000000000000000000000045
:102B900000000000000000000000000000000052E3
:102BA0006573746175726572207061722064656608
:102BB00061757400000000000000000000000000CB
:102BC00000000000005374616E6461726477657286
:102BD0007465206C6164656E0000000000000000F8
:102BE00000000000000000000000005265737461E6
:102BF0007572617220706F72206465666563746FB0
:102C000000000000000000000000000000000000C4
:102C10000052697072697374696E6120696D702EFB
:102C200000000000000000000000000000000000A4
:102C300000000000000000BEAFC3B2D8BEAFC400A9
:102C40000000000000000000000000000000000084
:102C5000000000000000000000000000005265734A
:102C60007461757261722070616472616F0000003E
:102C70000000000000000000000000000000000054
:102C80000000004865727374656C207374616E6433
:102C9000616172640000000000000000000000009C
:102CA0000000000000000000005661727361796945
:102CB0006C616E6120646F6E6475720000000000CC
:102CC000000000000000000000000000000000B64E
:102CD000E020E88BFC000000000000000000000085
:102CE00000000000000000000000000000000000E4
:102CF0000000000000D092D0BED181D181D182D01D
:102D0000B0D0BDD0BED0B2D0B8D182D18C20D0BD91
:102D1000D0B0D181D182D1802E00004C616E677518
:102D20006167650000000000000000000000000076
:102D300000000000008081BEBF2020202020202035
:102D40000000000000000000000000000000004C37
:102D500061206C616E677565000000000000000076
:102D6000000000000000000000537072616368659D
:102D70000000000000000000000000000000000053
:102D80000000004964696F6D6100000000000000F0
:102D9000000000000000000000000000006C696EF0
:102DA0006775616767696F00000000000000000040
:102DB000000000000000004C616E677561676500EF
:102DC0000000000000000000000000000000000003
:102DD000004C696E67756100000000000000000093
:102DE00000000000000000000000005461616C0061
:102DF00000000000000000000000000000000000D3
:102E0000000000000044696C0000000000000000A9
:102E1000000000000000000000000000000000C3EF
:102E2000C220B6E00000000000000000000000002A
:102E3000000000000000000000D184D0BED180D08E
:102E4000BCD183D0BBD0B8D180D0BED0B2D0BAD0A4
:102E5000B800005A204F6666736574205365747419
:102E6000696E6700000000BEBF5ACEC0C1000000FE
:102E700000000000000000000000005A204F6666BD
:102E80007365740000000000000000000000005A9C
:102E9000205665727361747A000000000000000023
:102EA00000000044657366617365205A00000000ED
:102EB000000000000000005A204F66667365740031
:102EC00000000000000000000000005AB5CCBEAFBA
:102ED000C4000000000000000000000000000044EA
:102EE000657376696F205A00000000000000000042
:102EF0000000005A204F66667365740000000000F1
:102F0000000000000000005A204F666673657400E0
:102F100000000000000000000000005A20CCB800B3
:102F2000000000000000000000000000000000D0D1
:102F3000A1D0BCD0B5D189D0B5D0BDD0B8D0B52046
:102F40005A000054656D7065726174757265000099
:102F50000000000000000000000000C9D2BEBF0059
:102F60000000000000000000000000000000000061
:102F700000000054656D70657261747572650000C3
:102F8000000000000000000000000054656D706546
:102F90007261747572000000000000000000000003
:102FA00000000054656D7065726174757261000097
:102FB000000000000000000000000054656D706516
:102FC0007261747572610000000000000000000072
:102FD000000000B5DDC4DE000000000000000000BD
:102FE000000000000000000000000054656D7065E6
:102FF0007261747572610000000000000000000042
:1030000000000054656D7065726174757572000022
:103010000000000000000000000000536963616BC5
:103020006C696B0000000000000000000000000060
:10303000000000CB9600000000000000000000002F
:103040000000000000000000000000D0A2D0B5D0B9
:10305000BCD0BFD0B5D180D0B0D182D183D180D007
:10306000B000004E6F7A7A6C65000000000000D35B
:10307000D4000000000000000000004275736500ED
:1030800000000000000000447573650000000000AF
:10309000000000426F7175696C6C610000000055A2
:1030A00067656C6C6F000000000000C9BDDED900D0
:1030B000000000000000004269636F000000000093
:1030C0000000004E6F7A7A6C650000000000004E30
:1030D0006F7A756C000000000000008FE5000000B2
:1030E00000000000000000D0A1D0BED0BFD0BBD0F7
:1030F000BE000043616E6E6F7420656E7465722051
:103100007375626469723A2000022E2E0050524993
:103110004E5420504155534544000000000000002B
:103120000000000000000000000000CAF3F1F220DF
:10313000202020200000000000000000000000000F
:10314000000000000000000000494D5052494D456C
:10315000522050415553454400000000000000003B
:1031600000000000000000445255434B20504155E0
:1031700053494552540000000000000000000000C8
:103180000000000000494D50522E2050415553413F
:1031900044410000000000000000000000000000AA
:1031A0000000005354414D504120494E205041559C
:1031B000534100000000000000000000000000007B
:1031C000005052494E542050415553454400000090
:1031D00000000000000000000000000000000049A6
:1031E0004D5052494D4952205041555341444F0092
:1031F0000000000000000000000000000041464404
:1032000052554B2047455041555A454552440000C0
:10321000000000000000000000000059415A44492D
:1032200052204455524455000000000000000000A8
:10323000000000000000000000EB9E20D7BDE4E687
:10324000000000000000000000000000000000007E
:1032500000000000000000D09FD0B5D187D0B0D1D1
:1032600082D18C20D0BDD0B020D0BFD0B0D183D0FF
:10327000B7D0B500004175746F20526574726163F8
:10328000742046696C616D656E740000000000007A
:103290000000000093E492942020202020000000F1
:1032A000000000000000000000000000000000001E
:1032B000000000446563686172676572206C652078
:1032C00066696C616D656E740000000000000000AE
:1032D000000046696C616D656E7420656E746C618A
:1032E00064656E00000000000000000000000000A7
:1032F0000072657472616363696F6E2066696C61E8
:103300006D656E746F00000000000000000000009A
:10331000536361726963612046696C616D656E74A7
:10332000000000000000000000000000000000CCD1
:10333000B2D7D2DDC420B1B3C40000000000000049
:1033400000000000000000000000000000005265C6
:1033500074726169722046696C616D656E746F008C
:103360000000000000000000000000000041757433
:103370006F20526574726163742046696C616D657B
:103380006E740000000000000000000046696C61DF
:103390006D656E746920476572692043656B000036
:1033A0000000000000000000000000F79CA0F220D8
:1033B000E9EB000000000000000000000000000039
:1033C00000000000000000000000D090D0B2D182C8
:1033D000D0BE20D092D182D18FD0B3D0B8D0B2D0CD
:1033E000B0D0BDD0B8D0B500004175746F2046652F
:1033F00065642046696C616D656E740000000000B4
:103400000000000000000000000000000000E4AB2D
:1034100092942020202020000000000000000000E6
:10342000000000000000000000000000000000009C
:1034300000000043686172676572206C65206669F0
:103440006C616D656E7400000000000000000000FB
:10345000000000000000000046696C616D656E743C
:10346000206C6164656E0000000000000000000038
:1034700000000000000000000000000000656E7405
:10348000726164612064652066696C616D656E744B
:103490006F000000000000000000000000000000BD
:1034A00000004361726963612066696C616D656EDD
:1034B000746F000000000000000000000000000029
:1034C00000000000000000CCB2D7D2DDC420B2DD85
:1034D00000000000000000000000000000000000EC
:1034E000000000000000000000000000416C696D59
:1034F000656E74652046696C616D656E74000000D0
:1035000000000000000000000000000000000000BB
:10351000004175746F20466565642046696C616D75
:10352000656E740000000000000000000000000054
:1035300000000000000059656D2046696C616D65F2
:103540006E74690000000000000000000000000030
:103550000000000000000000000000F79CA0F22026
:10356000B3D80000000000000000000000000000D0
:10357000000000000000000000000000000000004B
:10358000D097D0B0D0B3D180D183D0B7D0BAD0B09B
:1035900020D184D0B8D0BBD0B0D0BCD0B5D0BDD1B4
:1035A00082D0B000005075726765206D6F72650043
:1035B000000000000000000000000000000000000B
:1035C00000000000E4ABE0E1929400000000000085
:1035D00000000000000000000000000000000000EB
:1035E000000000507572676520706C7573000000F4
:1035F00000000000000000000000000000000000CB
:1036000000004D65687220656E746C656572656E4C
:1036100000000000000000000000000000000000AA
:1036200000707572676172206D61730000000000A8
:10363000000000000000000000000000000000008A
:103640004C696265726120646920706975000000D0
:10365000000000000000000000000000000000501A
:1036600075726765206D6F726500000000000000D4
:103670000000000000000000000000000000507585
:1036800072676172206D61697300000000000000C4
:1036900000000000000000000000000000507572F3
:1036A0006765206D65657200000000000000000085
:1036B000000000000000000000000000646168617C
:1036C00020746173666979652065740000000000EC
:1036D0000000000000000000000000E98320C0EBB3
:1036E00000000000000000000000000000000000DA
:1036F00000000000000000000000D09ED187D0B87C
:10370000D181D182D0B8D182D18C20D0B1D0BED0DD
:10371000BBD18CD188D0B50000436F6E74696E75D3
:10372000650000000000000000000000000000F440
:10373000F500000000000000000000000000000094
:103740000000000000436F6E74696E7565720000C2
:103750000000000000000000000000447275636B70
:103760006520776569746572000000000000000044
:1037700000536567756972000000000000000000DA
:103780000000000000000052697072656E646920DC
:103790007374616D706100000000000000CCDFD820
:1037A000DDC4BBB2B6B200000000000000000000A3
:1037B0000000005265746F6D617220696D707265F2
:1037C0007373616F000000000048657276617420B9
:1037D0007072696E7400000000000000000000427A
:1037E00061736B697969207375726475720000008A
:1037F000000000000088BA00000000000000000087
:103800000000000000000000000000D09FD180D028
:10381000BED0B4D0BED0BBD0B6D0B8D182D18C008F
:1038200000524553554D45204F5054494F4E533A41
:10383000000000000000F4F5FEFF20202020200002
:1038400000000000000000000000004F5054494FED
:103850004E5320444520524550524953453A0000AA
:10386000464F5254532E204F5054494F4E454E3AD6
:1038700000000000004F50432E205245494E49435E
:10388000494F3A000000000000004F505A494F4E87
:10389000493A000000000000000000000000005253
:1038A0004553554D45204F5054494F4E533A000013
:1038B000000000004F50434F4553204445205245DF
:1038C00053554D4F3A00000000524553554D452089
:1038D0004F50544945533A00000000000000444551
:1038E00056414D20534543454E454B4C4552493A70
:1038F000000000CCB920D0B03A0000000000000069
:103900000000000000000000D09FD090D0A0D09018
:10391000D09CD095D0A2D0A0D0AB3A000063686113
:103920006E6765000000000000000000000000005D
:103930000000FEFF2020000000000000000000004A
:10394000000000000000006368616E67656D656ED1
:1039500074000000000000000000000046696C6177
:103960006D656E747765636873656C730000000045
:103970000064652066696C616D656E746F0000009F
:1039800000000000000064692066696C616D656E6E
:10399000746F000000000000000000200000000024
:1039A0000000000000000000000000000000000017
:1039B00064652066696C616D656E746F000000005F
:1039C000000000000076657277697373656C656E40
:1039D0000000000000000000000064656769736972
:1039E0006D6900000000000000000000000000AE53
:1039F0008700000000000000000000000000000040
:103A000000000000D181D0BCD0B5D0BDD18B20D07A
:103A1000BDD0B8D182D0B800006F66207468652030
:103A200066696C616D656E74000000000092942000
:103A30002000000000000000000000000000000066
:103A40000064752066696C616D656E74000000002D
:103A500000000000005374617274206465730000FC
:103A6000000000000000000000656C2063616D62D2
:103A7000696F000000000000000000000064656C39
:103A80002063616D62696F000000000000000000AB
:103A900000BCCADED7B8B5CFC1B8C0DEBBB200002B
:103AA00000000000006461206D7564616E63610058
:103AB00000000000000000000066696C616D656E2A
:103AC0007420746500000000000000000066696C4E
:103AD000616D616E696E0000000000000000000072
:103AE00000F79CA0F20000000000000000000000B1
:103AF0000000000000D0BDD0B0D187D0B0D0BBD086
:103B0000B000000000000000005761697420666F7B
:103B100072207374617274000000000000FCFDB339
:103B2000B420202020200000000000000000000041
:103B300000417474656E64657A2064656275740012
:103B40000000000000576172746520617566206492
:103B5000656E00000000000000457370657265200E
:103B6000612071756520636F6D69656E6341747462
:103B7000656E6465726520617676696F000000008D
:103B800000BAB3B6DDA6B6B2BCBCCFBD0000000023
:103B9000000000000041677561726465206F206954
:103BA0006E6963696F000000005761636874207676
:103BB0006F6F722073746172740000000042617351
:103BC0006C616D612062656B6C656E69796F720006
:103BD00000BDDA000000000000000000000000004E
:103BE0000000000000D094D0BED0B6D0B4D0B8D180
:103BF00082D0B5D181D18C000020000000000000EF
:103C00000000000000000000000000000020000094
:103C100000000000000000000000000000000000A4
:103C20000064752066696C616D656E74000000004B
:103C300000000000006465732046696C616D656E6C
:103C400074732E2E2E00000000656C2066696C6176
:103C50006D656E746F000000000000000064656C0C
:103C60002066696C616D656E746F00000000000075
:103C70000020000000000000000000000000000024
:103C8000000000000066696C616D656E746F000075
:103C90000000000000000000007465206C61646595
:103CA0006E00000000000000000000000020000086
:103CB0000000000000000000000000000000000004
:103CC00000000000000000000000000000000000F4
:103CD0000000000000D0BDD0B8D182D0B8000000F4
:103CE00000000000000000000066696C616D656EF8
:103CF0007420756E6C6F6164000000000093E492A4
:103D0000942020202020000000000000000000007F
:103D10000064656368617267656D656E74000000BC
:103D200000000000004865726175736E61686D6522
:103D300000000000000000000073652064657363EC
:103D4000617267756500000000000000006C276567
:103D50007370756C73696F6E650000000000000081
:103D600000BCCADED7B8B5CFC1B8C0DEBBB2000058
:103D700000000000006465736361727265676172C0
:103D800000000000000000000066696C616D656E57
:103D90007420756974000000000000000066696C02
:103DA000616D616E696E2063696B6D61736900009E
:103DB00000F79CA0F220E9EB0000000000000000EA
:103DC0000000000000D0B2D18BD0B3D180D183D01D
:103DD000B7D0BAD0B8000000005761697420666F90
:103DE00072000000000000000000000000FCFD2048
:103DF00020000000000000000000000000000000A3
:103E000000417474656E64657A2000000000000053
:103E10000000000000576172746520617566000043
:103E2000000000000000000000457370657265200E
:103E3000612071756500000000000000004174748D
:103E4000656E6465726500000000000000000000FF
:103E500000CCA8D7D2DDC4C7B7C0DEBCC1ADB300AB
:103E6000000000000045737065726172207061721D
:103E70006100000000000000005761636874207654
:103E80006F6F720000000000000000000042656BD0
:103E90006C656E69796F7200000000000000000020
:103EA00000938B00000000000000000000000000F4
:103EB0000000000000D094D0BED0B6D0B4D0B8D1AD
:103EC00082D0B5D181D18C00002000506C65617327
:103ED0006520776169742E2E2E000000000000001E
:103EE0000000FCFD2E2E2E202020200000000000CF
:103EF000000000000000000000417474656E6465FD
:103F00007A2C205356502E2E2E0000000000000068
:103F100042697474652077617274656E2E2E2E006E
:103F20000000000000000045737065726520706F2E
:103F300072206661766F720000000000000041741C
:103F400074656E646572652E2E2E00000000000000
:103F50000000000000506C65617365207761697432
:103F60002E2E2E000000000000000000506F722076
:103F70006661766F722C2065737065726500000053
:103F8000000000576163687420612E752E622E0058
:103F9000000000000000000000004C757466656EB3
:103FA0002042656B6C6579696E2E2E2E0000000034
:103FB00000DBBD208B92A0B7CE2E2E2E000000007D
:103FC0000000000000000000D09FD0BED0B4D0BEE2
:103FD000D0B6D0B4D0B8D182D0B52E2E2E000048A5
:103FE000656174696E67206E6F7A7A6C6500000097
:103FF0000000000000000000000000000000C3C43A
:10400000D3D4202020202000000000000000000069
:104010000000000000000000000000000043686194
:1040200075666661676520646573206275736500F7
:1040300000000000000000000000000044757365EF
:10404000206865697A74206175662E2E2E00000046
:10405000000000000000000000000043616C656E7D
:1040600074616E646F20626F7175696C6C610000C1
:104070000000000000000000000052697363616CE2
:10408000642E207567656C6C6F00000000000000F6
:1040900000000000000000000048656174696E6760
:1040A000206E6F7A7A6C650000000000000000004E
:1040B00000000000000000004269636F206465207A
:1040C0006171756563696D656E746F000000000055
:1040D000000000000000004E6F7A7A6C6520766563
:1040E00072772E00000000000000000000000000B9
:1040F0000000000000004E6F7A756C204973696EF5
:1041000069796F72000000000000000000000000EC
:1041100000000000008FE52083C820E400000000BC
:10412000000000000000000000000000000000008F
:1041300000000000D09ED182D0BED0BFD0BBD0B591
:10414000D0BDD0B8D0B520D181D0BED0BFD0BBD0EB
:10415000BE0000200068656174206E6F7A7A6C651D
:104160002E00000000000000000000000000000021
:10417000C3C4D3D420202020200000000000000071
:104180000000000000000000000000706F75722049
:104190006368617566666572206C6120627573651F
:1041A00000000000000044757365206175667A7533
:1041B0006865697A656E2E0000000000000000004E
:1041C0000043616C656E746172206C6120626F7176
:1041D00075696C6C61000000000000007269736317
:1041E000616C64207567656C6C6F2E0000000000C8
:1041F0000000000000000068656174206E6F7A7A2C
:104200006C652E00000000000000000000000000AF
:104210000000706172612061717565636572206F65
:1042200020626F63616C0000000000000076657220
:10423000772E206E6F7A7A6C652E000000000000E9
:1042400000000000000000004275746F6E612042A3
:1042500061732E000000000000000000000000005C
:104260000000008FE52083C800000000000000006F
:104270000000000000000000000000000000D187E6
:10428000D182D0BED0B1D18B20D0BDD0B0D0B3D1EF
:1042900080D0B5D182D18C000050726573732062DA
:1042A0007574746F6E20746F0000000000000000D1
:1042B000000000000000008E8FB3B42020202020DA
:1042C00000000000000000000000000000000000EE
:1042D000000000000050726573736572206C6520E9
:1042E000626F75746F6E2E2E2E00000000000000AD
:1042F0000000004B6E6F706620647275636B656EB4
:1043000020756D00000000000000000000000000AB
:104310000050726573696F6E6520C3A96C20626F6F
:10432000746F6E2070617261000000000000005028
:1043300072656D6920706572000000000000000069
:104340000000000000000000000000000050726546
:10435000737320627574746F6E20746F00000000B8
:104360000000000000000000000000507265737340
:10437000696F6E65206F20626F74616F00000000CE
:104380000000000000000000004B6C696B206B6EA9
:104390006F70206F6D2E2E2E0000000000000000B8
:1043A000000000000000004E6F7A756C75204973A4
:1043B00069746D616B206963696E00000000000024
:1043C0000000000000AAF3D22090A0BDA0000000D1
:1043D00000000000000000000000000000000000DD
:1043E000000000D09DD0B0D0B6D0BCD0B8D182D023
:1043F000B520D0BAD0BDD0BED0BFD0BAD1832C00AA
:1044000000746F20636F6E74696E75652E2E2E00BA
:10441000000000000020000000000000000000007C
:10442000000000000000000000706F757220636FD4
:104430006E74696E7565722E2E2E000000647275A2
:10444000636B656E2E2E2E00000000000000000041
:10445000007061726120636F6E74696E7561722E97
:104460002E2E0000007072656D69207065722063E9
:104470006F6E7400000000000020000000000000CB
:1044800000000000000000000000000000706172E9
:104490006120636F6E74696E7561722E2E2E00003E
:1044A000006F6D207665726465722E2E2E000000FE
:1044B000000000000074757361206261732E2E2E5F
:1044C00000000000000000000088BA0000000000AA
:1044D00000000000000000000000000000D0BAD082
:1044E000BDD0BED0BFD0BAD1830000000000000014
:1044F00000616E6420707265737320627574746FEE
:104500006E000000008D8E8FF4F5202020202020EA
:1045100020000000000000000065742070726573C8
:10452000736572206C6520626F75746F6E756E6452
:10453000204B6E6F7066000000000000000000005D
:1045400000792070726573696F6E6520656C2062FA
:104550006F746F6E0066696C616D656E746F206557
:10456000000000000000000000B8D8AFB8BDD9C4FA
:10457000BFDEAFBAB3BCCFBD0000000000707265F3
:104580007373696F6E65206F20626F74616F0000D6
:1045900000656E206472756B206B6E6F700000009A
:1045A0000000000000766520646576616D20696317
:1045B000696E000000000000008AA08920AAF3D2E2
:1045C0002090A0B7CE0000000000000000D0B8206E
:1045D000D0BDD0B0D0B6D0BCD0B8D182D0B500005C
:1045E00000496E736572742066696C616D656E74E6
:1045F000000000000000000000000000AAAB929440
:1046000020202020202020000000000000000000CA
:1046100000000000000000496E736572657A206C2E
:10462000652066696C616D656E74000000000000B5
:10463000000046696C616D656E742065696E6C651D
:1046400067656E00000000000000000000496E7306
:10465000657274652066696C616D656E746F0000CB
:104660000000000000000000496E7365726973630A
:104670006920696C000000000000000000000000DC
:10468000000000CCA8D7D2DDC4A6BFB3C6ADB3BC72
:104690002C00000000000000000000000000496E37
:1046A000736972612066696C616D656E746F2065F7
:1046B0000000000000000000004C61616420666999
:1046C0006C616D656E740000000000000000000069
:1046D0000000000046696C616D616E692079756B40
:1046E0006C6500000000000000000000000000F702
:1046F0009CA0F220B3D800000000000000000000E1
:1047000000000000000000000000D092D181D182A2
:10471000D0B0D0B2D18CD182D0B520D0BDD0B8D15C
:1047200082D18C000020000000000000000000008A
:104730000000000000000000002000000000000059
:104740000000000000000000000000000020000049
:104750000000000000000000000000000000000059
:104760000020000000000000000000000000000029
:104770000000000000200000000000000000000019
:1047800000000000000000000064656C2066696C99
:10479000616D656E746F0000000000000020000075
:1047A0000000000000000000000000000000000009
:1047B00000200000000000000000000000000000D9
:1047C00000000000006C6164656E000000000000E5
:1047D00000000000000000000020000000000000B9
:1047E00000000000000000000000000000200000A9
:1047F00000000000000000000000000000000000B9
:104800000020000000000000000000000000000088
:10481000000000000066696C616D656E74206C6F4D
:1048200061640000000000000000000000000000C3
:10483000E4AB929420202020200000000000000023
:1048400000000000000000000000006475206669A0
:104850006C616D656E7400000000000000000000D7
:104860000000000000004C6164656E206465730008
:104870000000000000000000000000000000000038
:104880000064652066696C616D656E746F00000080
:10489000000000000000000000000000696C2063C0
:1048A00061726963616D656E746F000000000000E5
:1048B00000000000000000BCCADED7B8B5CFC1B808
:1048C000C0DEBBB2000000000000000000000000DD
:1048D000000064652066696C616D656E746F000030
:1048E0000000000000000000000000000066696C8D
:1048F000616D656E742074650000000000000000AA
:10490000000000000000000066696C616D616E6966
:104910006E2079756B6C656E6D65736900000000C3
:10492000000000F79CA0F220B3D8000000000000B7
:104930000000000000000000000000000000D0B7F0
:10494000D0B0D0B3D180D183D0B7D0BAD0B820D036
:10495000BDD0B8D182D0B800005761697420666FAD
:1049600072000000000000000000000000FCFD20BC
:104970002000000000000000000000000000000017
:1049800000417474656E647265206C6120636861B7
:10499000726765000057617274652061756600007A
:1049A0000000000000000000004573706572617235
:1049B000206C6120636172676100000000417474C3
:1049C000656E646572650000000000000000000074
:1049D00000CCA8D7D2DDC4BFB3C3DDC1ADB30000E6
:1049E000000000000041677561726465206120630A
:1049F000617267610000000000576163687420768F
:104A00006F6F720000000000000000000042656B44
:104A10006C656E69796F7200000000000000000094
:104A200000938B20E4000000000000000000000064
:104A30000000000000D094D0BED0B6D0B4D0B8D121
:104A400082D0B5D181D18C000020204E6F7A7A6C53
:104A5000653A200000000000000000000020D3D4D0
:104A6000C9D23A0000000000000000000000000071
:104A7000002020427573653A20000000000000000D
:104A800000000000002020447573653A20000000FB
:104A900000000000000000000020426F7175696C8A
:104AA0006C613A000000000000000000002020556A
:104AB00067656C6C6F3A2000000000000000000089
:104AC0000020204E6F7A7A6C653A200000000000CA
:104AD00000000000002020426F63616C3A2020003B
:104AE00000000000000000000020204E6F7A7A6C69
:104AF000653A200000000000000000000020204E69
:104B00006F7A756C3A200000000000000000000081
:104B10000020208FE53A2000000000000000000087
:104B20000000000000D09DD0B0D181D0B0D0B4D072
:104B3000BAD0B03A000000000020000000000000E1
:104B40000000000000000000000000000020000045
:104B50000000000000000000000000000000000055
:104B60000020000000000000000000000000000025
:104B7000000000000046696C616D656E7473000092
:104B80000000000000000000002000000000000005
:104B90000000000000000000000000000064656CE0
:104BA0002066696C616D656E746F00000000000026
:104BB00000200000000000000000000000000000D5
:104BC00000000000002000000000000000000000C5
:104BD00000000000000000000020000000000000B5
:104BE0000000000000000000000000000062656B93
:104BF0006C6579696E000000000000000000000094
:104C00000020000000000000000000000000000084
:104C10000000000000200000000000000000000074
:104C200000000000000000000066696C616D656EA8
:104C300074207075726765000000000000000000BD
:104C4000FCFDE4AB2020200000000000000000007C
:104C50000000000000000064752066696C616D65ED
:104C60006E74000000000000000000000000456EAF
:104C7000746C656572656E206465730000000000E9
:104C8000000000000064656C2066696C616D656EF3
:104C9000746F000000000000000000006C6F2073C3
:104CA000707572676F0000000000000000000000D7
:104CB00000000066696C616D656E742070757267C6
:104CC00065000000000000000000646F2066696C51
:104CD000616D656E746F0000000000000000000050
:104CE0000066696C616D656E747265696E6967698D
:104CF0006E6700000000000074656D697A6C69677A
:104D0000696E69000000000000000000000000F76C
:104D10009CA0F220C0EB000000000000000000009A
:104D2000000000000000D187D0B8D181D182D0BA74
:104D3000D0B820D0BDD0B8D182D0B80000576169BA
:104D40007420666F72000000000000000000000088
:104D50000020000000000000000000000000000033
:104D60000000000000417474656E64657A206C6117
:104D7000207075726765000000576172746520616C
:104D80007566000000000000000000000045737020
:104D900065726172206C612070757267610000003D
:104DA00000417474656E6465726500000000000067
:104DB00000000000005761697420666F72000000F7
:104DC000000000000000000000416775617264652A
:104DD0002061206C696D70657A6100000057616325
:104DE0006874206F700000000000000000000000E8
:104DF0000046696C616D656E740000000000000083
:104E00000000000000200000000000000000000082
:104E1000000000000000000000D094D0BED0B6D04A
:104E2000B4D0B8D182D0B5D181D18C00002000009F
:104E30000000000000000000000000000000000072
:104E40000020000000000000000000000000000042
:104E50000000000000200000000000000000000032
:104E6000000000000000000000447275636B657371
:104E70002E2E2E0000000000000000000020000088
:104E80000000000000000000000000000000000022
:104E90000064656C6C61207374616D70610000006A
:104EA00000000000002000000000000000000000E2
:104EB00000000000000000000020000000000000D2
:104EC00000000000000000000000000000746520E9
:104ED0006761616E0000000000000000000000003B
:104EE0000062656B6C6500000000000000000000BF
:104EF0000000000000200000000000000000000092
:104F0000000000000000000000D180D0B5D0B7D173
:104F10008ED0BCD0B50000000000000000746F20EF
:104F2000726573756D6500000000000000000000F0
:104F300000E7E8CAF3202020200000000000000065
:104F40000000000000706F75722072657072656EEF
:104F5000647265000000000000466F72747365742F
:104F60007A756E672064657300000000006C612034
:104F7000696D70726573696F6E000000000000005B
:104F8000006C61207269707265736100000000003E
:104F90000000000000BCCADED7B8B5CFC1B8C0DE83
:104FA000BBB20000000000000073657220726574DF
:104FB0006F6D61646100000000000000006F6D20F3
:104FC0007665726465720000000000000000000059
:104FD00000737572647572756C6D6573696E6900C6
:104FE0000000000000DD84F9919200000000000044
:104FF000000000000000000000D0BFD0B5D187D075
:10500000B0D182D18C20D0BDD0B0000000576169F2
:105010007420666F72207072696E74000000000068
:105020000000000000000000000000FCFD20200047
:105030000000000000000000000000000000000070
:10504000000000000000000000417474656E64659B
:105050007A20717565206C27696D7072657373694C
:105060006F6E000000000057617274652061756604
:105070000000000000000000000000000000000030
:1050800000000000004573706572616E646F2071EE
:105090007565207365207265616E7564650000003A
:1050A000000000417474656E646572650000000064
:1050B00000000000000000000000000000000000F0
:1050C00000CCDFD8DDC4A6BBB2B6B2BCCFBD0000F9
:1050D000000000000000000000000000000000418F
:1050E000677561726465206120696D7072657373A4
:1050F000616F0000000000000000000000576163C5
:10510000687420766F6F72207072696E7400000090
:1051100000000000000000000000004261736B69A5
:105120006E696E000000000000000000000000003A
:10513000000000000000000000EB9E20938B0000A8
:10514000000000000000000000000000000000005F
:1051500000000000000000D09FD0BED0B4D0BED070
:10516000B6D0B4D0B8D182D0B52C20D0BFD0BED06C
:10517000BAD0B000004D32342053256C6420542541
:105180006C64004D3233202573005A3A00473238A0
:105190002052302058205900436172642072656D9E
:1051A0006F76656400000000000000000000000051
:1051B00000000000000000A8A9ACAD000000000045
:1051C00000000000000000000000000000000000DF
:1051D00000000000000063617274652072657469EC
:1051E0007265650000000000000000000000000083
:1051F000000000000053442D4B6172746520656E01
:10520000746665726E74000000000000000000000B
:10521000000000005461726A6574612065787472E0
:1052200061696461000000000000000000000000EF
:10523000000000534420436172642072696D6F73F3
:10524000736100000000000000000000000000008A
:105250000000B6B0C4DEB6DEB1D8CFBEDD000000BF
:10526000000000000000000000000000000000003E
:105270000043617274616F2072656D6F7669646F4F
:10528000000000000000000000000000000000001E
:105290004B616172742076657277696A64657264C5
:1052A00000000000000000000000000000000053AB
:1052B000442063696B6172696C64692E00000000B0
:1052C0000000000000000000000000000000534447
:1052D000ED9920E18598000000000000000000002A
:1052E00000000000000000000000000000D09AD084
:1052F000B0D180D182D0B020D0B8D0B7D0B2D0BB9E
:10530000D0B5D187D0B5D0BDD0B0000043617264B4
:1053100020696E736572746564000000000000000F
:105320000000000000000000000000A8A9AAAB00D7
:10533000000000000000000000000000000000006D
:10534000000000000000000000006361727465202E
:10535000696E736572656500000000000000000062
:1053600000000000000000000053442D4B617274E7
:10537000652065726B616E6E7400000000000000B5
:1053800000000000000000005461726A6574612032
:10539000696E736572746164610000000000000052
:1053A0000000000000000053442043617264206943
:1053B0006E736572697461000000000000000000F7
:1053C000000000000000B6B0C4DEB6DEBFB3C6AD5C
:1053D000B3BBDACFBCC0000000000000000000003A
:1053E000000000000043617274616F20696E736594
:1053F0007269646F000000000000000000000000FF
:10540000000000004B6161727420696E67657374FF
:105410006F6B656E000000000000000000000000DF
:105420000000005344205965726C657374692E0046
:10543000000000000000000000000000000000006C
:1054400000005344ED9920B3D8982E0000000000CE
:10545000000000000000000000000000000000004C
:1054600000D09AD0B0D180D182D0B020D0B2D1813A
:10547000D182D0B0D0B2D0BBD0B5D0BDD0B00000BA
:1054800057656C636F6D6500000000000000000050
:10549000000057656C636F6D650000000000000040
:1054A000000000004269656E76656E75650000005B
:1054B00000000000000057696C6C6B6F6D6D656ECD
:1054C00000000000000000004269656E76656E69AC
:1054D000646F000000000000000042656E76656E9B
:1054E00075746F00000000000000000057656C63D9
:1054F0006F6D6500000000000000000000004265C4
:105500006D2076696E6461000000000000000000FC
:1055100057656C6B6F6D000000000000000000001C
:105520000000486F7367656C64696E697A000000FB
:1055300000000000FDC9F991EB8BA42100000000E0
:10554000000000000000D0B6D0B5D0BBD0B0D0BDB8
:10555000D0BDD18BD0B900007C3C3E5E2B3D3F2FAF
:105560005B5D3B2C2A225C00526573656E643A20B9
:10557000006F6B0020746F6F206C6F6E6720657812
:1055800074727573696F6E2070726576656E74657E
:10559000640A0020636F6C642065787472757369A7
:1055A0006F6E2070726576656E7465640A00627550
:1055B00073793A2070617573656420666F72206933
:1055C0006E7075740A00627573793A207061757334
:1055D000656420666F7220757365720A0062757368
:1055E000793A2070726F63657373696E670A004B56
:1055F000494C4C45442E20004B494C4C206361756E
:1056000073656420627920746F6F206D7563682004
:10561000696E6163746976652074696D65202D20FB
:1056200063757272656E7420636F6D6D616E643A3E
:105630002000506F72206661766F722C207265694F
:105640006E69636965005052494E54455220484185
:105650004C544544005072696E7465722068616CE8
:105660007465642E206B696C6C28292063616C6CF6
:105670006564210A000000D242000000000000C85A
:10568000423C3C3C207365745F617869735F697369
:105690005F61745F686F6D652800203A200A002002
:1056A0002063757272656E745F706F736974696F71
:1056B0006E3D005D203D20003E20686F6D655F6F90
:1056C00066667365745B003E3E3E207365745F6181
:1056D0007869735F69735F61745F686F6D652800D7
:1056E00000004842000048425555054100000000B6
:1056F0005761726E696E673A20486F6D696E6720F8
:1057000042756D702044697669736F72203C203158
:105710000A000202040000A0400000A040000000B7
:10572000400000D2420000F0420000C8423C3C3C35
:1057300020686F6D65617869732800203A203E20EB
:105740004146544552207365745F617869735F699F
:10575000735F61745F686F6D650A00202063757206
:1057600072656E745F706F736974696F6E3D004827
:105770006F6D65203220536C6F773A0A004D6F765B
:105780006520417761793A0A00486F6D65203120C4
:10579000466173743A0A0001FF013E3E3E20686F85
:1057A0006D65617869732800496E7365727420664F
:1057B000696C616D656E7420616E642070726573D2
:1057C0007320627574746F6E20286F72204D3130B3
:1057D00038290A0000002100240027002A002D009B
:1057E0003000330001010000040107010A0100003C
:1057F0002200250028002B002E0031003400020179
:105800000000050108010B01000020002300260014
:1058100029002C002F0032000001000003010601C6
:105820000901050505050705080808080202020226
:105830000A0A08080404040401010101010101012C
:105840000303030303030303040707070C0C0C0CF7
:105850000C0C0C0C020202020606060606060606E0
:105860000B0B0B0B0B0B0B0B07070A0A0A0A0A0A96
:10587000050501021020200808102040102040805B
:105880000201020108040201010204081020408004
:105890008040201008040201800402018040201092
:1058A00008040201080402010102040810204080DB
:1058B00001020408102040801008040880102040D5
:1058C000044000000A0B02090C0D0E080703040136
:1058D00000000000000000000000000000000000C8
:1058E0000000000000000000000000000000121195
:1058F0001000000000000000000000000000000098
:105900000000000000000000000000000000000097
:105910000000000000000000000000000000000087
:105920000000000000000000000000000000000077
:1059300000001F006007CFFFFF7FFFF9FFFF803FE0
:10594000FF001F007007CFFFFF7FFFF9FFFFC0FFC1
:10595000FF800F80F00F8FFFFF7FFFF9FFFFE1FF58
:10596000FFC00F80F80F8FFFFF7FFFF9FFFFF1FFF0
:10597000FFE007C1F81F0000000000000001F3FF76
:10598000FFE007C1FC1F0000000000000001F3F071
:1059900007E003E3FE3E0000000000000001F3E02A
:1059A00003E003E3FE3E0FFFFF7FFFF9E001F3E0BA
:1059B00003E001F7DF7C0FFFFF7FFFF9E001F3E079
:1059C00003E001F7DF7C0FFFFF7FFFF9E001F3E069
:1059D00003E000FF8FF80FFFFF7FFFF9E001F3E026
:1059E00003E000FF8FF80F80007C0001E001F3E08E
:1059F00003E0007F07F00F80007C0001E001F3F07E
:105A000007E0007F07F00F80007C0001E001F3FF5A
:105A1000FFE0003E03E00FFFFF7FFFF9FFFFF1FF14
:105A2000FFE0003E03C00FFFFF7FFFF9FFFFE1FF34
:105A3000FFC0001C01C00FFFFF7FFFF9FFFFC0FF89
:105A4000FF80001C01800FFFFF7FFFF9FFFF807FB9
:105A5000FF00000000000000000000000000000047
:105A60000000000000000000000000000000000036
:105A70000000000000000000000000000000000026
:105A80000000000000000000000000000000000016
:105A90000000473238205A20463330300D0A4D314D
:105AA00038004D313800473238205A2046333030E4
:105AB000005731303000554E4B4E4F574E00554E2B
:105AC0004B4E4F574E00554E4B4E4F574E00554E76
:105AD0004B4E4F574E00554E4B4E4F574E004E4F6C
:105AE0002057494649204D4F44554C4500202050F1
:105AF0006C616E6E65724275666665724279746538
:105B0000733A20002046726565204D656D6F72798D
:105B10003A2000436F6D70696C65643A205365707C
:105B200020313520323032310A00207C204175741A
:105B3000686F723A2028506572726F6E2C2057453C
:105B400045444F3344290A00323032302D31322D52
:105B5000323100204C617374205570646174656447
:105B60003A2000322E31352E320A004D61726C69B6
:105B70006E0020536F66747761726520526573659D
:105B8000740A00205761746368646F6720526573FC
:105B900065740A002042726F776E206F7574205210
:105BA000657365740A002045787465726E616C20B7
:105BB00052657365740A00506F77657255700A00FC
:105BC000575453544152540A0073746172740A005A
:105BD0006572726F722077726974696E6720746F74
:105BE0002066696C650A00456E6473746F7073207B
:105BF000256320256320256320256300205A3A0071
:105C000020593A0020583A00656E6473746F7073BF
:105C1000206869743A2000573230390057323033E7
:105C200000446F6E6520736176696E672066696CEB
:105C3000652E0A004D32390047312058313230206C
:105C4000593935204631353030004D3630303A2024
:105C5000546F6F20636F6C6400486F74656E6420CE
:105C6000746F6F20636F6C640A0043616E6E6F74B3
:105C7000206F70656E2073756264697220005072C7
:105C80006F7465637465642050696E0A00537461B3
:105C90006E6461726420446576696174696F6E3AFE
:105CA00020002052616E67653A2000204D61783AED
:105CB0002000204D696E3A20004D65616E3A20004B
:105CC00046696E6973686564210A002072616E67B7
:105CD000653A2000206D61783A2000206D696E3AA7
:105CE0002000207369676D613A2000206D65616E48
:105CF0003A20003A207A3A2000206F662000205A8D
:105D000000205900205800476F696E6720746F3A71
:105D100000436C6F636B776973650A00436F756E40
:105D20007465722D0020446972656374696F6E3A00
:105D30002000202020616E676C653A20005374615A
:105D40007274696E67207261646975733A200050DD
:105D50006F736974696F6E696E672074686520700F
:105D6000726F62652E2E2E0A003F4E756D6265724F
:105D7000206F66206C65677320696E206D6F766595
:105D80006D656E74206E6F7420706C6175736962DE
:105D90006C652028302D3135292E0A003F202858E7
:105DA0002C5929206F7574206F6620626F756E64A0
:105DB000732E0A003F53616D706C652073697A65BC
:105DC000206E6F7420706C61757369626C65202839
:105DD000342D3530292E0A004D3438205A2D50727A
:105DE0006F6265205265706561746162696C697487
:105DF0007920546573740A003F2856296572626FD2
:105E00007365206C6576656C20697320696D706CB4
:105E100061757369626C652028302D34292E0A0063
:105E20006F70656E206661696C65642C2046696CD4
:105E3000653A200057726974696E6720746F206636
:105E4000696C653A2000446973636F6E6E656374B4
:105E50006564004C4E3A257320533A256C64005615
:105E60004E3A257320483A257320463A257320413F
:105E70003A257320573A257320473A257300534635
:105E80003A257320503A256420423A257300545431
:105E9000303A25642054313A256420423A25642062
:105EA000433A256400005EBCE2613FDD83C29C7E14
:105EB00020A3FD1F419DC3217FFCA2401E5F01E383
:105EC000BD3E6082DC237D9FC1421CFEA0E1BF5D20
:105ED0000380DE3C62BEE0025CDF81633D7C22C069
:105EE0009E1D43A1FF4618FAA427799BC584DA3882
:105EF00066E5BB5907DB856739BAE406581947A53B
:105F0000FB7826C49A653BD987045AB8E6A7F91BE3
:105F100045C6987A24F8A6441A99C7257B3A648620
:105F2000D85B05E7B98CD2306EEDB3510F4E10F24D
:105F3000AC2F7193CD114FADF3702ECC92D38D6FEA
:105F400031B2EC0E50AFF1134DCE90722C6D33D1B7
:105F50008F0C52B0EE326C8ED0530DEFB1F0AE4CD0
:105F60001291CF2D73CA947628ABF517490856B411
:105F7000EA6937D58B5709EBB536688AD495CB29B2
:105F800077F4AA4816E9B7550B88D6346A2B75976B
:105F9000C94A14F6A8742AC896154BA9F7B6E80A98
:105FA00054D7896B35556E6B6E6F776E20636F6D4E
:105FB0006D616E643A202200203A203C3C3C207205
:105FC000756E5F7A5F70726F62650A00202063757C
:105FD0007272656E745F706F736974696F6E3D0085
:105FE000203A203C3C3C2072756E5F7A5F70726F85
:105FF00062650A00202063757272656E745F706F4F
:10600000736974696F6E3D00534C4F572050726F27
:106010006265206661696C210A00203A203E3E3E9E
:106020002072756E5F7A5F70726F62650A00202061
:1060300063757272656E745F706F736974696F6E89
:106040003D003C3C3C2070726F62655F70740A00DA
:1060500050726F62696E67206661696C65640000EA
:106060000000000000B1B2CFD09F9E0000000000F1
:1060700000000000000000000000457272657572AB
:1060800000000000000000000000000000000050C0
:10609000726F62696E6720676573636865697465AE
:1060A00072740000656C20736F6E64656F206661AA
:1060B0006C6C6F00000000000050726F62696E67C8
:1060C0002066616C6C69746F000000000000507203
:1060D0006F62696E67206661696C6564000000002C
:1060E000000000536F6E646167656D2066616C68C7
:1060F0006F7500000000000054657374656E2069C0
:1061000073206D69736C756B7400000000426173DD
:1061100061726973697A20736F6E64616C616D611D
:106120000000D9979AAA8C20BEF50000000000005C
:1061300000000000000000D0BDD0B520D183D0B455
:10614000D0B0D0BBD0BED181D18C0000205A3A2033
:106150000020593A200042656420583A2000203A35
:10616000200A00202063757272656E745F706F7311
:106170006974696F6E3D005F72656C617469766504
:10618000290A002C20002C20002C20002C20003E6E
:106190003E3E2070726F62655F70742800486F6DBC
:1061A000652025732573257320666972737400203A
:1061B00066697273740A005A0059005800486F6D7E
:1061C0006520004D3234004D323320257300534496
:1061D0002063617264206F6B0A006F70656E526F8E
:1061E0006F74206661696C65640A00766F6C756D0A
:1061F000652E696E6974206661696C65640A005376
:106200004420696E6974206661696C0A0020746FAD
:106210006F206C6F6E6720657874727573696F6E2E
:106220002070726576656E7465640A0020636F6C19
:106230006420657874727573696F6E20707265760C
:10624000656E7465640A00205A3A0020593A0020AD
:10625000436F756E7420583A0020453A00205A3A30
:106260000020593A00583A00205A0020590058009E
:1062700020204D61783A2000205A00205900580013
:1062800020204D696E3A20004F6E20004F66660058
:10629000536F667420656E6473746F70733A200078
:1062A00023646566696E652044454641554C545FDC
:1062B0004B64200023646566696E65204445464151
:1062C000554C545F4B69200023646566696E6520F8
:1062D00044454641554C545F4B7020005049442082
:1062E0004175746F74756E652066696E6973686553
:1062F00064212050757420746865206C617374206B
:106300004B702C204B6920616E64204B6420636FBE
:106310006E7374616E74732066726F6D2062656C4B
:106320006F7720696E746F20436F6E666967757250
:106330006174696F6E2E680A00504944204175747B
:106340006F74756E65206661696C6564212074697F
:106350006D656F75740A00453120544845524D41B2
:106360004C2052554E4157415900546865726D6139
:106370006C2052756E617761790045312048656106
:1063800074696E67206661696C6564004865617454
:10639000696E67206661696C6564005049442041FC
:1063A00075746F74756E65206661696C6564212013
:1063B00054656D706572617475726520746F6F20BD
:1063C000686967680A00204B643A2000204B693AEC
:1063D0002000204B703A20000A20436C61737369DF
:1063E0006320504944200A002054753A2000204B75
:1063F000753A2000206D61783A2000206D696E3A70
:10640000200020643A200020626961733A20005025
:106410004944204175746F74756E65206661696CBE
:1064200065642120426164206578747275646572C8
:10643000206E756D6265720A005049442041757482
:106440006F74756E652073746172740A004F6666AE
:1064500073657473206170706C6965640045727255
:106460003A20546F6F206661722100546F6F20666E
:1064700061722066726F6D207265666572656E630B
:106480006520706F696E740A00496E7365727420BE
:1064900066696C616D656E7420616E6420707265F2
:1064A000737320627574746F6E0A00507265737333
:1064B00020627574746F6E20746F2068656174203B
:1064C0006E6F7A7A6C650A00496E73657274206625
:1064D000696C616D656E7420616E642070726573A5
:1064E0007320627574746F6E20286F72204D313086
:1064F00038290A0024F4D43050C38E20C2A2401799
:10650000828B7011127A910D816CD90AA861E10811
:10651000C7586607615143061E4B5D05C145A70478
:106520001A411104093D9803713931034036DB02E9
:1065300065339102D4305402802E1D02632CEE018B
:10654000752AC501B028A001102781018F2564019B
:106550002B244B01E0223401AC211F018D200D01C1
:10656000801FFC00841EED00971DDF00B81CD200C8
:10657000E61BC600201BBC00641AB200B219A800BA
:106580000A19A0006A189900D117910040178B00D2
:10659000B516840031167E00B31579003A157300E4
:1065A000C7146F0058146A00EE1366008813630066
:1065B00025135E00C7125B006C12570015125400C1
:1065C000C111510070114F0021114B00D61049002C
:1065D0008D1047004610440002104200C00F4000DA
:1065E000800F3E00420F3C00060F3B00CB0E3800F0
:1065F000930E37005C0E3500270E3400F30D320089
:10660000C10D3100900D3000600D2E00320D2D00B7
:10661000050D2C00D90C2B00AE0C2900850C29008F
:106620005C0C2700350C27000E0C2600E80B24001C
:10663000C40B2400A00B23007D0B23005A0B210068
:10664000390B2100180B2000F80A1F00D90A1E0080
:10665000BB0A1E009D0A1D00800A1D00630A1C0063
:10666000470A1B002C0A1B00110A1A00F7091A001E
:10667000DD091900C4091900AB09190092091700B6
:106680007B091800630917004C091600360916002B
:10669000200916000A091500F5081500E008140085
:1066A000CC081400B8081400A408140090081300C3
:1066B0007D0812006B0813005808120046081200EB
:1066C00034081100230811001208110001081100FC
:1066D000F0071000E0071000D0071000C0071000FE
:1066E000B0070F00A107100091070E0083070F00ED
:1066F00074070F0065070E0057070E0049070E00CC
:106700003B070D002E070E0020070D0013070D009C
:1067100006070D00F9060C00ED060D00E0060C0062
:10672000D4060C00C8060C00BC060C00B0060C0019
:10673000A4060B0099060C008D060B0082060B00C8
:1067400077060B006C060B0061060A0057060B006B
:106750004C060A0042060A0038060A002E060A0005
:1067600024060A001A060A001006090007060A0095
:10677000FD050900F4050900EB050900E205090023
:10678000D9050900D0050900C7050900BE050900A3
:10679000B5050800AD050800A50509009C05080021
:1067A000940508008C050800840508007C05080095
:1067B000740508006C050700650508005D05070005
:1067C000560508004E05070047050700400508006C
:1067D00038050700310507002A05070023050700D3
:1067E0001C050600160507000F0507000805060032
:1067F00002050700FB040600F5040700EE0406008E
:10680000E8040600E2040700DB040600D5040600E5
:10681000CF040600C9040600C3040600BD04060038
:10682000B7040600B1040500AC040600A604060087
:10683000A00405009B0406009504050090040600D2
:106840008A04050085040500800406007A0405001A
:1068500075040500700405006B040500660405005E
:10686000610405005C04050057040500520405009E
:106870004D04050048040500430405003E040400DF
:106880003A04050035040500300404002C0405001A
:1068900027040400230405001E0404001A04040055
:1068A00016040500110404000D0404000904050089
:1068B0000404040000040400FC030400F8030400C2
:1068C000F4030400F0030400EC030400E8030400F4
:1068D000E4030400E0030400DC030400D803040024
:1068E000D4030400D0030400CC030400C803030055
:1068F000C503030024F404D9201BC40C5C0E9804C7
:10690000C4095F0265077101F405F900FB04B300D7
:1069100048048700C103690058035500030345007C
:10692000BE023A008402310053022A0029022500E7
:1069300004022000E4011C00C8011900AF01170087
:10694000980114008401130071011000610110000E
:1069500051010E0043010D0036010B002B010B000D
:1069600020010B00150109000C01090003010800BA
:10697000FB000800F3000800EB000700E40006003D
:10698000DE000600D8000600D2000600CC0005009C
:10699000C7000500C2000500BD000400B9000400E6
:1069A000B5000400B1000400AD000400A90004001B
:1069B000A5000300A20003009F0004009B00030049
:1069C000980003009500020093000300900003006C
:1069D0008D0002008B000300880002008600020088
:1069E00084000300810002007F0002007D0002009D
:1069F0007B000200790002007700010076000200AF
:106A00007400020072000100710002006F000200B9
:106A10006D0001006C0002006A00010069000200C4
:106A200067000100660001006500010064000200CB
:106A30006200010061000100600001005F000200CF
:106A40005D0001005C0001005B0001005A000100D4
:106A500059000100580001005700010056000100D4
:106A600055000100540001005300000053000100D4
:106A70005200010051000100500001004F000100D0
:106A80004E0000004E0001004D0001004C000100CE
:106A90004B0000004B0001004A00010049000100CA
:106AA00048000000480001004700010046000000C7
:106AB00046000100450000004500010044000100BF
:106AC00043000000430001004200000042000100BA
:106AD0004100000041000100400001003F000000B3
:106AE0003F0001003E0000003E0001003D000000AC
:106AF0003D0001003C0000003C0000003C000100A3
:106B00003B0000003B0001003A0000003A00010099
:106B10003900000039000100380000003800000092
:106B20003800010037000000370001003600000087
:106B3000360000003600010035000000350000007E
:106B40003500010034000000340000003400010072
:106B50003300000033000000330001003200000069
:106B6000320000003200010031000000310000005E
:106B70003100010030000000300000003000010052
:106B80002F0000002F0000002F0000002F00010048
:106B90002E0000002E0000002E0001002D0000003D
:106BA0002D0000002D0000002D0001002C00000031
:106BB0002C0000002C0000002C0001002B00000025
:106BC0002B0000002B0000002B0001002A00000019
:106BD0002A0000002A0000002A000100290000000D
:106BE0002900000029000000290000002900010000
:106BF00028000000280000002800000028000000F5
:106C000028000100270000002700000027000000E6
:106C100027000000270001002600000026000000D9
:106C200026000000260000002600010025000000CC
:106C300025000000250000002500000025000000C0
:106C400025000100240000002400000024000000B2
:106C500024000000240001002300000023000000A5
:106C60002300000023000000230000002300000098
:106C7000230001002200000022000000220000008A
:106C8000220000002200000022000100210000007C
:106C90002100000021000000210000002100000070
:106CA0002100000021000100200000002000000061
:106CB0002000000020000000200000002000000054
:106CC00020000000200001001F0000001F00000045
:106CD0001F0000001F0000001F0000001F00000038
:106CE0001F0001001E0000001E0000001E0000002A
:106CF0001E000000043700001E290000511B000088
:106D00005810000010090000CC04000078020000B8
:106D10004101000009FFFFFFFFFF00010101010128
:106D20006265640A002C2073797374656D20737436
:106D30006F7070656421204865617465725F4944B5
:106D40003A2000453120544845524D414C2052557F
:106D50004E4157415900546865726D616C205275FF
:106D60006E617761790045312048656174696E67AD
:106D7000206661696C65640048656174696E6720AE
:106D80006661696C656400466C6F77000000000006
:106D9000000000CCADD1D200000000000000004394
:106DA0006F756C6572000000000000466C757373AF
:106DB00072617465000000466C756A6F0000000027
:106DC000000000466C7573736F000000000000C483
:106DD000BCADC2D8AEB30000000000466C75786F41
:106DE00000000000000000466C6F7700000000000B
:106DF000000000416B69730000000000000000C04B
:106E0000EB20BA9600000000000000D09FD0BED159
:106E100082D0BED0BA000046616E20737065656492
:106E2000000000000000000000D5D6D1D200000014
:106E30000000000000000000000000566974657347
:106E400073652076656E74696C000000004C756691
:106E50007465720000000000000000000000005691
:106E6000656E74696C61646F720000000000000060
:106E70000056656C6F636974612076656E746F6C23
:106E8000610000CCA7DDBFB8C4DE00000000000038
:106E9000000000000056656C2E2076656E746F69E8
:106EA0006E68610000000046616E20736E656C685C
:106EB00065696400000000000046616E2048697A40
:106EC0006900000000000000000000F620BA9600F3
:106ED00000000000000000000000000000D09AD177
:106EE00083D0BBD0B5D1800000000000000000536B
:106EF00070656564000000000000000000000000F4
:106F000000D1D200000000000000000000000000DE
:106F10000000004C612076697465737365000000A1
:106F200000000000004765736368772E00000000D2
:106F30000000000000000056656C6F6369646164C6
:106F400000000000000000000056656C6F6369746B
:106F50006100000000000000000000BFB8C4DE00B7
:106F60000000000000000000000000000056656CFA
:106F70006F636964616465000000000000000053F5
:106F80006E656C6865696400000000000000000028
:106F90000048697A000000000000000000000000C6
:106FA000000000BA96000000000000000000000091
:106FB0000000000000D0A1D0BAD0BED180D0BED198
:106FC00081D182D18C000057697A6172640000001F
:106FD000000000000000000000000000000000A20F
:106FE000A3EEEF0000000000000000000000000021
:106FF000000000000000004C616E636572206C614F
:1070000020636F6E6669672E000000000000004D6F
:107010006167696572000000000000000000000068
:107020000000000000000057697A7A617264000075
:1070300000000000000000000000000000000070E0
:10704000726F6365647572612067756964617461EC
:1070500000000000000000B3B4B9B600000000005A
:1070600000000000000000000000000000000055CB
:1070700073616E646F206F20617373697374656EE2
:107080007465000000000044652077697A617264CD
:10709000206765627275696B656E000000000053C1
:1070A0006968697262617AC4B1206B756C6C616EDB
:1070B0006D610000000000A0EFBBBFABB20000009C
:1070C000000000000000000000000000000000D0F0
:1070D000BAD0BED0BBD0B4D183D0BD000000000078
:1070E0000000000000000044697361626C65207359
:1070F000746570706572730000000000000000008D
:107100000000000000B5B6B7B8B9BA000000000032
:10711000000000000000000000000000000000006F
:107120000000004465736163746976206C652070AB
:107130006173206120706173000000000000000096
:10714000004D6F746F72656E206465616B74697653
:10715000696572656E0000000000000000000041DB
:107160007061676172206D6F746F726573000000EB
:1071700000000000000000000000000000446973EF
:107180006162696C697461204D6F746F726900008F
:107190000000000000000000000000D3B0C0B0C339
:1071A000DEDDB9DEDD20B5CC00000000000000000F
:1071B0000000000000000000004465736163746912
:1071C000766172206D6F746F72657300000000004D
:1071D000000000000000004D6F746F72656E207536
:1071E00069740000000000000000000000000000C2
:1071F00000000000004D6F746F726C617269204472
:10720000757264757200000000000000000000004C
:10721000000000A0F020E4E60000000000000000F4
:10722000000000000000000000000000000000005E
:1072300000D092D18BD0BAD0BB2E20D0B4D0B2D057
:10724000B8D0B3D0B0D182D0B5D0BBD0B800004D4B
:107250003834004C6576656C20626564000000007F
:10726000000000000000000000000000000000001E
:1072700000000000B1B2CFD000000000000000000C
:1072800000000000000000000000000000000000FE
:1072900000000000004D6973652061206E6976650D
:1072A0006175000000000000000000000000000008
:1072B00000000000000042657474206E6976656C01
:1072C0006C696572656E000000000000000000003F
:1072D000000000000000004E6976656C617220704D
:1072E0006C617461666F726D6100000000000000E7
:1072F00000000000000000004C6976656C6C6120A5
:107300007069616E6F000000000000000000000066
:10731000000000000000000000CDDEAFC4DEDACDCA
:10732000DED8DDB8DE000000000000000000000034
:107330000000000000000000000043616D61206E4D
:107340006976656C61646100000000000000000067
:1073500000000000000000000000004C6576656C35
:1073600020626564000000000000000000000000D2
:107370000000000000000000000000005365766976
:107380007965207961746167690000000000000080
:1073900000000000000000000000000000CAF19D95
:1073A000AD00000000000000000000000000000030
:1073B0000000000000000000000000000000D09A63
:1073C000D0B0D0BBD0B8D0B1D180D0BED0B2D0B0C8
:1073D000D182D18C20D181D182D0BED0BB000047D8
:1073E0003238205A20463530300D0A47323820587E
:1073F00020592046313030300A4732390041757407
:107400006F20686F6D650000000000000000000044
:107410000000000000000000BBBCBD000000000038
:10742000000000000000000000000000000000005C
:107430000000005265746F7572206F726967696E23
:107440006500000000000000000000000000486F20
:107450006D6500000000000000000000000000005A
:107460000000000000000000004175746F20496EAC
:107470006963696F00000000000000000000000068
:10748000000000004175746F20486F6D65000000BA
:10749000000000000000000000000000000000B933
:1074A000DEDDC3DDCCAFB70000000000000000004F
:1074B00000000000000000000000497220706172AE
:1074C00061206F726967656D0000000000000000B8
:1074D00000000000004175746F20686F6D6500004A
:1074E000000000000000000000000000000000009C
:1074F000456B73656E6C6572692053696669726C61
:107500006100000000000000000000D0D1EC00008D
:10751000000000000000000000000000000000006B
:10752000000000000000D090D0B2D182D0BE20D0A8
:10753000BFD0B0D180D0BAD0BED0B2D0BAD0B00017
:1075400000473238205A20463530300D0A4732384D
:10755000205820592046313030300D0A473120580C
:10756000353520593535204631303030004D3130F9
:107570003420543020533231300D0A4D3730322010
:1075800054300D0A4D313034205330004D313034F9
:1075900020543020533231300D0A4D3730312054D1
:1075A000300D0A4D313034205330004D6F76652058
:1075B000302E316D6D000000000000000000000062
:1075C0000000000000C1B220302E316D6D000000BF
:1075D0000000000000000000000000000000004467
:1075E00065706C6163657220302E316D6D00000036
:1075F000000000000000000000302E316D6D000022
:10760000000000000000000000000000000000007A
:107610000000004D6F76657220302E316D6D0000D8
:10762000000000000000000000000000004D756F29
:10763000766920646920302E316D6D0000000000F5
:1076400000000000000000302E316D6D20B2C4DE5D
:10765000B300000000000000000000000000000077
:10766000004D6F76657220302E316D6D0000000088
:107670000000000000000000000000566572706C01
:107680006161747320302E316D6D000000000000C8
:107690000000000000302E316D6D00000000000081
:1076A00000000000000000000000000000000030AA
:1076B0002E316D6D20D49700000000000000000006
:1076C000000000000000000000D094D0B2D0B8D07C
:1076D000B6D0B5D0BDD0B8D0B520302E31D0BCD0CA
:1076E000BC00004D6F766520316D6D00000000001C
:1076F0000000000000000000000000C1B220316D59
:107700006D0000000000000000000000000000000C
:107710000000004465706C6163657220316D6D001E
:107720000000000000000000000000316D6D00004E
:107730000000000000000000000000000000000049
:107740000000004D6F76657220316D6D0000000005
:1077500000000000000000000000004D756F766919
:10776000206469202020316D6D00000000000000C1
:107770000000002020316D6D20B2C4DEB300000097
:1077800000000000000000000000004D6F766572F0
:1077900020316D6D000000000000000000000000BE
:1077A000000000566572706C6161747320316D6DFC
:1077B0000000000000000000000000316D6D0000BE
:1077C00000000000000000000000000000000000B9
:1077D000000000316D6D20D4970000000000000013
:1077E0000000000000000000000000D094D0B2D0E3
:1077F000B8D0B6D0B5D0BDD0B8D0B52031D0BCD07F
:10780000BC00004D6F76652031306D6D00000000CA
:10781000000000000000000000000000C1B22031A4
:10782000306D6D000000000000000000000000004E
:1078300000000000004465706C61636572203130A7
:10784000206D6D00000000000000000000003130DD
:107850006D6D00000000000000000000000000004E
:10786000000000000000004D6F7665722031306D21
:107870006D0000000000000000000000000000009B
:107880004D756F7669206469202031306D6D000080
:107890000000000000000000002031306D6D20B2BB
:1078A000C4DEB30000000000000000000000000083
:1078B00000004D6F7665722031306D6D0000000064
:1078C0000000000000000000000000566572706CAF
:1078D000616174732031306D6D00000000000000A4
:1078E0000000000031306D6D00000000000000005D
:1078F0000000000000000000000000000031306DBA
:107900006D20D4970000000000000000000000007F
:10791000000000000000D094D0B2D0B8D0B6D0B5EE
:10792000D0BDD0B8D0B5203130D0BCD0BC00004DD7
:107930006F76652061786973000000000000000028
:10794000000000000000000000000000000000C176
:10795000B2CE0000000000000000000000000000A7
:1079600000000000000000000000000000000044D3
:1079700065706C61636572206C276178650000003A
:1079800000000000000000000000000000000042B5
:1079900065776567656E000000000000000000006C
:1079A0000000000000000000000000000000004D8A
:1079B0006F76657220656A65730000000000000044
:1079C0000000000000000000000000000000004D6A
:1079D000756F766920417373650000000000000038
:1079E000000000000000000000000000000000BCDB
:1079F000DEB8B2C4DEB300000000000000000000EA
:107A00000000000000000000000000000000004D29
:107A10006F766572206569786F00000000000000D5
:107A20000000000000000000000000000000004115
:107A30007320766572706C61617473656E0000000E
:107A400000000000000000000000000000000045F1
:107A50006B73656E20596F6E657400000000000046
:107A6000000000000000000000000000000000EA2C
:107A700020D497000000000000000000000000007B
:107A8000000000000000000000000000000000D026
:107A900094D0B2D0B8D0B6D0B5D0BDD0B8D0B52083
:107AA000D0BFD0BE20D0BED181D18FD0BC00004588
:107AB00078747275646572000000000000000000B8
:107AC000000000CCADBA0000000000000000000083
:107AD00000000000000000457874727564657572DE
:107AE000000000000000000000000045787472757E
:107AF0006465720000000000000000000000004506
:107B000078747275736F720000000000000000004E
:107B10000000004573747275736F72650000000099
:107B200000000000000000B4B8BDC4D9B0C0DEB091
:107B300000000000000000000000004D6F7665723C
:107B4000204578747275736F720000000000004564
:107B50007874727564657200000000000000000017
:107B6000000000456B73747275646572000000005C
:107B700000000000000000D5BBF2A094000000004F
:107B80000000000000000000000000D0ADD0BAD11D
:107B900081D182D180D183D0B4D0B5D18000004DC5
:107BA0006F7665205A000000000000000000000011
:107BB0000000000000000000C1B2205A00000000D8
:107BC00000000000000000000000000000000000B5
:107BD000004465706C61636572205A00000000000B
:107BE000000000000000000000005665727363682A
:107BF00069656265205A0000000000000000000076
:107C00000000004D6F766572205A000000000000F1
:107C10000000000000000000000000004D756F76BD
:107C200069205A0000000000000000000000000071
:107C300000000000005ABCDEB820B2C4DEB3000071
:107C400000000000000000000000000000004D6F78
:107C5000766572205A00000000000000000000005D
:107C600000000000000000566572706C6161747362
:107C7000205A00000000000000000000000000008A
:107C80005A0000000000000000000000000000009A
:107C90000000000000000000005AEA20D497000015
:107CA00000000000000000000000000000000000D4
:107CB0000000D094D0B2D0B8D0B6D0B5D0BDD0B836
:107CC000D0B520D0BFD0BE205A00004D6F766520C1
:107CD000590000000000000000000000000000004B
:107CE00000000000C1B220590000000000000000A8
:107CF000000000000000000000000000004465706B
:107D00006C616365722059000000000000000000F3
:107D10000000000000005665727363686965626563
:107D20002059000000000000000000000000004D8D
:107D30006F7665722059000000000000000000000E
:107D400000000000000000004D756F7669205900AA
:107D50000000000000000000000000000000000023
:107D60000059BCDEB820B2C4DEB300000000000041
:107D7000000000000000000000004D6F76657220DA
:107D8000590000000000000000000000000000009A
:107D9000000000566572706C6161747320590000B8
:107DA000000000000000000000000000590000007A
:107DB00000000000000000000000000000000000C3
:107DC000000000000059EA20D497000000000000E5
:107DD0000000000000000000000000000000D0943F
:107DE000D0B2D0B8D0B6D0B5D0BDD0B8D0B520D0F4
:107DF000BFD0BE205900004D6F76652058000000AE
:107E00000000000000000000000000000000000072
:107E1000C1B2205800000000000000000000000077
:107E20000000000000000000004465706C616365A4
:107E30007220580000000000000000000000000058
:107E400000005665727363686965626520580000BA
:107E500000000000000000000000004D6F76657219
:107E6000205800000000000000000000000000009A
:107E7000000000004D756F7669205800000000007A
:107E80000000000000000000000000000058BCDE00
:107E9000B820B2C4DEB30000000000000000000003
:107EA0000000000000004D6F766572205800000051
:107EB000000000000000000000000000000000566C
:107EC0006572706C616174732058000000000000DE
:107ED000000000000000000058000000000000004A
:107EE0000000000000000000000000000000000092
:107EF0000058EA20D49700000000000000000000B5
:107F000000000000000000000000D094D0B2D0B803
:107F1000D0B6D0B5D0BDD0B8D0B520D0BFD0BE205F
:107F2000580000507265706172650000000000002A
:107F30000000000000000000000000A4A5EEEF001B
:107F40000000000000000000000000000000000031
:107F500000000050726570617265720000000000E0
:107F60000000000000000000000000566F72626513
:107F700072656974756E6700000000000000000003
:107F800000000050726570617261720000000000B4
:107F900000000000000000000000005072657061E9
:107FA00072610000000000000000000000000000FE
:107FB000000000BCDEADDDCBDEBEAFC3B200000012
:107FC00000000000000000000000005072657061B9
:107FD000726172000000000000000000000000005C
:107FE000000000566F6F72626572656964656E00AD
:107FF000000000000000000000000048617A697283
:108000006C696B0000000000000000000000000030
:10801000000000E3B120DAC400000000000000000E
:108020000000000000000000000000D09FD0BED083
:10803000B4D0B3D0BED182D0BED0B2D0B8D182D16C
:108040008C000070012C0190012701B0012201C0B9
:10805000011D01F00118011002130130020E016030
:1080600002090190020401C002FF000003FA00406F
:1080700003F5008003F000D003EB002004E600705D
:1080800004E100E004DC004005D700C005D2004058
:1080900006CD00D006C8008007C3003008BE00F03F
:1080A00008B900C009B400B00AAF00B00BAA00D0F4
:1080B0000CA500000EA000500F9B00C010960050B1
:1080C00012910000148C00C0158700B0178200B018
:1080D000197D00D01B7800001E730040206E0090B8
:1080E000226900F024640040275F0090295A00E0D4
:1080F0002B5500102E500020304B0010324600E06F
:1081000033410090353C001037370070383200A002
:10811000392D00B03A2800A03B2300603C1E00101F
:108120003D1900903D1400103E0F00703E0A00C043
:108130003E0500003F0000403FFBFF803FF6FFC0D0
:108140003FF1FF4531204572723A204D4158544568
:108150004D50004D415854454D5020747269676729
:1081600065726564004531204572723A204D494E72
:1081700054454D50004D494E54454D502074726940
:10818000676765726564004D383420582059205A5D
:10819000204500202F0020403A0025756825303208
:1081A000756D002530327568253032756D00257586
:1081B000642530327568253032756D00000609007F
:1081C000FE0701920321207FFF07FF07FF00000049
:1081D0000600000107070602008080808080008082
:1081E000030202060105A0A0050707060000505083
:1081F000F850F850500507070600002078A07028B6
:10820000F020050707060000C0C810204098180598
:1082100007070600006090A040A8906802030306CC
:108220000104C040800307070601002040808080D1
:1082300040200307070601008040202020408005E1
:10824000050506000120A870A82005050506000107
:108250002020F820200203030602FFC04080050111
:1082600001060003F8020202060200C0C00505056F
:1082700006000108102040800507070600007088EE
:10828000888888887003070706010040C040404086
:1082900040E0050707060000708808708080F80538
:1082A0000707060000F81020100808F00507070669
:1082B000000010305090F81010050707060000F875
:1082C00080F008088870050707060000708080F0BD
:1082D000888870050707060000F808102020202075
:1082E00005070706000070888870888870050707F2
:1082F00006000070888878080870020505060200EC
:10830000C0C000C0C00206060602FFC0C000C040D8
:10831000800407070600001020408040201005035D
:1083200003060002F800F804070706010080402059
:108330001020408005070706000070880810200004
:108340002005070706000070880868A8A8700507C0
:1083500007060000708888F88888880507070600E7
:1083600000F08888F08888F005070706000070880C
:108370008080808870050707060000F0888888885C
:1083800088F0050707060000F88080F08080F80577
:108390000707060000F88080F08080800507070648
:1083A0000000708880B8888870050707060000887C
:1083B0008888F88888880107070602008080808006
:1083C00080808005070706000038101010109060AC
:1083D0000507070600008890A0C0A0908805070741
:1083E000060000808080808080F805070706000076
:1083F00088D8A8888888880507070600008888C864
:10840000A8988888050707060000708888888888EB
:1084100070050707060000F08888F0808080050757
:108420000706000070888888A8906805070706007E
:1084300000F08888F0A09088050707060000788083
:1084400080700808F0050707060000F820202020AB
:10845000202005070706000088888888888870051E
:1084600007070600008888888888502005070706C7
:1084700000008888888888A85005070706000088BB
:108480008850205088880507070600008888885093
:10849000202020050707060000F80810204080F87B
:1084A000030707060100E08080808080E005050565
:1084B0000600018040201008030707060100E020A5
:1084C00020202020E0050303060004205088050139
:1084D00001060000F80202020602058040050505BB
:1084E000060000700878887805070706000080807D
:1084F000B0C88888F0050505060000708080887087
:1085000005070706000008086898888878050505AB
:108510000600007088F880700507070600003048E4
:10852000E0404040400506060600FF708888780855
:10853000700507070600008080B0C888888801079A
:108540000706020080008080808080030808060102
:10855000FF200020202020A0400407070600008004
:108560008090A0C0A090030707060100C0404040D3
:108570004040E0050505060000D0A8A8A8A805050C
:1085800005060000B0C8888888050505060000704B
:10859000888888700506060600FFF08888F08080CD
:1085A0000506060600FF7888887808080505050690
:1085B0000000B0C88080800505050600007080704E
:1085C00008F00407070600004040E0404040300546
:1085D00005050600008888889868050505060000DE
:1085E00088888850200505050600008888A8A850BE
:1085F000050505060000885020508805060606007F
:10860000FF888888780870050505060000F81020A6
:1086100040F8030707060100204040804040200149
:10862000070706020080808080808080030707069D
:1086300001008040402040408005020206000268A0
:108640009000000006000000060900FE07019103EB
:108650002020FFFF08FF07FF0000000600000107C1
:1086600007060200808080808000800302020601ED
:1086700005A0A00507070600005050F850F850501C
:108680000507070600002078A07028F020050707DE
:10869000060000C0C8102040981805070706000013
:1086A0006090A040A89068020303060104C04080C7
:1086B0000307070601002040808080402003070751
:1086C00006010080402020204080050505060001AD
:1086D00020A870A8200505050600012020F820200C
:1086E0000203030602FFC04080050101060003F8F3
:1086F000020202060200C0C00505050600010810BE
:10870000204080050707060000708898A8C8887078
:1087100003070706010040C040404040E00507074E
:10872000060000708808708080F8050707060000C2
:10873000F81020100808F005070706000010305058
:1087400090F81010050707060000F880F008088868
:1087500070050707060000304080F0888870050724
:1087600007060000F8081020202020050707060053
:108770000070888870888870050707060000708878
:108780008878081060020505060200C0C000C0C05D
:108790000206060602FFC0C000C0408004070706AC
:1087A000000010204080402010050303060002F85E
:1087B00000F80407070601008040201020408005D3
:1087C000070706000070880810200020050606062E
:1087D000000070880868A870050707060000708808
:1087E00088F8888888050707060000F08888F088E0
:1087F00088F0050707060000708880808088700573
:108800000707060000E09088888890E005070706C3
:108810000000F88080F08080F8050707060000F867
:108820008080F0808080050707060000708880B88F
:10883000888870050707060000888888F888888877
:10884000010707060200808080808080800507077E
:108850000600003810101010906005070706000091
:108860008890A0C0A090880507070600008080803F
:10887000808080F805070706000088D8A8888888C7
:10888000880507070600008888C8A8988888050713
:10889000070600007088888888887005070706002A
:1088A00000F08888F0808080050707060000708847
:1088B0008888A89068050707060000F08888F0A05F
:1088C0009088050707060000788080700808F0058A
:1088D0000707060000F820202020202005070706B3
:1088E0000000888888888888700507070600008847
:1088F00088888888502005070706000088888888AF
:1089000088A85005070706000088885020508888EE
:1089100005070706000088888850202020050707E3
:10892000060000F80810204080F803070706010041
:10893000E08080808080E005050506000180402001
:108940001008030707060100E02020202020E00592
:108950000303060004205088050101060000F80208
:108960000202060205804005050506000070087831
:1089700088780507070600008080B0C88888F00561
:108980000505060000708080887005070706000056
:10899000080868988888780505050600007088F83A
:1089A00080700507070600003048E0404040400561
:1089B00006060600FF70888878087005070706001D
:1089C000008080B0C8888888010707060200800000
:1089D00080808080800308080601FF20002020207E
:1089E00020A040040707060000808090A0C0A0904F
:1089F000030707060100C04040404040E005050570
:108A0000060000D0A8A8A8A8050505060000B0C863
:108A10008888880505050600007088888870050626
:108A2000060600FFF08888F080800506060600FF35
:108A3000788888780808050505060000B0C8808099
:108A40008005050506000070807008F00507070620
:108A500000004040E0404048300505050600008821
:108A600088889868050505060000888888502005D4
:108A700005050600008888A8A85005050506000021
:108A800088502050880506060600FF8888887808E8
:108A900070050505060000F8102040F803070706DA
:108AA000010020404080404020010707060200806E
:108AB000808080808080030707060100804040207E
:108AC0004040800502020600036890000000060096
:108AD000000000000600000000000600000000008A
:108AE0000600000000000600000000000600000074
:108AF0000000060000000000060000000000060064
:108B00000000000006000000000006000000000059
:108B10000600000000000600000000000600000043
:108B20000000060000000000060000000000060033
:108B30000000000006000000000006000000000029
:108B40000600000000000600000000000600000013
:108B50000000060000000000060000000000060003
:108B600000000000060000000000060000000000F9
:108B700006000000000006000000000006000000E3
:108B800000000600000000000600000000000600D3
:108B90000005080806000040F88080F08080F80595
:108BA000080806000050F88080F08080F80507076C
:108BB000060000E0404070484870050808060000C4
:108BC0001020F88880808080050707060000304864
:108BD00080E0804830050707060000708880700834
:108BE0008870030707060100E04040404040E00372
:108BF0000808060100A000E040404040E0050707EB
:108C000006000038101010109060050707060000DD
:108C1000A0A0A0B8A8A8B8050707060000A0A0A0BB
:108C2000F8A8A8B8040707060000E04070505050AC
:108C30005005080806000010208890A0E0908805E4
:108C4000080806000040208898A8C88888050909F7
:108C50000600FF502088888850202020050808063C
:108C600000FF888888888888F820050707060000A4
:108C7000708888F8888888050707060000F88080D3
:108C8000F08888F0050707060000F08888F08888DB
:108C9000F0050707060000F88880808080800508BE
:108CA000080600FF782828284888F888050707065E
:108CB0000000F88080F08080F8050707060000A813
:108CC000A8A870A8A8A8050707060000F008087063
:108CD0000808F0050707060000888898A8C8888853
:108CE00005080806000050208898A8A8C88805072D
:108CF000070600008890A0C0A0908805070706001E
:108D0000007828282828A84805070706000088D8E2
:108D1000A888888888050707060000888888F8885A
:108D2000888805070706000070888888888870058D
:108D30000707060000F888888888888805070706DE
:108D40000000F08888F0808080050707060000702A
:108D5000888080808870050707060000F8202020A2
:108D600020202005070706000088888850204080C2
:108D70000507070600002070A8A8A87020050707AF
:108D8000060000888850205088880508080600FFE3
:108D9000888888888888F80805070706000088887A
:108DA0008898680808050707060000A8A8A8A8A8CA
:108DB000A8F80508080600FFA8A8A8A8A8A8F80809
:108DC000050707060000C0404070484870050707C7
:108DD000060000888888C8A8A8C8050707060000FC
:108DE000808080F08888F0050707060000708808FA
:108DF0003808887005070706000090A8A8E8A8A80A
:108E000090050707060000788888782848880505B7
:108E10000506000070087888780507070600001826
:108E20006080F0888870040505060000E090E090FE
:108E3000E0050505060000F8888080800506060626
:108E400000FF78284888F888050505060000708826
:108E5000F88070050505060000A8A870A8A80505FB
:108E600005060000F0083008F0050505060000883A
:108E700098A8C88805070706000050208898A8C849
:108E80008804050506000090A0C0A0900505050611
:108E90000000F82828A84805050506000088D8A87D
:108EA00088880505050600008888F8888805050576
:108EB0000600007088888870050505060000F8889F
:108EC0008888880506060600FFF08888F0808005FF
:108ED0000505060000708080887005050506000005
:108EE000F8202020200506060600FF8888887808DC
:108EF000700506060600002070A8A870200505056C
:108F000006000088502050880506060600FF888865
:108F10008888F8080505050600008888F80808050F
:108F20000505060000A8A8A8A8F80506060600FF83
:108F3000A8A8A8A8F808050505060000C0407048C4
:108F4000700505050600008888C8A8C80305050641
:108F500001008080C0A0C0050505060000708838AB
:108F6000887005050506000090A8E8A8900505058D
:108F70000600007888782848050808060000402088
:108F8000007088F8807005070706000050007088A0
:108F9000F880700509090600FF40E0404078484825
:108FA0004810050808060000102000F8888080801E
:108FB0000505050600007088608870050505060037
:108FC0000070807008F001070706020080008080B2
:108FD000808080030707060100A000404040404019
:108FE0000308080601FF200020202020A0400505DE
:108FF00005060000A0A0B8A8B8050505060000A059
:10900000A0F8A8B805060606000040E040784848E9
:1090100004080806000010200090A0C0A0900508D9
:10902000080600004020008898A8C888050909069D
:1090300000FF502000888888780870050606060022
:10904000FF88888888F820000C0B00FE0701920337
:109050002120FFFF0AFF07FF00000006000A0107AA
:1090600007060200808080808000800302020601E3
:1090700005A0A00507070600005050F850F8505012
:109080000507070600002078A07028F020050707D4
:10909000060000C0C8102040981805070706000009
:1090A0006090A040A89068020303060104C04080BD
:1090B0000307070601002040808080402003070747
:1090C00006010080402020204080050505060001A3
:1090D00020A870A8200505050600012020F8202002
:1090E0000203030602FFC04080050101060003F8E9
:1090F000020202060200C0C00505050600010810B4
:10910000204080050707060000708898A8C888706E
:1091100003070706010040C040404040E005070744
:10912000060000708808708080F8050707060000B8
:10913000F81020100808F00507070600001030504E
:1091400090F81010050707060000F880F00808885E
:1091500070050707060000708080F088887005079A
:1091600007060000F8081020202020050707060049
:10917000007088887088887005070706000070886E
:109180008878080870020505060200C0C000C0C04B
:109190000206060602FFC0C000C0408004070706A2
:1091A000000010204080402010050303060002F854
:1091B00000F80407070600008040201020408005CA
:1091C0000707060000708808102000200507070622
:1091D000000070880868A8A87005070706000070DE
:1091E0008888F8888888050707060000F08888F0D6
:1091F0008888F005070706000070888080808870E6
:10920000050707060000F08888888888F0050707AA
:10921000060000F88080F08080F80507070600004F
:10922000F88080F080808005070706000070888045
:10923000B8888870050707060000888888F888883D
:1092400088010707060200808080808080800507F3
:109250000706000038101010109060050707060080
:10926000008890A0C0A090880507070600008080B5
:1092700080808080F805070706000088D8A88888C5
:1092800088880507070600008888C8A89888880588
:109290000707060000708888888888700507070619
:1092A0000000F08888F080808005070706000070C5
:1092B000888888A89068050707060000F08888F06D
:1092C000A09088050707060000788080700808F0E5
:1092D000050707060000F8202020202020050707AA
:1092E00006000088888888888870050707060000BF
:1092F00088888888885020050707060000888888A5
:109300008888A850050707060000888850205088E4
:109310008805070706000088888850202020050758
:1093200007060000F80810204080F8030707060031
:1093300000E08080808080E0050505060001804017
:10934000201008030707060000E02020202020E06E
:10935000050303060004205088050101060000F8FB
:10936000020202060205804005050506000070089D
:109370007888780507070600008080B0C88888F0E4
:109380000505050600007080808870050707060047
:109390000008086898888878050505060000708828
:1093A000F880700507070600003048E04040404064
:1093B0000506060600FF708888780870050707060E
:1093C00000008080B0C888888801070706020080F6
:1093D0000080808080800308080601FF2000202094
:1093E0002020A040040707060100808090A0C0A0B4
:1093F00090030707060100C04040404040E00505DB
:1094000005060000D0A8A8A8A8050505060000B01C
:10941000C88888880505050600007088888870055A
:1094200006060600FFF08888F08080050606060024
:10943000FF788888780808050505060000B0C88010
:10944000808005050506000070807008F00407079D
:109450000600004040E040404030050505060000A1
:109460008888889868050505060000888888502047
:109470000505050600008888A8A850050505060012
:109480000088502050880506060600FF88888878E6
:109490000870050505060000F8102040F8030707CE
:1094A00006010020404080404020010707060200DE
:1094B0008080808080808003070706010080404014
:1094C000204040800502020600036890000000066C
:1094D000000A00000006000A00000006000A000062
:1094E0000006000A0B0B160C00FE7C800480048032
:1094F000048004E0088008803080C0800080008004
:10950000090B160C02FEF48014801480148017805E
:109510002480248044808480048004800A0C180CF9
:1095200001FE00407C4004400440044005C0084067
:1095300010402040C04000400040090B160C02FEC5
:10954000F8800B8008801380E08000007F8000801E
:109550007F8040003F80090B160C02FEF8800880D7
:109560000B8010802380C08000003F00408040803E
:109570003F00090B160C02FEF28012801E80128042
:10958000128022802E8042808280028002800A0A1D
:10959000140C01FF7F800080008000800080088024
:1095A000088008800800FFC0090A140C02FFFF00B1
:1095B00001000100010001000100010001000100A3
:1095C000FF800A0B160C01FE7C400440044004405E
:1095D0000440084010402040C04000400040090BBB
:1095E000160C02FEFC800480048004801880E08059
:1095F00000003F00408040803F00090B160C02FE37
:10960000FC8024802480248027802480248048803B
:10961000988000800080090A140C02FFFF001100EE
:109620001100110011001100110011000000FF8055
:109630000A0A140C01FF40004000400040003F8037
:109640000000040004000400FFC00A0B160C01FE19
:109650008000800080007FC000000000FFC0040088
:10966000040004000400090B160C01FE80808080B9
:10967000808080808080808080807E8000800080EC
:1096800000800A0B160C01FEFE80808080808080A6
:1096900080C0808080807E800080008000800A0BF7
:1096A000160C01FEFD4081408140814081C0814017
:1096B000814081407D40014001400A0B160C01FEB3
:1096C000FE4080408040804083C080408040804099
:1096D0007E40004000400A0B160C01FEF94081401C
:1096E000814081408F4081408140814079400140EC
:1096F00001400A0A140C01FF7F8040004000400036
:1097000040003F80000004000400FFC00A0B160C5C
:1097100001FE7F80400040003F800400FFC0000049
:109720003F00408040803F000A0B160C01FE7E4047
:10973000404040403E400840FF4000007FC0404065
:1097400040403FC00A0A140C01FF7F8040004000E7
:10975000400040003F80000000000000FFC0090BF7
:10976000160C02FEF880808080808080808080805F
:1097700080807C800080008000800A0B160C01FE37
:10978000FE408040804080407E40004000003F809E
:10979000404040403F800B0B160C01FEFC800480D3
:1097A0000480FC8080E0808080807E80008000805B
:1097B00000800A0B160C01FEF94009400940F940EF
:1097C0008740814081407D400140014001400A0BBB
:1097D000160C01FEFC400440FDC0804080407E40ED
:1097E00000007FC00040004000400A0B160C01FE44
:1097F0007F80008000807F80400040003F8000002C
:1098000004000400FFC00A0B160C01FE7F800080DC
:1098100000807F80400040003F8000001200120066
:10982000FFC00A0B160C01FE7F8000807F80400085
:109830003F800000FFC004000400040004000A0B85
:10984000160C01FE7F80008000807F804000400079
:109850003F80000000000000FFC00A0B160C01FE54
:10986000FC4004400440FC408040804080407E40FA
:109870000040004000400B0B160C01FEFC80848071
:109880008480848084E0848084807C800080008068
:1098900000800A0B160C01FEF940894089408F4078
:1098A00089408940894079400140014001400A0BCC
:1098B000160C01FEF94089408F408940894079406B
:1098C00000004000400040003FC00A0B160C01FEA3
:1098D000FC4085C0844085C084407C40000040003E
:1098E000400040003FC00A0A140C01FF7F80408006
:1098F0004080408040803F80000004000400FFC0A2
:109900000A0B160C01FEFC408440844084408440D5
:10991000844084407C400040004000400A0B160C0C
:1099200001FE844084408440FC4085C084408440E3
:109930007C400040004000400A0B160C01FE8440B1
:109940008440FDC0844084407C40000040407FC093
:1099500040403FC00A0B160C01FE894089408940F7
:10996000FF408940894089407940014001400140E1
:109970000A0B160C01FE89408940FF40894079405E
:1099800000007FC000407FC040003FC00A0B160CA3
:1099900001FE844085C0FC4085C084407C400000BE
:1099A0004000400040003FC00A0A140C01FF408004
:1099B00040807F804080408040803F8004000400E1
:1099C000FFC00A0B160C01FE40807F8040807F8024
:1099D0000400FFC000007F800080008000800A0B30
:1099E000160C01FE424042407E40424042403E4012
:1099F00008400840FF40004000400B0B160C01FEE1
:109A0000108010801080108028E0288044804480DE
:109A10008280008000800B0B160C01FE10801080ED
:109A200010E0288044808280000040807F80408059
:109A30003F800B0B160C01FE1080108010E0288078
:109A40004480828000003F00408040803F000A0B3D
:109A5000160C01FE1040104011C0284044408240C6
:109A600000004000400040003FC0090B160C02FE01
:109A7000208020802380508088800000FF8000802C
:109A8000FF8080007F800A0B160C01FE1140114000
:109A9000114011402F40294045404540834001403E
:109AA00001400A0B160C01FE1140114017402940DD
:109AB000454083400000040004001B0060C00A0B06
:109AC000160C01FE104011C0104029C044408240D5
:109AD00000004000400040003FC0090B160C02FE91
:109AE000080008003600C1800800FF800000FF80E9
:109AF000008000800080090A140C02FF08000800A2
:109B000014002200C1800000000000000000FF805F
:109B1000090B160C02FE080008003600C180000088
:109B2000FF8000008080FF8080807F80090B160C02
:109B300001FE1080108010801080288028804480D2
:109B40004480828000800080090B160C01FE10808A
:109B5000108028804480828000007F8000807F8089
:109B600040003F800B0B160C01FE7880848084E05F
:109B700084808480788000007F80408040803F80A7
:109B80000B0B160C01FE7880848084E08480848036
:109B90007880000040807F8040803F800A0B160C58
:109BA00001FE7140894089C08940894071400000B0
:109BB00040407FC040403FC00A0B160C01FE784079
:109BC00084408440844085C0844084408440784000
:109BD000004000400A0B160C01FE7840844085C00E
:109BE00084408440784000004000400040003FC076
:109BF0000A0B160C01FE7840844085C084408440E6
:109C00007840000040407FC040403FC00B0B160C26
:109C100001FE7840844085C0844084407840000044
:109C200044807C8045403E200A0B160C01FE7840A3
:109C3000844085C08440844085C08440844078400E
:109C4000004000400A0B160C01FE784085C084409D
:109C5000844085C0784000004000400040003FC084
:109C60000A0B160C01FE784085C0844085C0784000
:109C700000007FC000407FC040003FC00A0B160CB0
:109C800001FE784085C08440844085C07840000053
:109C90003F80404040403F80090A140C01FF1C00F7
:109CA00022004100410022001C00000008000800C2
:109CB000FF800A0B160C01FE3F00408040803F00F1
:109CC0000800FFC000004000400040003F80090B3A
:109CD000160C01FE3F00408040803F000800FF80DE
:109CE000000040807F8040803F800B0B160C01FEFF
:109CF0007C80828082E07C801080FE80000080007A
:109D0000800080007F80090A140C01FF1C002200E3
:109D10004100410022001C00000022002200FF80C0
:109D20000A0B160C01FE3F00408040803F000000FF
:109D3000FFC004004400400040003F800A0B160CA6
:109D400001FE3C4042403DC00040FF40084008400A
:109D50004840400040003FC0090B160C02FE7880CE
:109D600084808480848078800080FE8010801080D1
:109D7000108010800A0B160C01FE3F0040803F004F
:109D80000000FFC000007F8000807F8040003F8097
:109D90000A0B160C01FE3F00408040803F0000008F
:109DA000FFC000007F80408040803F800A0B160C7F
:109DB00001FE784084408440844084408440844054
:109DC00084407840004000400A0B160C01FE7840A9
:109DD0008440844084408440784000007FC000403C
:109DE000004000400A0B160C01FE7840844084407D
:109DF00084408440784000004000400040003FC064
:109E00000A0B160C01FE7840844084408440784060
:109E100000007FC000407FC040003FC00A0B160C0E
:109E200001FE7840844084408440844078400000B3
:109E300040407FC040403FC00B0B160C01FEFE802F
:109E400010801080108028E0288044804480828028
:109E5000008000800B0B160C01FEFE80108010E0CD
:109E600028804480828000007F8000800080008005
:109E70000B0B160C01FEFE80108010E02880448041
:109E8000828000007F80408040803F800B0B160C5A
:109E900001FEFE80108010E0288044808280000057
:109EA0003F00408040803F000A0B160C01FEFD4041
:109EB00011401140114029C02940454045404540CE
:109EC000014001400A0B160C01FEFE4010401040FC
:109ED000104029C028404440444082400040004097
:109EE0000A0B160C01FEFE40104011C028404440F1
:109EF000824000004000400040003FC00A0B160CAA
:109F000001FEFE40104011C0284044408240000045
:109F10003F80404040403F800A0B160C01FEFD4050
:109F2000114011401740294029404540454081409B
:109F300001400140090A140C01FF7F0008000800DD
:109F4000140022004100080008000800FF80090BEF
:109F5000160C01FEFF8008001400E3800000FF8063
:109F600008008800800080007F80090B160C01FE2D
:109F7000FF8008001400E3800000FF8008007F00DD
:109F8000808080807F00090B160C01FEFF80080096
:109F9000F7800000FF800000FF800080FF808000CD
:109FA0007F80090B160C01FEFE801080108010804F
:109FB0002880288044804480828000800080090BB3
:109FC000160C01FEFE801080108028804480828064
:109FD00000007F80408040803F800B0A140C01FF0E
:109FE0000E0000007FC004000A00110064C00400DD
:109FF0000400FFE00A0B160C01FE1E000000FFC06B
:10A000000C00120061800000FFC004000400040086
:10A010000A0B160C01FE1E0000007F800C007380EE
:10A020000000FFC004007F80008000800A0B160C37
:10A0300001FE0400FFC00C007380FFC004007F809D
:10A0400000807F8040003F800A0B160C01FE3840E4
:10A050000040FE4010401040104028402440424044
:10A06000804000400A0B160C01FEF90009000900AF
:10A07000F90009C0110011002100C1000100010018
:10A080000A0B160C01FEFA4082408240FBC082405F
:10A09000824082407A400240024002400A0B160C85
:10A0A00001FEF2408240F3C0824082407A400000CC
:10A0B0007FC0004000400040090B160C01FEF880F4
:10A0C00080808080F880838080808080788000809D
:10A0D000008000800A0A140C01FF7F8040007F800E
:10A0E000400040003F80000004000400FFC00A0A56
:10A0F000140C01FF7F80400040007F804000400042
:10A100003F8000000000FFC00A0B160C01FE7F809C
:10A1100040007F8040003F800000FFC00000400002
:10A1200040007F800B0B160C01FEFC8000804880F5
:10A13000488048E048804880FC80008000800080A3
:10A140000A0B160C01FEFD4001404940494049C040
:10A1500049404940FD400140014000400A0B160CB7
:10A1600001FEFD400140494049C04940FD400140D9
:10A170004140400040003FC00A0C180C01FE004066
:10A180007E40244024402440FF4008403FC000401F
:10A190003FC020003FC00C0B160C01FE38400040B1
:10A1A000FE40004038404470444044404440384001
:10A1B00000400B0B160C01FE38800080FEE028806A
:10A1C00044804480388020803F8020801F800A0B9C
:10A1D000160C01FE31400140FDC03140494049406C
:10A1E000314000001F8020401F800A0B160C01FE2A
:10A1F0001E000000FFC01E002100210021001E00E3
:10A2000004000400FFC00B0B160C01FE3880008018
:10A21000FE80288044E0448038801080FE800080EA
:10A2200000800B0B160C01FE1080FE8028804480FD
:10A2300044E038801080FE80400040003F800A0BE0
:10A24000160C01FE1E000000FFC0330040803F00DE
:10A250000000FFC00400040004000A0B160C01FEFD
:10A26000FE80808080C0808080807E8000004000F2
:10A27000400040003F800000060900FE07019103F6
:10A280002220FFFF08FE07FF000000060000010774
:10A2900007060200808080808000800302020601A1
:10A2A00005A0A00507070600005050F850F85050D0
:10A2B0000507070600002078A07028F02005070792
:10A2C000060000C0C81020409818050707060000C7
:10A2D0006090A040A89068020303060104C040807B
:10A2E0000307070601002040808080402003070705
:10A2F0000601008040202020408005050506000161
:10A3000020A870A8200505050600012020F82020BF
:10A310000203030602FFC04080050101060003F8A6
:10A32000020202060200C0C0050505060001081071
:10A33000204080050707060000708898A8C888702C
:10A3400003070706010040C040404040E005070702
:10A35000060000708808708080F805070706000076
:10A36000F81020100808F00507070600001030500C
:10A3700090F81010050707060000F880F00808881C
:10A3800070050707060000304080F08888700507D8
:10A3900007060000F8081020202020050707060007
:10A3A000007088887088887005070706000070882C
:10A3B0008878081060020505060200C0C000C0C011
:10A3C0000206060602FFC0C000C040800407070660
:10A3D000000010204080402010050303060002F812
:10A3E00000F8040707060100804020102040800587
:10A3F00007070600007088081020002005060606E2
:10A40000000070880868A8700507070600007088BB
:10A4100088F8888888050707060000F08888F08893
:10A4200088F0050707060000708880808088700526
:10A430000707060000E09088888890E00507070677
:10A440000000F88080F08080F8050707060000F81B
:10A450008080F0808080050707060000708880B843
:10A46000888870050707060000888888F88888882B
:10A470000107070602008080808080808005070732
:10A480000600003810101010906005070706000045
:10A490008890A0C0A09088050707060000808080F3
:10A4A000808080F805070706000088D8A88888887B
:10A4B000880507070600008888C8A89888880507C7
:10A4C00007060000708888888888700507070600DE
:10A4D00000F08888F08080800507070600007088FB
:10A4E0008888A89068050707060000F08888F0A013
:10A4F0009088050707060000788080700808F0053E
:10A500000707060000F82020202020200507070666
:10A5100000008888888888887005070706000088FA
:10A520008888888850200507070600008888888862
:10A5300088A85005070706000088885020508888A2
:10A540000507070600008888885020202005070797
:10A55000060000F80810204080F8030707060100F5
:10A56000E08080808080E00507070600008850F8C2
:10A5700020F82020030707060100E02020202020EB
:10A58000E0050303060004205088050101060000D1
:10A59000F80202020602058040050505060000706B
:10A5A000087888780507070600008080B0C888888A
:10A5B000F005050506000070808088700507070615
:10A5C000000008086898888878050505060000706E
:10A5D00088F880700507070600003048E0404040DA
:10A5E000400506060600FF70888878087005070792
:10A5F0000600008080B0C88888880107070602002E
:10A60000800080808080800308080601FF200020F1
:10A61000202020A040040707060000808090A0C0F2
:10A62000A090030707060100C04040404040E005FD
:10A630000505060000D0A8A8A8A805050506000085
:10A64000B0C888888805050506000070888888706D
:10A650000506060600FFF08888F0808005060606DD
:10A6600000FF788888780808050505060000B0C84E
:10A6700080808005050506000070807008F00507E1
:10A68000070600004040E040404830050505060050
:10A690000088888898680505050600008888885025
:10A6A000200505050600008888A8A85005050506B0
:10A6B000000088502050880506060600FF8888881C
:10A6C000780870050505060000F8102040F803071B
:10A6D0000706010020404080404020010707060295
:10A6E0000080808080808080030707060100804012
:10A6F00040204040800505050600012010F810208C
:10A700000505050600012040F84020000000060075
:10A71000000000000600000000000600000000002D
:10A720000600000000000600000000000600000017
:10A730000000060000000000060000000000060007
:10A7400000000000060000000000060000000000FD
:10A7500006000000000006000000000006000000E7
:10A7600000000600000000000600000000000600D7
:10A7700000000000060000000000060000000000CD
:10A7800006000000000006000000000006000000B7
:10A7900000000600000000000600000000000600A7
:10A7A000000000000600000000000600000000009D
:10A7B0000600000000000600000000000600000087
:10A7C0000000060000000000060000000000060077
:10A7D00000030303060000E0A0E0030404060203F4
:10A7E000E0808080030404060000202020E00303B2
:10A7F00003060000804020020202060102C0C005DC
:10A800000606060000F808F80810200505050600F1
:10A8100000F808302040040505060000102060A064
:10A820002005050506000020F88808300504040608
:10A830000000F82020F805050506000010F830504B
:10A840009005050506000040F84850400504040640
:10A850000000701010F8040505060000F010F0105C
:10A86000F0050404060000A8A80830050101060050
:10A8700003F8050707060000F808283020204005E7
:10A88000070706000008102060A020200507070623
:10A89000000020F88888081020050606060000F849
:10A8A00020202020F805070706000010F81030507F
:10A8B000901005070706000040F8484848489005F2
:10A8C000070706000020F820F820202005060606CD
:10A8D00000007848880810600507070600004078E7
:10A8E0009010101020050606060000F80808080859
:10A8F000F805070706000050F850501020400506E4
:10A9000006060000C008C80810E00506060600009C
:10A91000F8081020508805070706000040F8485046
:10A920004040380506060600008888480810600583
:10A9300006060600007848A81810600507070600FC
:10A940000010E020F8202040050606060000A8A818
:10A95000A80810200507070600007000F820202036
:10A9600040030707060100808080C0A080800507A3
:10A97000070600002020F82020408005060606007B
:10A98000007000000000F8050606060000F80850F8
:10A9900020508005070706000020F8102070A8202E
:10A9A000030707060100202020202040800506061E
:10A9B00006000020108888888805070706000080A8
:10A9C00080F880808078050606060000F8080808F0
:10A9D000106005050506000140A0100808050707DE
:10A9E00006000020F82020A8A82005060606000082
:10A9F000F80808502010040606060100E000E000F8
:10AA0000E01005060606000020408088F8080506CC
:10AA100006060000080850205080050606060000C3
:10AA2000F840F84040380507070600004040F84865
:10AA3000504040050707060000701010101010F875
:10AA4000050606060000F808F80808F805070706D6
:10AA500000007000F80808102004070706000090A6
:10AA600090909010204005060606000020A0A0A8A7
:10AA7000A8B00507070600008080808890A0C00568
:10AA80000606060000F888888888F805060606008D
:10AA900000F88888081020050606060000C0000897
:10AAA0000810E0040303060004209040030303069B
:10AAB0000004E0A0E005050506000148A8909068A4
:10AAC0000507070600005000700878887804080819
:10AAD0000601FF609090E09090E08005050506007B
:10AAE0000070806088700506060600FF888898E878
:10AAF000888005050506000078A090887005070786
:10AB00000600FE30488888F080800508080600FEB0
:10AB100078888888780808700505050600013820BF
:10AB200020A04004030306000310D0100408080608
:10AB300000FF1000301010109060030303060004A3
:10AB4000A040A00507070600002070A0A0A8702064
:10AB50000507070600004040E040E0407805070791
:10AB60000600007000B0C888888805070706000046
:10AB7000500070888888700507070600FFB0C888F5
:10AB800088F080800507070600FF689888887808A5
:10AB9000080506060600007088F88888700503031B
:10ABA00006000258A8D005050506000070888850E8
:10ABB000D8050707060000500088888898680507B0
:10ABC00007060000F88040204080F80505050600D3
:10ABD00000F850505098050707060000F80088500C
:10ABE0002050880507070600FF8888888878087045
:10ABF00005060606000008F020F8202005050506D9
:10AC00000000F840784888050505060000F8A8F817
:10AC100088880505050600012000F80020000000D6
:10AC2000060000060A0A0600FEFCFCFCFCFCFCFC1C
:10AC3000FCFCFC000C0B00FE070192032120FFFF2F
:10AC40000AFF07FF00000006000A010707060200CE
:10AC500080808080800080030202060105A0A0059C
:10AC600007070600005050F850F850500507070637
:10AC700000002078A07028F020050707060000C01B
:10AC8000C810204098180507070600006090A040F3
:10AC9000A89068020303060104C04080030707066A
:10ACA00001002040808080402003070706010080CB
:10ACB00040202020408005050506000120A870A83E
:10ACC000200505050600012020F8202002030306C8
:10ACD00002FFC04080050101060003F802020206DF
:10ACE0000200C0C0050505060001081020408005CF
:10ACF0000707060000708898A8C888700307070631
:10AD0000010040C040404040E005070706000070D9
:10AD10008808708080F8050707060000F8102010EA
:10AD20000808F005070706000010305090F81010D2
:10AD3000050707060000F880F00808887005070777
:10AD4000060000708080F088887005070706000004
:10AD5000F8081020202020050707060000708888CA
:10AD600070888870050707060000708888780808D2
:10AD700070020505060200C0C000C0C0020606063B
:10AD800002FFC0C000C0408004070706000010207A
:10AD90004080402010050303060002F800F8040775
:10ADA00007060000804020102040800507070600AD
:10ADB0000070880810200020050707060000708832
:10ADC0000868A8A870050707060000708888F8883A
:10ADD0008888050707060000F08888F08888F00555
:10ADE00007070600007088808080887005070706C6
:10ADF0000000F08888888888F0050707060000F8BA
:10AE00008080F08080F8050707060000F88080F059
:10AE1000808080050707060000708880B8888870E9
:10AE2000050707060000888888F8888888010707D2
:10AE30000602008080808080808005070706000071
:10AE4000381010101090600507070600008890A0C9
:10AE5000C0A0908805070706000080808080808061
:10AE6000F805070706000088D8A88888888805079D
:10AE7000070600008888C8A8988888050707060084
:10AE80000070888888888870050707060000F088A9
:10AE900088F080808005070706000070888888A8F1
:10AEA0009068050707060000F08888F0A0908805E4
:10AEB0000707060000788080700808F0050707067D
:10AEC0000000F82020202020200507070600008829
:10AED0008888888888700507070600008888888821
:10AEE0008850200507070600008888888888A850B1
:10AEF0000507070600008888502050888805070746
:10AF000006000088888850202020050707060000DA
:10AF1000F80810204080F8030707060000E0808052
:10AF2000808080E0050505060001804020100803B0
:10AF30000707060000E02020202020E0050303068C
:10AF40000004205088050101060000F802020206F4
:10AF50000205804005050506000070087888780520
:10AF600007070600008080B0C88888F00505050640
:10AF700000007080808870050707060000080868D8
:10AF8000988888780505050600007088F8807005A7
:10AF900007070600003048E040404040050606062E
:10AFA00000FF708888780870050707060000808019
:10AFB000B0C888888801070706020080008080806A
:10AFC00080800308080601FF200020202020A040E8
:10AFD000040707060100808090A0C0A09003070727
:10AFE000060100C04040404040E005050506000065
:10AFF000D0A8A8A8A8050505060000B0C8888888BC
:10B00000050505060000708888887005060606009C
:10B01000FFF08888F080800506060600FF788888A3
:10B02000780808050505060000B0C8808080050581
:10B030000506000070807008F00407070600004055
:10B0400040E04040403005050506000088888898AB
:10B050006805050506000088888850200505050656
:10B0600000008888A8A85005050506000088502023
:10B0700050880506060600FF888888780870050550
:10B0800005060000F8102040F8030707060100201D
:10B0900040408040402001070706020080808080F9
:10B0A00080808003070706010080404020404080E8
:10B0B00005020206000368900B0B160C00FF9FE0D0
:10B0C0004020002080208020802080208020802040
:10B0D000802080E00B0B160C00FF8FE041000FC0BA
:10B0E000C24044404FE040004FE048206820CFE09D
:10B0F0000B0B160C00FF7FC00000FFE000007FC0BC
:10B1000000007FC000007FC040407FC00B0B160CCA
:10B1100000FFFFE0040004000400440047E0440096
:10B12000440044004400FFE00B0B160C00FF080035
:10B13000FFE008001000110021006FE0A1002100D5
:10B1400021002FE00B0B160C00FFFFE008000800A9
:10B150000A000900088008400800080008000800EC
:10B160000B0B160C00FFFFE00A007FC04A407FC0B7
:10B170000800FFE0108031000E00F1E00B0B160C10
:10B1800000FF21002FE041004FE0C92049204FE09F
:10B190004100450042004DE00B0B160C00FF7FC044
:10B1A000444044407FC0444044407FC04440444009
:10B1B000844084C00B0B160C00FF0400FFE08920C4
:10B1C00052409C203080DF800000444044407FC0DB
:10B1D0000B0B160C00FFF7C040404240424072404B
:10B1E000D7E05020502057A0702000E00B0B160C29
:10B1F00000FF4100F2804440ABA0A000FE202AA046
:10B200002EA0FAA02E202A600B0B160C00FF0400C3
:10B210000400FFE02080208011000A0004000A00E2
:10B220003180C0600B0B160C00FF290029004FE095
:10B230005100C10041005FE0410041004100410078
:10B240000B0B160C00FF208011007FC011001100B5
:10B250001100FFE011001100210041000B0B160C42
:10B2600000FF4100EFE0482042006FE0C44044404E
:10B270004E80410046C0D8200B0B160C00FF410049
:10B2800063C099400FE0F1405BC04900EFC0590036
:10B290004D0073E00B0B160C00FF42007BE0A48016
:10B2A000FFC004407FC044007FE0142024E0C400BD
:10B2B0000B0B160C00FF00C07F00400040007FE039
:10B2C000400040005FC0504090409FC00B0B160CE8
:10B2D00000FF2040AA40A9402040FA402140706071
:10B2E00068C0A340204020400B0B160C00FF41E03B
:10B2F0007D2091201120FD2011205D2051205160E2
:10B300005D00F1000B0B160C00FF20802080410037
:10B310008A205140208041009A60E3800000FFE0D5
:10B320000B0B160C00FF53E0520052007BE0432051
:10B3300042A072A05240524054A094A00B0B160C95
:10B3400000FF04000400FFE0150015001500248034
:10B3500024805F40842004000B0B160C00FF7FC08C
:10B3600040407FC0404040407FC01100912051408C
:10B370003180FFE00B0B160C00FF7FC000000000C7
:10B380000000FFE0040004004440444084201C000E
:10B390000B0B160C00FFFFE0802088A0AAA09120D4
:10B3A00091209120AAA0AAA0802080E00B0B160C6F
:10B3B00000FF440047E08420EA4041804E60800066
:10B3C000EFE008202820CFE00B0B160C00FF410017
:10B3D00049004960EBA05D20492049604900682090
:10B3E000C8200FE00B0B160C00FF20802480248067
:10B3F000F48024E02480248024803480E4800FE0E2
:10B400000B0B160C00FFFFE00200020004000D0011
:10B4100014802440C4200400040004000B0B160C0C
:10B4200000FFF9008A00ABE0AC40AA40AA40AA4065
:10B43000AA80210052808C600B0B160C00FF2400A8
:10B4400024003F80440084000400FFE00A00110053
:10B450002080C0600B0B160C00FF240024003FC0AE
:10B4600044000400FFE0090009001120212040E011
:10B470000B0B160C00FF20003DE051209120112005
:10B48000FF201120292025E0452080000B0B160C01
:10B4900000FF1800FFE0802080209F209120912055
:10B4A00091209F20802080E00B0B160C00FF7FC0B6
:10B4B00040407FC0400040207FE00100FFE02100CD
:10B4C000110003000B0B160C00FF04808FE04900F5
:10B4D00019002FC0090009002FC0490089000FE0A2
:10B4E0000B0B160C00FF10003F8051000E00318046
:10B4F000C0603F8024803F8024803F800B0B160C6F
:10B5000000FF2280FA4007E0FA808A808A80FA8071
:10B510002280B280AAA064E00B0B160C00FF222050
:10B5200047409280EFE0220047C0EC4007C0344023
:10B53000C7C004400B0B160C00FF08000FC008002A
:10B540000800FFE008000E0009800840080008001D
:10B550000A0B160C00FFFF80008000808080808036
:10B56000FF8080008000804080407FC00B0B160C65
:10B5700000FF47C04100EFE0410045006960C9207D
:10B580004D6049204FE0C8200B0B160C00FF08004F
:10B59000040004000A000A000A00110011002080C3
:10B5A000404080200B0B160C00FF22402200F7E0E9
:10B5B000220023E03520E520254028802940722004
:10B5C0000B0A140C00004440444044407FC0040077
:10B5D0000400842084208420FFE00B0B160C00FF65
:10B5E000040000007FC00400040004007FC00400C9
:10B5F00004000400FFE00B0B160C00FFFFE011003D
:10B6000001C0FE00488025000400FFE015002480F2
:10B61000C4600B0B160C00FF11007FC044407FC0BC
:10B6200044407FC00400FFE0040004000400090B54
:10B63000160C00FF1000FF8080808080FF808080DB
:10B640008080FF8080808080FF800B0B160C00FFC5
:10B650007100010003E0F9202120412051208920C0
:10B66000FA20022004C00B0B160C00FF7FC0110053
:10B67000110011001100FFE0110011002100210054
:10B6800041000B0B160C00FF21002200F44057E094
:10B69000502057C094405440244057C094400B0B56
:10B6A000160C00FF11000A007FC004000400FFE038
:10B6B00004000A0011002080C0600A0B160C00FF75
:10B6C0005FC0004084408440BF4084408C40944030
:10B6D000A4408C4081C00B0B160C00FF240027C037
:10B6E00024002400FFE000001440248047000C00E8
:10B6F00070000B0B160C00FF248004800FC0E48048
:10B7000024803FE024802480288050008FE00B0BB1
:10B71000160C00FF08000800FF8088808880FF80EA
:10B7200088808880FFA0882007E00B0B160C00FFA4
:10B7300027802480F480248074806C80A4802480FE
:10B7400024A028A030600A0B160C00FFFFC0804028
:10B7500080409E40924092409E4080408040FFC08A
:10B7600080400B0B160C00FF7FC044005FC05040B0
:10B770005FC050405FC042004A805240A6200B0B81
:10B78000160C00FF040007E004007FC0404040406A
:10B7900040407FC00000524089200B0B160C00FF78
:10B7A0004780248004800480E86020002FC024406B
:10B7B0002280310026C00B0B160C00FF7FC04A40D0
:10B7C0007FC00400FFE004003F80208024802480AC
:10B7D000FFE00B0B160C00FF22004FE048204FE06B
:10B7E000C8004FE04AA05AA06FE04AA048600B0B87
:10B7F000160C00FFF3C024402A80F100228065E08F
:10B800007220A540208023002C000B0B160C00FF9B
:10B810000400FFE080200000FFE00400240027C0B7
:10B82000240054008FE00B0B160C00FF73E0108017
:10B83000510023E0FA202AA022A022A0208021404B
:10B8400062200B0B160C00FF2200F780228036804E
:10B85000E2A025A0246068200000524089200B0B44
:10B86000160C00FF73C0420042007BE04A404A4091
:10B870007A404A404240444088400B0B160C00FF7F
:10B880000800FFE008001FC030405FC090401FC0AC
:10B890001040104010C00B0B160C00FF02007FE0A0
:10B8A000420042005FC0420047004A80524062208E
:10B8B00082000B0B160C00FFF3C096409180A6602F
:10B8C000A10097C091009500E7E0810081000B0B7B
:10B8D000160C00FF0F8088804F8008808F8040000A
:10B8E0001FC03540554095403FE00B0B160C00FF44
:10B8F00027E02080F880208020803880E080208031
:10B900002080208061800B0B160C00FF1FE091004F
:10B9100057C0144017C0944057C01100554099209B
:10B9200023000B0B160C00FF208027E0F240218043
:10B9300022403420E24022402240224064400B0B4F
:10B94000160C00FF410041004FE0E920492049204A
:10B950006FE0C92049204920CFE00B0B160C00FFF7
:10B960002100F1004FE0A920F9202FE03920E92043
:10B9700029202FE028200B0B160C00FF8FE0492018
:10B980000920CBA049204FE048204BA04AA06BA043
:10B9900050E00B0B160C00FF7FC004004440244015
:10B9A00024800400FFE004000400040004000B0BEA
:10B9B000160C00FF820042001FE0C2005FC0524030
:10B9C0005FC047004A805240BFE00B0B160C00FFDF
:10B9D00004007FE048807FE048804F8040005FC0E7
:10B9E0004840478098600B0B160C00FF0100EFE009
:10B9F000A100A440AFE0A440AFE0A920E92002806C
:10BA00000C600B0B160C00FF14C0F6A0BC60A780E6
:10BA1000A880BFE0A920EFE009200FE009200B0B70
:10BA2000160C00FF7F8040804280628054804880F6
:10BA3000488054A062A0406080200B0B160C00FFD1
:10BA400004007FE040207FE040007DE054204CA0D7
:10BA5000546064A08D600B0B160C00FF82005FE049
:10BA6000040008409FE040200A800A804AA092A07B
:10BA700022600B0B160C00FF41004FE0E8204280D3
:10BA800044406820C7C0410041004100CFE00B0B9B
:10BA9000160C00FF50207D209120FF2011207D20DA
:10BAA0005520552054205C2010E00B0B160C00FF95
:10BAB0003F8020803F802080FFE048007BC04940DD
:10BAC00079404880FB600B0B160C00FF040004005B
:10BAD00004002480244044404420842004000400C6
:10BAE0001C000B0B160C00FF040004000400FFE018
:10BAF00004000A000A00110011002080C060090A39
:10BB0000140A0000888049000800FF80008000803F
:10BB10007F8000800080FF800B0B160C00FF21004F
:10BB20001200FFE0000078804A807A804A807A80A4
:10BB3000488059800B0B160C00FF27C00000000046
:10BB4000EFE02100220024402FE0202050008FE071
:10BB50000B0B160C00FFFFE004007FC044407FC0C9
:10BB600044407FC0440024001800E7C00B0B160CB3
:10BB700000FF04000F8070800900060019E0E22039
:10BB80000C20024001803E000B0B160C00FF004011
:10BB9000F8400BE00840884052405140214050405E
:10BBA000484089C00A0B160C00FF84008440848042
:10BBB000F5008600840084009400A440C44083C043
:10BBC0000B0B160C00FF11207D001100FFE0290077
:10BBD000FD4049407C8008A0FD600A200B0B160C3C
:10BBE00000FF17C02440244067C0A1002FE02100BF
:10BBF00023802540292021000B0B160C00FF080094
:10BC0000FFE0100027C020806100AFE0210021008C
:10BC1000210023000B0B160C00FF24002FE0B400C2
:10BC2000A480A4A0AAC02A802880294032402420D1
:10BC30000B0B160C00FF7FE080003FC020403FC090
:10BC400010001FC010402880470038E00B0B160C76
:10BC500000FF7FE040004000400040004000400006
:10BC600040004000400080000B0B160C00FFFFE07E
:10BC700004007FC044407FC044407FC04400240093
:10BC80001800E7E00B0B160C00FF11E0FD0045006B
:10BC900029E0FD4011407D40114055409240344024
:10BCA0000B0B160C00FF21005FE04000CFC04000EE
:10BCB0004FC040004FC048404FC048400B0B160CCF
:10BCC00000FF04007FC040407FC040407FC0404034
:10BCD0007FC004405220BFA00B0B160C00FF7FC09A
:10BCE00044407FC044407FC004001B00E0E01100DE
:10BCF000110061000B0B160C00FFFFE004000800B0
:10BD00007FE049204F2049204F20492049207FE0F3
:10BD10000B0B160C00FFFDE0564079403880554073
:10BD20009220FFE0040027C02400FFE00B0B160C5C
:10BD300000FFFB8052007BE01240FA4014403F803D
:10BD400020803F8020803F800B0B160C00FF1FE0FF
:10BD5000200027C06440A7C020002FE0282027C073
:10BD6000210023000B0B160C00FFF3E08220822041
:10BD7000FA20822082208A20B220C2E00200020043
:10BD80000B0B160C00FF248046A095C0E48027E032
:10BD90004480F5C006A03480C48007E00B0B160C6D
:10BDA00000FF27C0410087E0E02022804580F2802C
:10BDB0000FE03080C14002200B0B160C00FF020088
:10BDC0000200220023C022002200220022002200C2
:10BDD0002200FFE0090B160C00FF08000800FF809E
:10BDE000888088808880FF80888088808880FF8025
:10BDF0000B0B160C00FF210053A04100F7E051008F
:10BE000053C0564053C05A4053C042400B0B160C0F
:10BE100000FF7FC0040004000400FFE00A000A00E5
:10BE200012002220422081E00A01020C0104FFC01E
:10BE30000B0B160C00FFFFE004007FC040404440A5
:10BE400044404440444044401B00E0E00B0B160CCF
:10BE500000FF7BE0948004007FC00400FFE001004D
:10BE6000FFE02100110007000B0B160C00FF210062
:10BE700047C091002FE06080AFE0208024802280C6
:10BE8000208023800B0B160C00FF27C02440F7C036
:10BE90002EE02AA03EE0E1002FE02380254069202B
:10BEA0000B0B160C00FF140027E02A006200A3C051
:10BEB0002200220023E022002200220000000609C6
:10BEC00000FE000000000001090008FE0000050857
:10BED0000806000040F0C888889878100508080611
:10BEE0000000C0F88888888888F8050505060001E4
:10BEF0002030F830200508080600002070F82020C7
:10BF00002020E00509090600FF2070A8A8B888884D
:10BF100070200509090600FFE080C0B0A82830287D
:10BF2000280509090600FFF8A88888888888A8F8E5
:10BF3000050A0A0600FE205050505088A8A88870B4
:10BF400003030306000340A04074686520706F7708
:10BF5000657200000000000000000000000000000A
:10BF600000000000000000000000000020000000B1
:10BF700000000000000000000000000000000000C1
:10BF8000000000000000000000000000000000634E
:10BF90006F7570657A206C27616C696D656E746170
:10BFA00074696F6E000000000000000000000000D7
:10BFB0000000200000000000000000000000000061
:10BFC0000000000000000000000000000000000071
:10BFD00000000000006C7565676F20617061677517
:10BFE00065000000000000000000000000000000EC
:10BFF00000000000000000007175696E6469207324
:10C000007065676E6572650000000000000000004A
:10C01000000000000000000000000074686520704F
:10C020006F77657200000000000000000000000053
:10C03000000000000000000000000000000061207F
:10C04000656E657267696100000000000000000015
:10C0500000000000000000000000000000000000E0
:10C06000007A6574206465207374726F6F6D20753B
:10C0700069740000000000000000000000000000E3
:10C080000000000067756375206B61706174696EF4
:10C0900000000000000000000000000000000000A0
:10C0A00000000000000000DFD000000000000000E1
:10C0B0000000000000000000000000000000000080
:10C0C00000000000000000000000D0B2D18BD0BA08
:10C0D000D0BBD18ED187D0B8D182D0B520D0BFD03F
:10C0E000B8D182D0B0D0BDD0B8D0B5000073746FD5
:10C0F000702C207468656E207475726E206F666691
:10C10000000000B5B6B9CB00000000000000000040
:10C110000000000000000000006465206C27696DCD
:10C120007072657373696F6E2C207075697300642B
:10C13000616E6E20417573736368616C74656E0027
:10C140000000000000646574656E6761206C61200A
:10C15000696D70726573696F6E2C006C6120737409
:10C16000616D70612C000000000000000000000004
:10C170000073746F702C207468656E207475726E15
:10C18000206F6666000000696D7072657373616F81
:10C190002065206465736C6967756500006B6B656D
:10C1A0006E2074652073746F7070656E2C000000D3
:10C1B0000000006261736B692062656B6C65796970
:10C1C0006E0000000000000000E4E620FE208DE785
:10C1D000000000000000000000000000000000D18E
:10C1E00081D182D0BED0BF2C20D0B7D0B0D182D0E8
:10C1F000B5D0BC00005761697420666F7220707200
:10C20000696E74696E6700000000000000000000A5
:10C21000000000000000FCFDCAF3F2F691000000EF
:10C22000000000000000000000000000000000000E
:10C2300000000000000000417474656E64657A209F
:10C240006C2761727265740000000000000000003D
:10C25000000000000000000057617274656E2066E7
:10C26000757220447275636B73746F707000000098
:10C27000000000000000000000457370657265203A
:10C2800061207175652073650000000000000000EA
:10C2900000000000000000000000417474656E643E
:10C2A000657265206665726D617461000000000052
:10C2B00000000000000000000000005761697420C9
:10C2C000666F72207072696E74696E67000000009C
:10C2D00000000000000000000000000041677561E0
:10C2E0007264652061207061726164612064610024
:10C2F0000000000000000000000000000057616323
:10C30000687420746F742068657420616664727547
:10C310002D0000000000000000000000000044614B
:10C32000686120736F6E72612C206475726475721F
:10C330006D6100000000000000000000000000EB44
:10C340009E20CDA020938B00000000000000000084
:10C3500000000000000000000000000000000000DD
:10C36000D094D0BED0B6D0B4D0B8D182D0B5D1811F
:10C37000D18C20D0BFD0B5D187D0B0D182D0B80079
:10C380000053617665205072696E74696E67206132
:10C390006E64204F6666000000000000E5E6B5BA56
:10C3A000202020200000000000000000000000000D
:10C3B00000000000000000456E72656769737472CA
:10C3C0006572206574204F464600000000000000A2
:10C3D000000053706569636865726E20756E642035
:10C3E00077656700000000000000000000477561ED
:10C3F000726461722079206170616761720000006F
:10C40000000000000000000053616C76612073742E
:10C41000616D70612065204F6666000000000000BD
:10C4200000000053617665205072696E74696E6712
:10C4300020616E64204F66660000000000005361BA
:10C440006C766172206520446573617469766172EF
:10C450000000000000000000004F70736C61616E0E
:10C4600020656E204F66660000000000000000009E
:10C47000000000004B6179646574207665204B6193
:10C48000706174000000000000000000000000EB7C
:10C490009E20DEDC20FE208DE70000000000000072
:10C4A00000000000000000000000D0A1D0BED18537
:10C4B000D180D0B0D0BDD0B8D182D18C20D0B8201E
:10C4C0004F6666000041646A757374205A204F6697
:10C4D00066736574286D6D2900000000005ACEC097
:10C4E000C1286D6D29000000000000000000000060
:10C4F0000000000000416A7573746572205A204F75
:10C50000666673657420286D6D290000005A2D56EB
:10C5100065727361747A20286D6D29000000000037
:10C520000000000000416A75737465205A204F6650
:10C5300066736574286D6D2900000000004F666603
:10C54000736574205A20286D6D29000000000000DA
:10C55000000000000041646A757374205A204F6621
:10C5600066736574286D6D290000000000416A75CE
:10C5700073746172205A206F6666736574286D6DDE
:10C58000290000000050617373656E205A204F66C9
:10C590006673657420286D6D29000000005A204FD5
:10C5A0006673657420286D6D2920617961726C61F4
:10C5B00000000000005AEA20CCB820E2E0000000B1
:10C5C00000000000000000000000000000D0A1D02A
:10C5D000BCD0B5D189D0B5D0BDD0B8D0B5205A28FF
:10C5E0006D6D290000473238205A20463530300D15
:10C5F0000A473238205820592046313030300A4717
:10C6000032390A47312058353020593530204631EB
:10C610003030300A4731205A302046313030004E19
:10C620004F4E45004E4F4E45004E4F4E45004E4F2B
:10C630004E45004E4F4E45004E4F4E45004E4F4E1C
:10C6400045004572726F723A20636F6D6D656E744E
:10C65000206C696E6520746F6F206C6F6E670A00C6
:10C660002569670046696C616D656E745573656414
:10C670003A0054494D453A004578747275646572C4
:10C680003054656D70657261747572653A00496EFB
:10C6900066696C6C44656E736974793A004C6179B3
:10C6A0006572206865696768743A0046696C616DF7
:10C6B000656E74547970653A004D616368696E65A2
:10C6C000547970653A004E657874000000000000EF
:10C6D00000000000000000000000000091FAFB00D4
:10C6E000000000000000000000000000000000004A
:10C6F000000050726F636861696E00000000000006
:10C7000000000000000000004E61636873746572F1
:10C710000000000000000000000000000000507257
:10C720006F78696D6F0000000000000000000000DD
:10C730000000000050726F7373696D6F000000009D
:10C74000000000000000000000004E65787400004A
:10C7500000000000000000000000000000000000D9
:10C7600050726F78696D6F000000000000000000DB
:10C77000000000000000766F6C67656E6465000065
:10C78000000000000000000000000000536F6E7207
:10C79000616B690000000000000000000000000064
:10C7A00000004E65787400000000000000000000EA
:10C7B0000000000000000000D181D0BBD0B5D0B493
:10C7C000D183D18ED189D0B8D0B900000000507289
:10C7D0006576696F757300000000000000000000BE
:10C7E00000000000DEFAFB00000000000000000076
:10C7F00000000000000000000000507265636564E6
:10C80000656E7400000000000000000000000000E1
:10C810004269736865726967650000000000000086
:10C82000000000000000416E746572696F720000C4
:10C83000000000000000000000000000507265636E
:10C840006564656E74650000000000000000000073
:10C85000000050726576696F75730000000000007B
:10C860000000000000000000416E746572696F7284
:10C870000000000000000000000000000000766FD3
:10C880006F726761616E64000000000000000000CC
:10C89000000000004F6E63656B690000000000003F
:10C8A0000000000000000000000050726576696F13
:10C8B0007573000000000000000000000000000090
:10C8C000D09DD0B0D0B7D0B0D0B4000000000000F0
:10C8D0000000000000004D61696E000000000000D3
:10C8E00000000000000000000000AEAFB00000003B
:10C8F00000000000000000000000000000004D6586
:10C900006E75000000000000000000000000000044
:10C91000000048617570746D656E75000000000060
:10C920000000000000004D656E75207072696E6336
:10C930006970616C0000000000004D656E7520702C
:10C9400072696E636970616C650000000000D2B2AC
:10C95000DD000000000000000000000000000000FA
:10C9600000004D656E75207072696E636970616C50
:10C97000000000000000486F6F66646D656E750012
:10C9800000000000000000000000416E6100000097
:10C990000000000000000000000000000000A0D621
:10C9A0000000000000000000000000000000000087
:10C9B0000000D09CD0B5D0BDD18E0000000000009A
:10C9C00000000000000054656D706572617475723E
:10C9D000653A000000000000000054656D7065724B
:10C9E00061747572653A0000000000000000546533
:10C9F0006D70657261747572653A00000000000028
:10CA0000000054656D70657261747572653A00005E
:10CA100000000000000054656D70657261747572ED
:10CA2000653A000000000000000054656D706572FA
:10CA300061747572653A00000000000000005465E2
:10CA40006D70657261747572653A000000000000D7
:10CA5000000054656D70657261747572653A00000E
:10CA600000000000000054656D706572617475729D
:10CA7000653A000000000000000054656D706572AA
:10CA800061747572653A0000000000000000546592
:10CA90006D70657261747572653A00000000000087
:10CAA000000054656D70657261747572653A0000BE
:10CAB00000000000000055736167653A0000000047
:10CAC000000055736167653A00000000000055736F
:10CAD0006167653A00000000000055736167653AC0
:10CAE00000000000000055736167653A0000000017
:10CAF000000055736167653A00000000000055733F
:10CB00006167653A00000000000055736167653A8F
:10CB100000000000000055736167653A00000000E6
:10CB2000000055736167653A00000000000055730E
:10CB30006167653A00000000000055736167653A5F
:10CB400000000000000046696C616D656E743A007B
:10CB5000000000000046696C616D656E743A00006B
:10CB60000000000046696C616D656E743A0000005B
:10CB700000000046696C616D656E743A000000004B
:10CB8000000046696C616D656E743A00000000003B
:10CB90000046696C616D656E743A0000000000002B
:10CBA00046696C616D656E743A00000000000046D5
:10CBB000696C616D656E743A0000000000004669A2
:10CBC0006C616D656E743A00000000000046696C8F
:10CBD000616D656E743A00000000000046696C618A
:10CBE0006D656E743A00000000000046696C616D6E
:10CBF000656E743A00000000000044656E7369744D
:10CC0000793A00000000000044656E736974793A57
:10CC100000000000000044656E736974653A00000E
:10CC20000000000044656E736974793A00000000EA
:10CC3000000044656E736974793A000000000000DA
:10CC400044656E736974793A000000000000446521
:10CC50006E736974793A00000000000044656E73D9
:10CC60006974793A00000000000044656E736974CD
:10CC7000793A00000000000044656E736974793AE7
:10CC800000000000000044656E736974793A00008A
:10CC90000000000044656E736974793A000000007A
:10CCA00000005072696E7454696D653A00000000AE
:10CCB0000000000000005072696E7454696D653A9E
:10CCC0000000000000000000000054656D7073203B
:10CCD0006427696D7072653A0000000000005072B0
:10CCE000696E7454696D653A000000000000000030
:10CCF00000005072696E7454696D653A000000005E
:10CD00000000000000005072696E7454696D653A4D
:10CD1000000000000000000000005072696E7454B2
:10CD2000696D653A000000000000000000005072CC
:10CD3000696E7454696D653A0000000000000000DF
:10CD400000005072696E7454696D653A000000000D
:10CD50000000000000005072696E7454696D653AFD
:10CD6000000000000000000000005072696E745462
:10CD7000696D653A0000000000000000000050727C
:10CD8000696E7454696D653A00000000000000008F
:10CD900000004C617965724865696768743A000003
:10CDA000000000004C617965724865696768743AF3
:10CDB000000000000000507265636973696F6E3A8D
:10CDC00000000000000000004C6179657248656950
:10CDD0006768743A0000000000004C617965724891
:10CDE00065696768743A0000000000004C6179656D
:10CDF000724865696768743A0000000000004C6181
:10CE00007965724865696768743A0000000000003F
:10CE10004C617965724865696768743A0000000082
:10CE200000004C617965724865696768743A000072
:10CE3000000000004C617965724865696768743A62
:10CE40000000000000004C61796572486569676800
:10CE5000743A0000000000004C6179657248656911
:10CE60006768743A0000000000004D616368696EF5
:10CE7000653A200000000000000000000000BEA590
:10CE80003A20000000000000000000000000000048
:10CE900000004D616368696E653A20000000000083
:10CEA0000000000000004D61736368696E653A2000
:10CEB000000000000000000000004D617175696E07
:10CEC000613A2000000000000000000000004D61F9
:10CED000636368696E613A20000000000000000092
:10CEE00000004D616368696E653A20000000000033
:10CEF0000000000000004D617175696E613A20000C
:10CF0000000000000000000000004D616368696ED1
:10CF1000653A2000000000000000000000004D61A4
:10CF20006B696E653A200000000000000000000000
:10CF30000000DCEC3A2000000000000000000000CF
:10CF4000000000000000D09CD0B0D188D0B8D0BD87
:10CF5000D0B03A2000000000000051756974000054
:10CF60000000000000000000000000000000B5B656
:10CF700000000000000000000000000000000000B1
:10CF800000005175697474657200000000000000B3
:10CF90000000000000005665726C617373656E00DE
:10CFA0000000000000000000000053616C69720086
:10CFB0000000000000000000000000000000536DB1
:10CFC00065747465726500000000000000000000D8
:10CFD00000005175697400000000000000000000AE
:10CFE00000000000000053616972000000000000B2
:10CFF000000000000000000000004F70686F7564C2
:10D00000656E000000000000000000000000636981
:10D010006B6D616B0000000000000000000000006C
:10D020000000E4E600000000000000000000000036
:10D03000000000000000D0A3D0B2D0BED0BBD0B85A
:10D04000D182D18CD181D18F00005072696E740071
:10D0500000000000000000000000CAF30000000013
:10D0600000000000000000000000496D7072657350
:10D0700073696F6E000000000000447275636B6599
:10D080006E000000000000000000496D70726573C2
:10D09000696F6E000000000000005374616D7061E4
:10D0A000000000000000000000005072696E740073
:10D0B00000000000000000000000496D7072657300
:10D0C00073616F00000000000000686574206472E6
:10D0D000756B6B656E00000000004261736B690048
:10D0E00000000000000000000000EB9E20E40000B3
:10D0F00000000000000000000000D0BFD0B5D187C4
:10D10000D0B0D182D18C00000000526573756D657E
:10D11000207072696E74696E672E2E2E00000000FA
:10D120000000E7E8CAF32E2E2E00000000000000E9
:10D13000000000000000000000005265707269737A
:10D14000652E2E2E000000000000000000000000F0
:10D150000000447275636B20666F72747365747A35
:10D16000656E2E2E2E00000000005265746F6D61FA
:10D170007220696D70726573696F6E000000000047
:10D18000000052697072656E6469207374616D701D
:10D19000612E2E2E000000000000526573756D6533
:10D1A000207072696E74696E672E2E2E000000006A
:10D1B0000000437572726963756C6F2E2E2E00002D
:10D1C00000000000000000000000446F6F72676103
:10D1D000616E206D65742E2E2E0000000000000090
:10D1E00000005375726475726D65202E2E2E00003E
:10D1F00000000000000000000000DD842E2E2E0044
:10D20000000000000000000000000000000000001E
:10D210000000D0A0D0B5D0B7D18ED0BCD0B8D180CE
:10D22000D183D18F202E2E2E000020005754434D45
:10D23000443A5749464944454641554C540A002012
:10D240005057443A00535349443A005754434D44CD
:10D250003A4A4F494E2000204D50657263656E7406
:10D260003A00204D54696D653A00204D46696C6561
:10D270003A004D5374617475733A002F2F616374D3
:10D28000696F6E3A63616E63656C0A004D333100FD
:10D290004D3138005072696E742070617573656429
:10D2A000000000000000000000000000000000007E
:10D2B0000000CAF3F1F200000000000000000000CE
:10D2C000000000000000000000000000000000005E
:10D2D000496D7072696D6572206D697320656E208D
:10D2E000706175736500000000000000000044726A
:10D2F00075636B207061757369657274000000005E
:10D300000000000000000000000000005061757384
:10D31000617220696D70726573696F6E0000000044
:10D32000000000000000000000005374616D706197
:10D3300020736F73706573610000000000000000CF
:10D3400000000000000000005072696E74207061DF
:10D35000757365640000000000000000000000001C
:10D36000000000000000496D7072696D69722070E4
:10D3700061757361646F0000000000000000000030
:10D38000000000005072696E74206F6E64657262F6
:10D39000726F6B656E00000000000000000000006E
:10D3A00000004261736B6920647572616B6C61741B
:10D3B000696C6469000000000000000000000000CB
:10D3C000EB9E20D7BDE0E60000000000000000005A
:10D3D0000000000000000000000000000000D09FDE
:10D3E000D0B5D187D0B0D182D18C20D0BDD0B020E3
:10D3F000D0BFD0B0D183D0B7D0B500004D313235D9
:10D40000005072696E74696E672E2E2E0000000047
:10D410000000000000CAF32E2E2E000000000000C5
:10D42000000000000000000000496D707265737319
:10D43000696F6E2E2E2E00000000000000447275F1
:10D44000636B656E2E2E2E000000000000000000B1
:10D4500000496D70726573696F6E2E2E2E0000008C
:10D4600000000000005374616D70612E2E2E0000CC
:10D470000000000000000000005072696E74696EC8
:10D48000672E2E2E000000000000000000496D7085
:10D4900072657373616F2E2E2E0000000000000075
:10D4A00000686574206472756B6B656E202E2E2E7D
:10D4B00000000000004261736B692E2E2E000000F8
:10D4C000000000000000000000EB9E20E42E2E2E45
:10D4D00000000000000000000000000000D09FD00D
:10D4E000B5D187D0B0D182D18C2E2E2E0000000075
:10D4F000000D0A00434845434B46494C4553495AA1
:10D50000453A0057726974696E6720746F206669C6
:10D510006C653A20006F70656E206661696C6564A9
:10D520002C2046696C653A20002066696C653A20BB
:10D5300000617070656E64004E6F772000446973FF
:10D54000636F6E6E6563746564004D3130342053D3
:10D5500030004D373032205430004D3130342054BB
:10D56000302053323130004D313034205330004DB3
:10D57000373031205430004D313034205430205376
:10D5800032313000537061726B4F6E65204F6666AA
:10D590006C696E6500537061726B4F6E65204F6EE3
:10D5A0006C696E650048617264636F6465642044F1
:10D5B000656661756C742053657474696E67732059
:10D5C0004C6F616465640A00B80B0000B80B000082
:10D5D00064000000400600000000964300009643EF
:10D5E000000020410000C8410000C8420000C842BD
:10D5F0000000C8430000B4423A0A0020286D6D299B
:10D600000020204D36303320002055004C00466964
:10D610006C616D656E74206C6F61642F756E6C6FDC
:10D620006164206C656E677468733A0A0020204D4F
:10D63000383531205A005A2D50726F6265204F667E
:10D64000667365740020440020490020204D33306B
:10D65000312050005049442073657474696E6773BB
:10D660003A0A0020460020420020480020204D3188
:10D6700034352053004D6174657269616C206865B2
:10D680006174757020706172616D65746572733A52
:10D690000A0020204D3432302053004175746F2031
:10D6A000426564204C6576656C696E673A0A0020B5
:10D6B0005A0020590020204D323036205800486F43
:10D6C0006D65206F66667365743A0A002045002018
:10D6D0005A002059002058002054002053002020D8
:10D6E0004D32303520510020453C6D61785F655FDB
:10D6F0006A65726B3E0020583C6D61785F785F6AA6
:10D7000065726B3E20593C6D61785F795F6A657226
:10D710006B3E205A3C6D61785F7A5F6A65726B3E42
:10D7200000416476616E6365643A20513C6D696EB8
:10D730005F7365676D656E745F74696D655F757342
:10D740003E20533C6D696E5F666565647261746509
:10D750003E20543C6D696E5F74726176656C5F66E5
:10D76000656564726174653E00205400205200209B
:10D77000204D323034205000416363656C65726126
:10D7800074696F6E2028756E6974732F7332293A2D
:10D7900020503C7072696E745F616363656C3E20FB
:10D7A000523C726574726163745F616363656C3E61
:10D7B00020543C74726176656C5F616363656C3E96
:10D7C0000A00204500205A0020590020204D323008
:10D7D000312058004D6178696D756D204163636536
:10D7E0006C65726174696F6E2028756E6974732F31
:10D7F0007332293A0A00204500205A00205900209F
:10D80000204D3230332058004D6178696D756D20A0
:10D810006665656472617465732028756E697473DA
:10D820002F73293A0A00204500205A002059002071
:10D83000204D393220580053746570732070657222
:10D8400020756E69743A0A0020204D323030204431
:10D85000300A0020204D32303020440020446973CB
:10D8600061626C65640A0046696C616D656E742066
:10D8700073657474696E67733A0020204D313439D2
:10D880002043203B20556E69747320696E204365E8
:10D890006C736975730A00202047323120202020E4
:10D8A0003B00FFE0FFD11000FFFEFFD0FFE0FFC113
:10D8B000FFD1E240A0C8A6A32FF800238127AC0027
:10D8C000AFFF64A5FF64FF64A4FFD0FFFE20526594
:10D8D0006164792E000000000000000000000000DC
:10D8E00000A4A5A6A70000000000000000000000A2
:10D8F00000000000002050726574652E00000000DA
:10D90000000000000000000000204265726569749C
:10D9100000000000000000000000000000206C6912
:10D9200073746F2E00000000000000000000000073
:10D93000002070726F6E746F2E00000000000000F7
:10D9400000000000002072656164792E0000000074
:10D950000000000000000000002070726F6E746113
:10D960002E0000000000000000000000002067659D
:10D97000726565642E0000000000000000000000D9
:10D98000002068617AC4B1722E000000000000001F
:10D9900000000000002052656164792E0000000044
:10D9A00000000000000000000020D0B3D0BED182F3
:10D9B000D0BED0B22E0000000000000000507269FE
:10D9C0006E74696E672E2E2E0000000000000000AD
:10D9D00000CAF32E2E2E0000000000000000000000
:10D9E0000000000000496D7072657373696F6E2EE0
:10D9F0002E2E00000000000000447275636B656EFF
:10DA00002E2E2E00000000000000000000496D7066
:10DA1000726573696F6E2E2E2E00000000000000EC
:10DA2000005374616D70612E2E2E00000000000006
:10DA300000000000005072696E74696E672E2E2E11
:10DA4000000000000000000000496D7072657373F3
:10DA5000616F2E2E2E00000000000000006865742B
:10DA6000206472756B6B656E202E2E2E00000000F8
:10DA7000004261736B692E2E2E0000000000000032
:10DA80000000000000EB9E20E42E2E2E000000007F
:10DA9000000000000000000000D09FD0B5D187D06A
:10DAA000B0D182D18C2E2E2E000000000050726961
:10DAB0006E742070617573656400000000000000E2
:10DAC0000000000000000000000000CAF3F1F200B6
:10DAD0000000000000000000000000000000000046
:10DAE000000000000000000000496D7072696D6563
:10DAF00072206D697320656E20706175736500001A
:10DB000000000000000000447275636B20706175B6
:10DB100073696572740000000000000000000000DE
:10DB2000000000000050617573617220696D7072B1
:10DB30006573696F6E0000000000000000000000C7
:10DB40000000005374616D706120736F73706573B2
:10DB50006100000000000000000000000000000064
:10DB6000005072696E742070617573656400000006
:10DB7000000000000000000000000000000000495C
:10DB80006D7072696D6972207061757361646F0088
:10DB9000000000000000000000000000005072695A
:10DBA0006E74206F6E64657262726F6B656E0000DA
:10DBB00000000000000000000000004261736B697B
:10DBC00020647572616B6C6174696C64690000003B
:10DBD000000000000000000000EB9E20D7BDE0E642
:10DBE0000000000000000000000000000000000035
:10DBF00000000000000000D09FD0B5D187D0B0D188
:10DC000082D18C20D0BDD0B020D0BFD0B0D183D0B5
:10DC1000B7D0B50000CAF3F2F600473238205230D0
:10DC20002058205900506F776572204C6F73732015
:10DC30005265636F76657279000000000000000095
:10DC4000000000E7E8CAF300000000000000000048
:10DC500000000000000000000000000000000000C4
:10DC60000052656375702E20646573207065727450
:10DC70006573000000000000000000000000005775
:10DC800069656465726865727374656C6C756E67DE
:10DC9000000000000000000000000000005265636A
:10DCA000757065726163696F6E20656E6572676914
:10DCB0006100000000000000000000526563757004
:10DCC00065726F000000000000000000000000000E
:10DCD000000000000000000000506F776572204CCB
:10DCE0006F7373205265636F766572790000000070
:10DCF000000000000000005265746F6D61722061C9
:10DD000020726563757065726163616F0000000069
:10DD100000000000004865727374656C20737472B3
:10DD20006F6F6D7665726C696573000000000000AE
:10DD3000000000477563204B617962C4B1204B75C8
:10DD4000727461726D61000000000000000000004C
:10DD500000B0D00000000000000000000000000043
:10DD6000000000000000000000000000000000D0E3
:10DD7000B2D0BED181D181D182D0B0D0BDD0BED001
:10DD8000B2D0BBD0B5D0BDD0B8D0B500004D313287
:10DD900035004D3234002F2F616374696F6E3A7015
:10DDA000617573650A002F2F616374696F6E3A7233
:10DDB0006573756D650A004D313034205430205341
:10DDC0003231300D0A4D373032205430004D313071
:10DDD0003420543020533231300D0A4D3730312049
:10DDE00054300054657374696E67204D656E75001C
:10DDF0004E6F2053442063617264000000000000F5
:10DE0000000000000000F9A8000000000000000071
:10DE10000000000000000000000000004175637574
:10DE20006E65206361727465205344000000000039
:10DE300000004B65696E652053442D4B617274651B
:10DE400000000000000000004E6F2068617920741F
:10DE500061726A65746120534400000000005344FD
:10DE6000206E6F6E2070726573656E7465000000C1
:10DE7000000000005344B6B0C4DEB6DEB1D8CFBE59
:10DE8000DD00000000000000000053656D206361AC
:10DE90007274616F20534400000000000000000015
:10DEA0004765656E205344206B6161727400000009
:10DEB0000000000000005344204B61727420596F31
:10DEC0006B00000000000000000000005344ED99CA
:10DED0008320C5BC91922E000000000000000000CD
:10DEE0000000D09DD0B5D18220534420D0BAD0B00C
:10DEF000D180D182D18B000053746F702070726911
:10DF00006E7400000000000000000000000000002F
:10DF10000000000000000000000000F2F6CAF3005C
:10DF200000000000000000000000000000000000F1
:10DF3000000000000000000000000000000041722E
:10DF400072657420696D7072657373696F6E00001D
:10DF500000000000000000000000000000000000C1
:10DF60000053442D447275636B2041626272756385
:10DF70006800000000000000000000000000000039
:10DF800000000000446574656E657220696D7072F2
:10DF90006573696F6E000000000000000000000063
:10DFA000000000000000004172726573746120730C
:10DFB00074616D706100000000000000000000004E
:10DFC00000000000000000000000CCDFD8DDC4C36A
:10DFD000B2BC0000000000000000000000000000D3
:10DFE000000000000000000000000000005061720E
:10DFF000617220696D7072657373616F000000005B
:10E000000000000000000000000000000000000010
:10E010005072696E742073746F7070656E000000CA
:10E0200000000000000000000000000000000000F0
:10E03000000000447572647572000000000000006A
:10E0400000000000000000000000000000000000D0
:10E05000000000000000EB9E20E4E600000000004D
:10E0600000000000000000000000000000000000B0
:10E07000000000000000000000D09ED181D182D0BD
:10E08000B0D0BDD0BED0B2D0B8D182D18C20D0BF5C
:10E09000D0B5D187D0B0D182D18C00004D31303491
:10E0A00020543020533231300D0A4D373032205455
:10E0B00030004D31303420543020533231300D0A8D
:10E0C0004D37303120543000526573756D652070C6
:10E0D00072696E7400000000000000000000000083
:10E0E0000000000000000000000000F4F5CAF3008A
:10E0F0000000000000000000000000000000000020
:10E100000000000000000000000000000000526558
:10E110007072656E64726520696D70726573736983
:10E120006F6E000000000000000000000000000012
:10E130000053442D447275636B20466F727473658F
:10E14000747A756E67000000000000000000000097
:10E15000000000005265746F6D617220696D70720D
:10E160006573696F6E000000000000000000000091
:10E170000000000000000052697072656E64692042
:10E180007374616D70610000000000000000000009
:10E1900000000000000000000000CCDFD8DDC4BBA0
:10E1A000B2B6B20000000000000000000000000055
:10E1B0000000000000000000000000000052657434
:10E1C0006F6D617220696D7072657373616F0000AD
:10E1D000000000000000000000000000000000003F
:10E1E0005072696E742068657276617474656E0031
:10E1F000000000000000000000000000000000001F
:10E200000000005375726475720000000000000089
:10E2100000000000000000000000000000000000FE
:10E22000000000000000EB9E20DD840000000000E4
:10E2300000000000000000000000000000000000DE
:10E24000000000000000000000D09FD180D0BED0B0
:10E25000B4D0BED0BBD0B6D0B8D182D18C20D0BF84
:10E26000D0B5D187D0B0D182D18C00005061757308
:10E2700065207072696E74000000000000000000EC
:10E280000000000000F1F2CAF300000000000000EE
:10E2900000000000000000000000000000005061CD
:10E2A00075736520696D7072657373696F6E0000B8
:10E2B0000000000000000053442D447275636B2081
:10E2C0005061757365000000000000000000000050
:10E2D00050617573617220696D70726573696F6EDC
:10E2E0000000000000000000005061757361000034
:10E2F000000000000000000000000000000000001E
:10E300000000B2C1BCDEC3B2BC00000000000000CF
:10E310000000000000000000000000506175736103
:10E320007220696D7072657373616F000000000088
:10E33000000000005072696E74207061757A657219
:10E34000656E0000000000000000000000447572CF
:10E35000616B6C61740000000000000000000000B0
:10E36000000000000000EB9E20D7BDE4E6000000A6
:10E37000000000000000000000000000000000D0CD
:10E380009FD0B0D183D0B7D0B020D0BFD0B5D18787
:10E39000D0B0D182D0B8000054756E650000000086
:10E3A000000000000000000000000000CFF00000AE
:10E3B000000000000000000000000000000000005D
:10E3C0005265676C657200000000000000000000EC
:10E3D000000000004A757374696572756E6700000D
:10E3E0000000000000000000416A75737461720053
:10E3F0000000000000000000000000005265676F90
:10E400006C6100000000000000000000000000003F
:10E41000C1AEB3BEB200000000000000000000006A
:10E42000000000004166696E61720000000000009B
:10E43000000000000000000041667374656C6C65AC
:10E440006E000000000000000000000041796172D1
:10E4500000000000000000000000000000000000BC
:10E46000E2E00000000000000000000000000000EA
:10E4700000000000D09DD0B0D181D182D180D0BE2B
:10E48000D0B8D182D18C0000496E666F2073637260
:10E4900065656E0000000000000000000000000044
:10E4A000000000000000000000000000000000006C
:10E4B00000ECEDEEEF0000000000000000000000A6
:10E4C000000000000000000000000000000000004C
:10E4D00000000000000000000000456372616E2033
:10E4E000696E666F7300000000000000000000000D
:10E4F000000000000000000000000000000000001C
:10E50000000000496E666F0000000000000000007F
:10E5100000000000000000000000000000000000FB
:10E5200000000000000000000000000050616E7458
:10E53000616C6C6120696E666F726D6163696F6E8C
:10E5400000000000000000000000000000000000CB
:10E550000000000000477561726461000000000067
:10E5600000000000000000000000000000000000AB
:10E570000000000000000000000000000000BCDE01
:10E58000AEB3CEB3B6DED2DD000000000000000066
:10E59000000000000000000000000000000000007B
:10E5A000000000000000004D6F6E69746F72697AA0
:10E5B0006172000000000000000000000000000088
:10E5C000000000000000000000000000000000004B
:10E5D000496E666F2073636865726D00000000000D
:10E5E000000000000000000000000000000000002B
:10E5F00000000000000000000042696C67692045CF
:10E600006B72616E690000000000000000000000F5
:10E6100000000000000000000000000000000000FA
:10E620000000B4EE20E0AF00000000000000000099
:10E6300000000000000000000000000000000000DA
:10E640000000000000000000000000D098D0BDD104
:10E6500084D0BED180D0BCD0B0D186D0B8D0BED00E
:10E66000BDD0BDD18BD0B920D18DD0BAD180D0B0A2
:10E67000D0BD00006E6F5F66696C6500534420700A
:10E6800072696E74696E6720627974653A004E6FC4
:10E6900074205344207072696E74696E670A005466
:10E6A0005249474745524544006F70656E003A2015
:10E6B000007A5F6D6178007A5F6D696E00795F6DD9
:10E6C000696E00785F6D6178005265706F72746971
:10E6D0006E6720656E6473746F70207374617475F7
:10E6E000730A002569730025696D2025697300256B
:10E6F00069682025696D20256973002569642025D6
:10E7000069682025696D20256973002569792025B0
:10E710006964202569682025696D20256973004694
:10E72000696C652064656C657465643A0044656C69
:10E730006574696F6E206661696C65642C2046693A
:10E740006C653A200057726974696E6720746F2097
:10E7500066696C653A20006F70656E206661696C51
:10E7600065642C2046696C653A20006F70656E20E8
:10E770006661696C65642C2046696C653A200046C8
:10E78000696C652073656C65637465640A00205369
:10E79000697A653A200046696C65206F70656E6520
:10E7A000643A20002066696C653A2000646F696EE7
:10E7B00067006672657368004E6F772000454E44AF
:10E7C00020535542524F5554494E450A002220705D
:10E7D0006F73002220706172656E743A2200535587
:10E7E00042524F5554494E452043414C4C20746190
:10E7F000726765743A22004B494C4C45442E200008
:10E80000747279696E6720746F2063616C6C207319
:10E8100075622D67636F64652066696C6573207728
:10E8200069746820746F6F206D616E79206C6576F5
:10E83000656C732E204D4158206C6576656C20699F
:10E84000733A004572726F723A006F70656E20669F
:10E8500061696C65642C2046696C653A20004361EF
:10E860006E6E6F74206F70656E207375626469726E
:10E8700020006563686F3A0046696C616D656E746F
:10E8800020757365643A200053746174733A2000F4
:10E890002C204C6F6E67657374206A6F623A20009B
:10E8A000546F74616C2074696D653A200053746113
:10E8B00074733A20002C204661696C65643A20002C
:10E8C0002C2046696E69736865643A20005072694D
:10E8D0006E74733A200053746174733A20002057A9
:10E8E0003A00436F6F6C696E672E2E2E0000000099
:10E8F000000000000000000000000000436F6F6C8B
:10E90000696E672E2E2E000000000000000000003F
:10E91000000000000000436F6F6C696E672E2E2EA2
:10E9200000000000000000000000000000000000E7
:10E93000436F6F6C696E672E2E2E00000000000082
:10E9400000000000000000000000436F6F6C696E63
:10E95000672E2E2E000000000000000000000000C6
:10E9600000000000436F6F6C696E672E2E2E000052
:10E970000000000000000000000000000000436FE5
:10E980006F6C696E672E2E2E0000000000000000E4
:10E990000000000000000000436F6F6C696E672E7E
:10E9A0002E2E00000000000000000000000000000B
:10E9B0000000436F6F6C696E672E2E2E0000000002
:10E9C000000000000000000000000000436F6F6CBA
:10E9D000696E672E2E2E000000000000000000006F
:10E9E000000000000000436F6F6C696E672E2E2ED2
:10E9F0000000000000000000000000000000000017
:10EA0000436F6F6C696E672E2E2E000000000000B1
:10EA10000000000000000000000048656174696E9D
:10EA2000672E2E2E00000000000000000000486548
:10EA30006174696E672E2E2E000000000000000039
:10EA4000000048656174696E672E2E2E000000007C
:10EA500000000000000048656174696E672E2E2E6C
:10EA60000000000000000000000048656174696E4D
:10EA7000672E2E2E000000000000000000004865F8
:10EA80006174696E672E2E2E0000000000000000E9
:10EA9000000048656174696E672E2E2E000000002C
:10EAA00000000000000048656174696E672E2E2E1C
:10EAB0000000000000000000000048656174696EFD
:10EAC000672E2E2E000000000000000000004865A8
:10EAD0006174696E672E2E2E000000000000000099
:10EAE000000048656174696E672E2E2E00000000DC
:10EAF00000000000000048656174696E672E2E2ECC
:10EB000000000000000000000000020029010B01CD
:10EB100011241FBECFEFD1E2DEBFCDBF00E00CBF9E
:10EB200013E0A0E0B2E0EEE8F3E003E00BBF02C0C8
:10EB300007900D92AC39B107D9F72BE1ACE9B3E0FE
:10EB400001C01D92AF3EB207E1F715E7C7E8D5E770
:10EB500000E006C021970109802FFE010F94058176
:10EB6000C638D10780E00807A9F70F945A6A0D94B8
:10EB7000B6810C9400002F923F924F925F926F9259
:10EB80007F928F929F92AF92BF92CF92DF92EF923D
:10EB9000FF920F931F93CF93DF93CDB7DEB7A99763
:10EBA0000FB6F894DEBF0FBECDBF21E02093FF0467
:10EBB0008091E71B8D3409F465C224F4873471F029
:10EBC0000C941C88843511F40C948487873511F0DB
:10EBD0000C941C880F9418350C941E8880914F114A
:10EBE000909150118C31910509F4A6C05CF48430E9
:10EBF0009105B9F11CF4029768F140C24B9709F4F2
:10EC00006FC03CC28A35910509F4C4C144F48D310A
:10EC1000910509F4E5C04E9709F4E6C02FC28B3583
:10EC2000910509F4BBC18C35910509F027C27AEE34
:10EC3000272E72E0372EE7EEEE2EE4E0FE2E2FECCC
:10EC400039E039A728A7FAE7CF2EFAE0DF2E00E057
:10EC500010E0E4C18091300281110C9423880C945F
:10EC60001E8880E50F944754882329F00F948B5316
:10EC70006B017C0103C0C12CD12C760183E50F947C
:10EC80004754882361F00F94CB5320E030E04AE7EB
:10EC900054E40F940A780F94577F6B017C010F9412
:10ECA00073008091A90A811105C060E082E494E0BC
:10ECB0000E94BFC20F94AC45C60ED71EE81EF91EB7
:10ECC0000F94AC45DC01CB018C199D09AE09BF093D
:10ECD000B7FD02C00C941E8880E00E9434D4F0CFAF
:10ECE0000E94D7ED81110C941E8880E090E0A4EB87
:10ECF000B2E489839A83AB83BC8380E090E0A6EE84
:10ED0000B2E48D839E83AF83B88719861A861B86EB
:10ED10001C8680E50F944754882319F00F949B5369
:10ED200001C060E068A3BE016F5F7F4FCE01809697
:10ED30000F94575F0C941E888091860A85FF12C03D
:10ED4000EDEAF4E0F4908F010F5F1F4FFF2041F0D8
:10ED50008F2D0F94F45F8F2D0F94ED5FF801F2CF9C
:10ED60000E94FAA98091740A8770873011F00C9480
:10ED700028888FE40F944754882379F00F94BC536C
:10ED8000882311F40C9428888091860A85FD02C09E
:10ED90000C941E88E2E9F4E00BC08FE40F94FE535C
:10EDA000EFCF8F2D0F94F45F8F2D0F94ED5FF8014F
:10EDB000F4908F010F5F1F4FF110F3CFE9E8F4E0FB
:10EDC000F4908F010F5F1F4FFF2011F40C941E88E9
:10EDD0008F2D0F94F45F8F2D0F94ED5FF801F0CF1E
:10EDE0000E94B0AB0C941E88C090CF09D090D0097F
:10EDF000E090D109F090D20988E50F944754811131
:10EE000008C020E030E0A901C701B6010F94707E70
:10EE100002C00F94CB5368A379A38AA39BA3C0908D
:10EE2000D309D090D409E090D509F090D60989E5AE
:10EE30000F944754811108C020E030E0A901C701B8
:10EE4000B6010F94707E02C00F94CB539B01AC01AE
:10EE500069837A838B839C8368A179A18AA19BA112
:10EE60000E9447D3882311F40C941E8880E00E94EE
:10EE7000439D0E94E09685E40F944754882321F037
:10EE80000F94BC53182F04C085E40F94FE5311E077
:10EE900086E50F944754882321F00F949B53262F27
:10EEA00001C021E0412FBE016F5F7F4FCE018096F0
:10EEB0000E9482EE6B017C019B01AC010F948C805F
:10EEC000811162C088A099A0AAA0BBA020E030E078
:10EED000A901C501B4010F94A57787FF05C027E1FB
:10EEE00037EB41E558EB04C027E137EB41E558E348
:10EEF000C501B4010F94707EAB01BC0180EC94E0BD
:10EF00000F946E2D89809A80AB80BC8020E030E029
:10EF1000A901C501B4010F94A57787FF05C027E1BA
:10EF200037EB41E558EB04C027E137EB41E558E307
:10EF3000C501B4010F94707EAB01BC018BEB94E072
:10EF40000F946E2D20E030E0A901C701B6010F94A7
:10EF5000A57787FF05C027E137EB41E558EB04C0F3
:10EF600027E137EB41E558E3C701B6010F94707E06
:10EF7000AB01BC0186EB94E00F946E2D8AE00F94F8
:10EF8000F45F8AE00F94ED5F0E94BD960F94DB0959
:10EF90000C941E881092B1030C941E882093B10328
:10EFA0000C941E880F94CB532B013C01133049F075
:10EFB000F60120813181428153810F946F7E2B01B4
:10EFC0003C01E8A5F9A52081318142815381C3012B
:10EFD000B2010F946F7E4B015C012DEB37E346E8E5
:10EFE00055EB0F940F8087FD21C02DEB37E346E8EA
:10EFF00055E3C501B4010F94A5771816BCF01F5F47
:10F00000F4E0EF0EF11C28A539A52C5F3F4F39A77E
:10F0100028A734E0C30ED11C143031F1F1018191E5
:10F020001F010F944754882351F3BCCF133051F480
:10F030004092DB095092DC096092DD097092DE0992
:10F0400001E0DDCFA5019401F7016081718182812A
:10F0500093810F94707EF701608371838283938321
:10F06000812F0E940997CBCF002321F08BED99E0EF
:10F070000E948DED0F94DB090C941E880E942EF2E5
:10F080000C941E8880914F119091501185379105F5
:10F0900009F49EC70CF0DBC08B34910509F44AC417
:10F0A0000CF057C08931910509F436C31CF5843141
:10F0B000910509F4DEC17CF48131910509F454C253
:10F0C0002CF4029708F4D8C10C948187429709F474
:10F0D0004FC60C9481878631910509F491C20CF4D6
:10F0E0008BC28731910509F491C2489709F4A6C2F1
:10F0F0000C9481878E31910509F454C384F48B31CB
:10F10000910509F428C30CF418C38C31910509F456
:10F110003FC34D9711F40C941E880C948187813263
:10F12000910509F491C34CF48F31910509F49DC305
:10F13000809709F447C30C9481878A32910509F4BA
:10F14000C5C3C09711F00C9481870E94F2DB0C9428
:10F150001E888936910509F406C50CF042C0823537
:10F16000910509F4FCC524F58D34910509F4EAC331
:10F170000CF4E4C38E34910509F4E8C3813591059C
:10F1800011F00C9481870F9403250F94B80010920E
:10F19000600610925F0668EE73E080E090E00F94E6
:10F1A000CC3A60E08DE595E00E94BFC20C941E88C9
:10F1B0008535910509F411C654F48335910509F498
:10F1C000D2C58435910509F4D3C50C9481878C355B
:10F1D000910509F41DC68836910509F4BBC30C944A
:10F1E00081878E36910509F4E6C39CF48B36910530
:10F1F00009F420C50CF400C58C36910509F477C4D8
:10F200008D36910511F00C9481870F943B620C941C
:10F210001E888137910509F472C46CF48F3691050C
:10F2200009F4DCC38037910511F00C9481878AE4DE
:10F2300095E00E94C9D38237910509F472C68337DD
:10F24000910511F00C948187EEE6F5E0B1C68E329F
:10F25000E1E09E0711F40C943B840CF077C08B3CEA
:10F26000910511F40C947F81ACF58D37910509F46B
:10F27000F3C4ACF48737910509F469C70CF40DC7E2
:10F280008837910509F466C78937910511F00C9408
:10F29000818710923205109231050C941E888B39AB
:10F2A000910509F482C434F48139910509F458C7F1
:10F2B0000C948187883C910509F4B8C7893C910575
:10F2C00011F00C9481878AEEE82E82E0F82E02EC91
:10F2D00014E0FCC78C3D910511F40C94A282B4F4A7
:10F2E0008D3C910511F40C94128214F40C949A81C3
:10F2F0008E3C910511F40C947D82833D910511F0B3
:10F300000C9481870F94E4080C941E88823221E0CB
:10F31000920711F40C94588364F48D3D910511F417
:10F320000C94AF82823E910511F40C942F830C94BF
:10F3300081878C32E1E09E0711F40C9463838D3257
:10F34000914011F40C948C830C948187863F21E0CA
:10F35000920711F40C9459850CF04AC08239E1E00F
:10F360009E0711F40C94B8840CF5833621E09207C3
:10F3700009F47BC04CF48F32914011F00C948187DA
:10F380000F9478040C941E888039F1E09F0711F4E3
:10F390000C94B5848139914011F00C94818781E0FF
:10F3A0000E9429A00F94DB090C941E888C3A31E04E
:10F3B000930711F40C949F8264F48A39F1E09F075B
:10F3C00009F499C3843A914011F40C94BE840C94CE
:10F3D0008187843F31E0930711F40C945785853F72
:10F3E000914011F00C9481870F94EA410C941E888F
:10F3F0008D3BF2E09F0711F40C942086B4F4883F13
:10F4000031E0930711F40C94688514F40C945C8536
:10F410008835F2E09F0711F40C9494858B35924067
:10F4200011F40C9497850C9481878B3833E0930703
:10F4300011F40C941E886CF48E3BF2E09F0711F4DB
:10F440000C9423868335934011F40C94EC860C9431
:10F450008187803A33E0930709F4FAC1873E9340ED
:10F4600011F40C9464870C948187E3E4F8EE0C9417
:10F470009E84E1EFF4E087C0A0904D11B0904E1152
:10F4800080E50F944754882359F00F948B536B01F8
:10F490007C0111E0672B682B692B31F410E004C06C
:10F4A00010E0C12CD12C760183E50F9447548823BA
:10F4B00011F40C94E1880F94CB5320E030E04AE73C
:10F4C00054E40F940A780F94577F6B017C0111115B
:10F4D0000BC0672B682B692B39F4A114B10421F000
:10F4E000F5018081811102C010E001C011E00F948C
:10F4F0007300112329F061E0C5010E94FBC205C021
:10F5000060E088EC94E00E94BFC283E08093FF0437
:10F5100081E080939904C114D104E104F104B1F0B5
:10F520000F94AC45C60ED71EE81EF91E0F94AC45CD
:10F53000DC01CB018C199D09AE09BF09B7FF0EC0D4
:10F540008091990481110C94E68808C080919904F7
:10F55000882321F080E00E9434D4F8CF0F94ED4747
:10F56000109299040C941E8860E089ED94E00E944A
:10F57000BFC212988A988091080181708093060119
:10F580005F980C941E88F4908F010F5F1F4FFF202F
:10F5900041F08F2D0F94F45F8F2D0F94ED5FF801E4
:10F5A000F2CF1092831382E592E10E943F966EE4BF
:10F5B00072E1CE0101960F94084F40E050E0BE0189
:10F5C0006F5F7F4F80E090E00F949756CE010196D9
:10F5D0000E944A96E2EEF4E0F4908F010F5F1F4F15
:10F5E000FF2011F40C941E888F2D0F94F45F8F2D43
:10F5F0000F94ED5FF801F0CF0E94F5EA0C941E889D
:10F6000010922212109223120C941E880E9464ED14
:10F61000E0914D11F0914E118081882329F08032C4
:10F6200009F410823196F8CF40E061E080914D11ED
:10F6300090914E110F942F590C941E8880E090E009
:10F64000A8E4B2E489839A83AB83BC8318A219A28D
:10F650001AA21BA21CA21DA21EA21FA28091081901
:10F66000882361F000E020E0AE014F5F5F4FBE01F4
:10F67000605E7F4FCE0184960F94616183E50F94A5
:10F680004754882381F00F949B53AB01BC014093F6
:10F690007F1350938013609381137093821381E1E1
:10F6A00093E10F94393080912312882319F081E07F
:10F6B0008093221284E50F9447548823B1F00F946D
:10F6C0009B536B017C010F94830FC092240BD0924B
:10F6D000250BE092260BF092270BCD28CE28CF28C1
:10F6E00031F081E08093741102C00E944FCD81E01F
:10F6F00080936B0AE2E0F5E0F4908F010F5F1F4FFB
:10F70000FF2011F40C941E888F2D0F94F45F8F2D21
:10F710000F94ED5FF801F0CF109222120F949E0F1C
:10F7200082E195E09093D60A8093D50A0E943B9897
:10F7300082E080936B0A0C941E88809123128823A8
:10F7400011F40C941E8883E50F94475481110C9496
:10F75000EB880C941E8883E40F94FE538823A1F059
:10F76000E7E1F5E0F4908F010F5F1F4FFF2041F0BC
:10F770008F2D0F94F45F8F2D0F94ED5FF801F2CF72
:10F780000F94F94C0C941E880F94A54C0C941E8871
:10F7900040E060E080914D1190914E110F942F59EF
:10F7A0000C941E8880912312882311F40C941E88D7
:10F7B0000F94575680914D1190914E110F94C85A45
:10F7C0000C941E888091221281110F9473008091F5
:10F7D0002312882311F40C941E8880E50F9447545B
:10F7E000882319F00F94BC5303C080E50F94FE5397
:10F7F000182F482F61E080914D1190914E110F9478
:10F800002F5983E50F944754882381F00F949B531D
:10F81000AB01BC0140937F1350938013609381131D
:10F820007093821381E193E10F9439308091231218
:10F83000882319F081E08093221211110C941E8804
:10F840000E944FCD0C941E880E942BE30C941E88BE
:10F8500080914D1190914E1121E02093211240E0B2
:10F8600060E00F942F590C941E880F944F0F68A3DB
:10F8700079A38AA39BA3BE016F5F7F4FCE018096C1
:10F880000F94535460E0CE0101960E94FBC2E2E760
:10F89000F8EEF4908F010F5F1F4FFF2041F08F2D86
:10F8A0000F94F45F8F2D0F94ED5FF801F2CFBE013E
:10F8B0006F5F7F4F86E295E00F94EF2D8AE00F9403
:10F8C000F45F8AE00F94ED5F0C941E8883E50F943B
:10F8D0004754882311F40C941E880F94AB53E82EE0
:10F8E00080E50F944754882339F00F94AB53182FB9
:10F8F00087FF03C00C941E881DE089E40F944754D1
:10F90000882341F00F94BC5381110C94D989E9E10B
:10F91000F6E00BC089E40F94FE53F6CF319626E053
:10F92000E634F20711F40C94D98984911813F6CFB8
:10F930000C9455890E944FCD0C941E880F949E0FF5
:10F940000C941E880E9496CD0C941E880F942064FF
:10F950000C941E8888E690E00E949D9781110C947B
:10F960001E888091860A83FF02C00C941E8883E55E
:10F970000F944754882311F40C941E880F94CB5392
:10F980000F94527F70937B0460937A0480E00F940D
:10F99000B7240F94CB5320E030E04AEA52E40F94AE
:10F9A000A577181614F40C941E880E9496CD0F9417
:10F9B000ED470C941E888EE40F944754882311F46D
:10F9C0000C941E880F949B536093CB097093CC09C1
:10F9D0008093CD099093CE090C941E8883E50F94F3
:10F9E000FE53882359F083E50F944754882319F078
:10F9F0000F94AB5301C080E08093860AE2E7F8EEF3
:10FA0000F4908F010F5F1F4FF11003C0E3E4F5E0A6
:10FA100008C08F2D0F94F45F8F2D0F94ED5FF801C8
:10FA2000EFCFF4908F010F5F1F4FFF2041F08F2D1C
:10FA30000F94F45F8F2D0F94ED5FF801F2CF80915A
:10FA4000860A811103C0EFE3F5E03BC063E3C62EF5
:10FA500065E0D62EE12CF12C20E08091860A90E022
:10FA60000E2C02C0959587950A94E2F780FF1EC080
:10FA7000AA24A394A20E222331F08CE20F94F45F07
:10FA80008CE20F94ED5FF60185919491FC01B490A6
:10FA90008F010F5F1F4FBB2041F08B2D0F94F45F40
:10FAA0008B2D0F94ED5FF801F2CF2A2D3FEFE31A73
:10FAB000F30A82E0C80ED11C96E0E916F10469F65B
:10FAC0000EC0F4908F010F5F1F4FFF2041F08F2D6C
:10FAD0000F94F45F8F2D0F94ED5FF801F2CF8AE061
:10FAE0000F94F45F8AE00F94ED5F0C941E881092DF
:10FAF0001B020C941E880F9443040C941E8883E50B
:10FB00000F944754811103C0E2E7F8EE0DC00F9443
:10FB1000AB538D3320F480930A020C941E888CE33F
:10FB200080930A020C941E88F4908F010F5F1F4F80
:10FB3000FF2041F08F2D0F94F45F8F2D0F94ED5F18
:10FB4000F801F2CF40910A0250E060E070E083E5F6
:10FB500095E00F944B2D8AE00F94F45F8AE00F94A8
:10FB6000ED5F0C941E8889E690E00E949D978111BC
:10FB700018C0EAE5F5E0F4908F010F5F1F4FFF20FA
:10FB800041F08F2D0F94F45F8F2D0F94ED5FF801EE
:10FB9000F2CF0F94D0228AE00F94F45F8AE00F94A2
:10FBA000ED5F1092FF040C94F88983E50F9447549D
:10FBB000882311F40C941E880F94AB53182F8D33A7
:10FBC00008F01CE3109334050F94AC456B017C01E5
:10FBD000212F30E0A8EEB3E00F94607EC60ED71E52
:10FBE000E81EF91EC092E304D092E404E092E5041A
:10FBF000F092E6040C941E8880E50F94475481111E
:10FC000006C083E50F944754882361F006C00F9423
:10FC1000AB5381110C941E88F4CF0F949B536F3F0C
:10FC2000710510F06FEF70E07093600660935F06EF
:10FC30000C941E8880E50F944754811106C01092E1
:10FC4000600610925F060C941E880F949B53672BDE
:10FC500011F00C941E88F3CF8CE40F94FE5388238C
:10FC600081F00F94CB536B017C0120E030E0A901BF
:10FC70000F940F8087FF0AC0F7FAF094F7F8F0941A
:10FC800005C0C12CD12CE12C50E4F52EF7FAF094EC
:10FC9000F7F8F094CCA2DDA2EEA2FFA280E090E003
:10FCA000A4EBB2E489839A83AB83BC8380E090E0C9
:10FCB000A6EEB2E48D839E83AF83B88719861A8639
:10FCC0001B861C8688E50F944754882379F088E5C5
:10FCD0000F944754882319F00F94CB5303C060E06E
:10FCE00070E0CB0169837A838B839C8389E50F94D1
:10FCF0004754882379F089E50F944754882319F0F5
:10FD00000F94CB5303C060E070E0CB016D837E8322
:10FD10008F8398878AE50F944754882379F08AE582
:10FD20000F944754882319F00F94CB5303C060E01D
:10FD300070E0CB0169877A878B879C8718A219A20C
:10FD40001AA21BA220E0AE01405E5F4FBE016F5FB2
:10FD50007F4FCE0184960E944EE20C941E88109232
:10FD6000B0030C941E8881E08093B0030C941E882D
:10FD700083E50F9447548823A1F00F94CB5320E0E0
:10FD800030E04AE754E40F940A780F94577F609369
:10FD90000B0270930C0280930D0290930E020C9450
:10FDA0001E8888E50F94FE5381110C94FC8889E528
:10FDB0000F94FE5381110C94FC888AE50F94FE5336
:10FDC00081110C94FC8885E40F94FE5381110C94EE
:10FDD000FC880F94B8000C941E8883E50F94FE53A2
:10FDE000882311F40C941E880F94CB5320E030E04C
:10FDF0004AE754E40F940A780F94577F6093DF0426
:10FE00007093E0048093E1049093E2040C941E88C4
:10FE10003AEEC32E32E0D32E48E9E42E4AE0F42E27
:10FE200010E0F60181916F010F94FE53882309F4CD
:10FE30006DC0133009F063C00F94CB534B015C01CC
:10FE400020E030E040EA51E40F94A57787FF4EC0F0
:10FE5000A50194016091A40A7091A50A8091A60A57
:10FE60009091A70A0F94EA7E2B013C019B01AC0103
:10FE70006091E30A7091E40A8091E50A9091E60AA4
:10FE80000F940A786093E30A7093E40A8093E50A7A
:10FE90009093E60AA30192016091FF0A7091000B12
:10FEA0008091010B9091020B0F940A786093FF0AE6
:10FEB0007093000B8093010B9093020B6091BE0432
:10FEC0007091BF048091C0049091C1040F94A977F0
:10FED000A30192010F940A780F94577F6093BE0498
:10FEE0007093BF048093C0049093C1048092A40ACD
:10FEF0009092A50AA092A60AB092A70A07C00F94F2
:10FF0000CB53F70160837183828393831F5FF4E097
:10FF1000EF0EF11C143009F084CF0E941FD00C9416
:10FF20001E880F94730083E50F944754882309F4C7
:10FF3000A1C80F949B536230710509F09BC80E94C1
:10FF400093DA8BE50F94F45F8BE50F94ED5F60918E
:10FF5000F3047091F4048091F5049091F60442E06A
:10FF60000F9487604091F7045091F8046091F90470
:10FF70007091FA048BE695E00F946E2D4091FB048E
:10FF80005091FC046091FD047091FE0488E695E0B8
:10FF90000F946E2D8DE50F94F45F8DE50F94ED5F5A
:10FFA0008AE00F94F45F8AE00F94ED5F0C941E8852
:10FFB000F4908F010F5F1F4FFF2011F40C941E88E7
:10FFC0008F2D0F94F45F8F2D0F94ED5FF801F0CF1C
:10FFD00000914D1110914E11F8018081882309F490
:10FFE00059C001900020E9F731977F01E01AF10A2A
:10FFF000F9E0EF16F1040CF448C05801AE0CBF1C38
:020000021000EC
:10000000680167E273E0C6010F949C81801B910B2D
:100010002FEFC21AD20A18161906ACF58E159F05D5
:10002000A4F5CA14DB0439F0F801E80FF91F319781
:100030002081203231F7AC01475F5F4FB801640F78
:10004000751FFB014E155F0534F42191203219F024
:100050004F5F5F4FF7CF49305105B9F04950510913
:100060008A01081B190BA80182EB93E00F943281DF
:10007000F801EE54FC4F108282EB93E00F948676E9
:1000800080931F04DBC70097B1F260E0C8010E94B3
:10009000FBC2D4C70F94ED47D1C700914D11109109
:1000A0004E1183E0C12C40E08150E1F0F8019081D5
:1000B000292F2B7F2134C1F721812133A9F79134D6
:1000C00021F0953421F441E002C0CC24C39498017E
:1000D0002E5F3F4F89012F5F3F4FF8019081903293
:1000E000C9F3E2CF442389F0E2E7F8EED4907F0130
:1000F0002FEFE21AF20ADD2041F08D2D0F94F45F0C
:100100008D2D0F94ED5FF701F1CFCC2089F0E5ED57
:10011000F5E0D4907F013FEFE31AF30ADD2041F0D0
:100120008D2D0F94F45F8D2D0F94ED5FF701F1CFBE
:100130007801F8018081882309F4D1CC0F94F45F11
:100140000F5F1F4FF70180810F94ED5FF1CF0F9488
:10015000B95574C781E080933205809331056EC72D
:1001600083E50F944754882319F00F949B5302C0E2
:1001700060E070E08B0111270230110514F1E3E417
:10018000F8EEF4908F010F5F1F4FF11003C0E9EDFF
:10019000F5E008C08F2D0F94F45F8F2D0F94ED5F65
:1001A000F801EFCFF4908F010F5F1F4FFF2009F48C
:1001B00045C78F2D0F94F45F8F2D0F94ED5FF801DD
:1001C000F1CF88E40F9447548823A1F00F949B53F8
:1001D0006A3A710534F0623E71052CF061EE70E010
:1001E00002C06AEA70E0F801EE0FFF1FE056FC4F14
:1001F0007183608386E40F944754882309F41EC7F3
:100200000F949B53000F111FF801E456FC4F7183AC
:1002100060836F3F710519F014F06FEF70E077FFA6
:1002200002C060E070E07183608308C788EC90E0F2
:100230000E949D97811102C784E40F94FE53882386
:1002400009F441C00F94CB536B017C0111E020E015
:1002500030E0A9010F94A577811101C010E010933F
:100260000F1B20E030E0A901C701B6010F94A5776C
:10027000882349F10F94CB53E091D90B24E0E29FFE
:10028000F0011124E05FF44E6083718382839383D5
:1002900020E030E0A9016091101B7091111B80914A
:1002A000121B9091131B0F94A57781110CC080E055
:1002B00090E0A0EEBFE38093101B9093111BA093DE
:1002C000121BB093131B0F94025DB8C6F701819106
:1002D0007F010F94FE53882349F00F94CB530F9462
:1002E000577FF80160837183828393830C5F1F4F74
:1002F000F4E0023D1F0751F70E94EACE9FC60AEEC6
:10030000E02E02E0F02E03EF1AE0F70181917F0169
:100310000F94FE53882339F00F94CB53F801608378
:100320007183828393830C5F1F4FFBE003301F07B1
:1003300061F784C683E50F9447548823A1F00F9496
:10034000CB536093EB0A7093EC0A8093ED0A909381
:10035000EE0A6093E70A7093E80A8093E90A9093A3
:10036000EA0A10E001C011E080E50F9447548823A9
:1003700059F00F94CB536093EB0A7093EC0A80937F
:10038000ED0A9093EE0A10E082E50F94475488231B
:1003900059F00F94CB536093EF0A7093F00A809357
:1003A000F10A9093F20A10E084E50F9447548823F1
:1003B00059F00F94CB536093E70A7093E80A809347
:1003C000E90A9093EA0A3AC6112309F437C6409124
:1003D000EB0A5091EC0A6091ED0A7091EE0A81E00F
:1003E00096E00F946E2D4091EF0A5091F00A6091C3
:1003F000F10A7091F20A8EEF95E00F946E2D409104
:10040000E70A5091E80A6091E90A7091EA0A8BEFD5
:1004100095E00F946E2D8AE00F94F45F8AE00F94BC
:10042000ED5F0CC681E50F94FE53882351F00F94C5
:100430008B536093030B7093040B8093050B909385
:10044000060B83E50F94FE53882351F00F94CB5392
:1004500060930B0B70930C0B80930D0B90930E0B12
:1004600084E50F94FE53882351F00F94CB5360938F
:10047000070B7093080B8093090B90930A0B88E588
:100480000F94FE53882351F00F94CB536093D70AF7
:100490007093D80A8093D90A9093DA0A89E50F9469
:1004A000FE53882351F00F94CB536093DB0A709373
:1004B000DC0A8093DD0A9093DE0A8AE50F94FE53EE
:1004C000882351F00F94CB536093DF0A7093E00AB6
:1004D0008093E10A9093E20A85E40F94FE53882307
:1004E00009F4ACC50F94CB536093E30A7093E40A0C
:1004F0008093E50A9093E60AA1C5BAEECB2EB2E04E
:10050000DB2E1BE4E12E15E0F12E10E0F6018191C7
:100510006F010F94FE53882351F00F94CB53F701D2
:100520006083718382839383812F0E9409971F5F69
:10053000F4E0EF0EF11C133049F70C943A780F9465
:10054000B60A7CC583E50F944754882309F476C521
:100550000F949B5370933402609333026FC58DEDFB
:1005600090E00E949D97811169C583E50F944754DF
:10057000811103C0E2E7F8EE3AC00091D90B10E018
:100580000F949B53000F111FF801EF5CFD4F718317
:1005900060838091D90B90E08C01000F111F000F38
:1005A000111F98012B5F3D4F7901880F991FFC01A6
:1005B000EF5CFD4F60817181072E000C880B990B59
:1005C0000F94AB772AE037ED43E25CE30F940A78AF
:1005D000F801E454F44F20813181428153810F941A
:1005E0000A78F701608371838283938327C5F4902F
:1005F0008F010F5F1F4FFF2041F08F2D0F94F45F8D
:100600008F2D0F94ED5FF801F2CF85E40F94F45F26
:1006100085E40F94ED5F8091D90B805D0F94F45FBA
:100620008091D90B805D0F94ED5FE091D90BF0E0E4
:10063000EE0FFF1FEF5CFD4F6081718181E196E05D
:100640000F94B32D85E20F94F45F85E20F94ED5F74
:100650008AE00F94F45F8AE00F94ED5FEFC480E5C9
:100660000F94FE53882309F4E9C40F949B536B0144
:100670007C0183E50F944754882321F00F949B530A
:100680008B0102C00FEF1FEFC8010196039708F01E
:10069000D5C4D7FCD3C48C2DE9E1F6E09491891739
:1006A00009F403C6319626E0E634F207B9F7D4C55B
:1006B0008AE50F9447548111FBC583E50F94475495
:1006C0008111F6C5BBC483E50F944754882319F004
:1006D0000F949B5302C064E071E079A368A380E5A6
:1006E0000F944754882339F00F949B53693833E1B2
:1006F000730730F402C068EE73E07A83698304C044
:1007000088E893E19A838983BE01605E7F4FCE01C2
:1007100001960F94645692C485E40F944754811156
:1007200010C080E50F94FE53882391F00F94CB53B3
:100730006093340B7093350B8093360B9093370B8B
:1007400007C00F94AB53882361F3E3E4F8EE7CC059
:1007500089E40F94FE53882381F00F94CB532CEA45
:1007600035EC47E25EE30F940A786093300B7093A8
:10077000310B8093320B9093330B84E40F94FE5330
:10078000882381F00F94CB532CEA35EC47E25EE3EB
:100790000F94EA7E6093380B7093390B80933A0B79
:1007A00090933B0BE2E7F8EEF4908F010F5F1F4F41
:1007B000FF2041F08F2D0F94F45F8F2D0F94ED5F8C
:1007C000F801F2CF4091340B5091350B6091360B0C
:1007D0007091370B8FE596E00F946E2D2CEA35EC77
:1007E00047E25EE36091300B7091310B8091320BE8
:1007F0009091330B0F94EA7EAB01BC018BE596E040
:100800000F946E2D2CEA35EC47E25EE36091380BD5
:100810007091390B80913A0B90913B0B0F940A78B1
:10082000AB01BC0187E596E00F946E2D8AE00F9432
:10083000F45F8AE00F94ED5F01C48F2D0F94F45F95
:100840008F2D0F94ED5FF801F4908F010F5F1F4F14
:10085000F110F3CFE3E6F6E0F4908F010F5F1F4F46
:10086000FF2009F4EBC38F2D0F94F45F8F2D0F94AD
:10087000ED5FF801F1CF83E50F94FE53182F882325
:1008800071F00F94CB530F94527F709326026093B4
:10089000250221E0672B09F020E020930F0B80E573
:1008A0000F94FE53882359F020912502309126029F
:1008B000232B11F00F94BC5380930F0BBFC3111166
:1008C000BDC3E2E7F8EEF4908F010F5F1F4FFF20EA
:1008D00041F08F2D0F94F45F8F2D0F94ED5FF80191
:1008E000F2CF80910F0B882319F068E173E002C00A
:1008F0006BE173E08AE896E00F94EF2D609125029A
:100900007091260289E796E00F94B32DE5E7F6E0B3
:10091000F4908F010F5F1F4FFF2009F48FC38F2DBD
:100920000F94F45F8F2D0F94ED5FF801F1CF8F2DB1
:100930000F94F45F8F2D0F94ED5FF801F4908F0109
:100940000F5F1F4FF110F3CFEDE9F6E0F4908F0148
:100950000F5F1F4FFF2009F471C38F2D0F94F45FB9
:100960008F2D0F94ED5FF801F1CF0F94730066C3E4
:1009700080E00E9429A00F94DB0960C383E50F94F7
:10098000FE53882349F00F94BC53182F811106C0E1
:1009900080E00E94439D02C01091D2048091CF0953
:1009A0009091D009A091D109B091D20989839A83FD
:1009B000AB83BC838091D3099091D409A091D509D0
:1009C000B091D6098D839E83AF83B8878091D70974
:1009D0009091D809A091D909B091DA0989879A87AD
:1009E000AB87BC8786E50F94FE53882321F089ED01
:1009F00096E00E9456F1812F0E94439D111103C081
:100A0000E2E7F8EE25C08091D2048111F9CFE3E44A
:100A1000F8EEF4908F010F5F1F4FF11003C0EAEB67
:100A2000F6E008C08F2D0F94F45F8F2D0F94ED5FCB
:100A3000F801EFCFF4908F010F5F1F4FFF2001F3FC
:100A40008F2D0F94F45F8F2D0F94ED5FF801F2CF8F
:100A5000F4908F010F5F1F4FFF2041F08F2D0F94F7
:100A6000F45F8F2D0F94ED5FF801F2CF8091D204E7
:100A7000882319F06FE173E002C063E273E08CEA4F
:100A800096E00F94EF2D8AE00F94F45F8AE00F94C4
:100A9000ED5F4CE050E06FEC79E0CE0101960F94F1
:100AA0002581892B09F4CAC20F94DB09C7C2B1D5CD
:100AB000C5C20F94B040C2C283E50F94FE53882391
:100AC00021F00F94BC5391E089270F942F3BB6C2BD
:100AD00081E08093A4030E94EC8F1092A4038823EA
:100AE00009F4ACC2E2E7F8EEF4908F010F5F1F4FFC
:100AF000F11003C0E6EFF6E008C08F2D0F94F45F0D
:100B00008F2D0F94ED5FF801EFCFF4908F010F5F01
:100B10001F4FFF2009F492C28F2D0F94F45F8F2D89
:100B20000F94ED5FF801F1CF0F94410287C28BE57E
:100B300092E00E949D97811181C285E50F94FE533A
:100B40008823D9F10091D90B10E00F94CB536B019E
:100B50007C0120E030E0A9010F940F8087FF04C0E2
:100B6000F7FAF094F7F8F094000F111F000F111F1F
:100B7000F801E755FC4FC082D182E282F3820091F6
:100B8000D90B84E0089F8001112407551C4F20E0F9
:100B900030E04AEF53E4F8016081718182819381F2
:100BA0000F940F8018164CF480E090E0AAEFB3E4A5
:100BB000F80180839183A283B3838CE40F94FE5366
:100BC000882309F43BC20091D90B10E00F94CB535A
:100BD0006B017C0120E030E0A9010F940F8087FFBA
:100BE00004C0F7FAF094F7F8F094000F111F000F0B
:100BF000111FF801EB55FC4FC082D182E282F382D3
:100C00000091D90BF4E00F9F800111240B551C4F6C
:100C100020E030E04AEF53E4F80160817181828185
:100C200093810F940F8018160CF008C280E090E0BA
:100C3000AAEFB3E4F80180839183A283B383FEC15A
:100C40000F94F700FBC18EEB92E00E949D978111FB
:100C5000F5C18AE50F944754882309F4BFC38AE598
:100C60000F944754882309F4B9C30F94CB534B0115
:100C70005C014091D90B62E081E00E94B2C820E0A3
:100C800030E0A901C501B4010F940F8018167CF55E
:100C900080E090E0A0EAB0E489839A83AB83BC83D0
:100CA0002091D7093091D8094091D9095091DA099A
:100CB000C501B4010F94707E6B017C0120E030E02F
:100CC00048EC52E40F94A57787FD06C0C12CD12CC7
:100CD00088ECE82E82E4F82EC8A2D9A2EAA2FBA2F0
:100CE000BE016F5F7F4FCE0180960E94B59F85E564
:100CF0000F94FE53882329F00F94CB536B017C0192
:100D00000CC0E091D90B24E0E29FF0011124E755DB
:100D1000FC4FC080D180E280F38020E030E0A90168
:100D2000C701B6010F940F8087FF04C0F7FAF09453
:100D3000F7F8F094F7FAF094F7F8F094C982DA82B1
:100D4000EB82FC8281E0809397048093960442E0DA
:100D500061E0CE0101960E94ADE1109297041092DD
:100D6000960420E030E0A901C501B4010F940F8082
:100D700018165CF580E090E0A0EAB0E489839A83DD
:100D8000AB83BC83A50194016091D7097091D80908
:100D90008091D9099091DA090F946F7E6B017C01E3
:100DA00020E030E0A9010F940F8018161CF0C12C30
:100DB000D12C7601C8A2D9A2EAA2FBA2BE016F5F24
:100DC0007F4FCE0180960E94B59F40917C0460E0E9
:100DD00087E00E94B2C832C18AE50F94475481115E
:100DE00003C0E2E7F8EE47C00F94CB536B017C01E0
:100DF00020E030E040EA51EC0F940F8087FD0AC0FC
:100E000020E030E040EA51E4C701B6010F94A57735
:100E100018161CF4E3E4F8EE10C0C092760AD092E3
:100E2000770AE092780AF092790A08C18F2D0F9420
:100E3000F45F8F2D0F94ED5FF801F4908F010F5F39
:100E40001F4FF110F3CFE3E1F7E0F4908F010F5F54
:100E50001F4FFF2009F4F2C08F2D0F94F45F8F2DE8
:100E60000F94ED5FF801F1CF8F2D0F94F45F8F2D6C
:100E70000F94ED5FF801F4908F010F5F1F4FF11099
:100E8000F3CFE4E0F7E0F4908F010F5F1F4FFF20F6
:100E900041F08F2D0F94F45F8F2D0F94ED5FF801CB
:100EA000F2CF4091760A5091770A6091780A70915A
:100EB000790A81E097E00F946E2D8AE00F94F45F39
:100EC0008AE00F94ED5FBAC081E080933002109207
:100ED000D40A83E50F944754882379F00F94BC53C8
:100EE0008111ACC01092CB091092CC091092CD099F
:100EF0001092CE090E94D6DAA1C083E50F94FE536A
:100F0000EFCF0E942EF29AC060914F117091501154
:100F1000F62E8091860A85FF17C077278EE997E025
:100F20000F94B32D89E20F94F45F89E20F94ED5F83
:100F30008AE00F94F45F8AE00F94ED5F6FE777E04B
:100F40008AE897E00E9440E40F9473001091D20465
:100F500080E00E94439DFF2099F1E2E7F8EEE490E3
:100F60008F010F5F1F4FEE2041F08E2D0F94F45F25
:100F70008E2D0F94ED5FF801F2CF84E50F94F45FAE
:100F800084E50F94ED5F6F2D70E080E090E04AE023
:100F90000F94FB5F80E20F94F45F80E20F94ED5FAB
:100FA000E2E4F7E0F4908F010F5F1F4FFF2051F153
:100FB0008F2D0F94F45F8F2D0F94ED5FF801F2CF1A
:100FC00010927C04812F0E94439DE2E7F8EEF4909A
:100FD0008F010F5F1F4FFF2041F08F2D0F94F45FA3
:100FE0008F2D0F94ED5FF801F2CF60917C0470E0DB
:100FF00080E397E00F94B32D8AE00F94F45F8AE0CA
:101000000F94ED5F8091860A85FF18C061E677E056
:101010008BE697E00E9440E4E4E5F7E0F4908F016E
:101020000F5F1F4FFF2051F08F2D0F94F45F8F2D16
:101030000F94ED5FF801F2CF0E942EF21092FF04A0
:101040000E94AFDAD5C10E94DBB00E9495D8F6CFDE
:101050000F94730080E00E94439D0E94E09680916F
:10106000860A85FD9DC011E01093320588E50F9436
:10107000FE53B82E89E50F94FE53082F8AE50F948E
:10108000FE53F82EB11004C0011104C0182705C08A
:10109000011102C010E001C0182F0F942F5511113B
:1010A00002C0FF2019F082E00E9489D182E50F94EE
:1010B0004754882309F443C00F94CB536B017C0140
:1010C00020E030E0A9010F94A5778823C1F1111128
:1010D00005C0B11003C0002309F440C0C0927104E0
:1010E000D0927204E0927304F09274042091D709B4
:1010F0003091D8094091D9095091DA09C701B60158
:101100000F940F801816DCF48091860A85FF0CC0BE
:10111000B701A60184E594E00F946E2D8AE00F9448
:10112000F45F8AE00F94ED5F19821A821B821C82A1
:10113000BE016F5F7F4F81E794E00E94B59F111160
:1011400005C0B11003C0011106C008C080E00E94B4
:1011500089D11123C1F381E00E9489D10E949C9B17
:1011600080913105809332050E94BD9683E0809383
:1011700024020F94DB098091860A85FF5FCFEBE4A0
:10118000F4E0F4908F010F5F1F4FFF2009F456CF5A
:101190008F2D0F94F45F8F2D0F94ED5FF801F1CF39
:1011A000E0E7F4E0F4908F010F5F1F4FFF2009F498
:1011B0005ACF8F2D0F94F45F8F2D0F94ED5FF801B0
:1011C000F1CF11110C94747A0C946D7A80E00E9426
:1011D00034D40C94967A0F949B53AB01BC0140938A
:1011E0007F1350938013609381137093821381E176
:1011F00093E10F94393022CF0F94730088E50F9458
:10120000FE53882331F0129A8091740A8E7F809366
:10121000740A89E50F94FE53882331F08A9A8091ED
:10122000740A8D7F8093740A8AE50F94FE53882395
:1012300059F080910801809581708093060180911A
:10124000740A8B7F8093740A85E40F94FE5388237D
:1012500009F4F4CE5F9AF2CE0F947300BC2C60E0D8
:101260008C2D0E94B6DB0F3F3FEF130759F48C2DF6
:101270000E9460DB31E020E0892B09F030E0032F91
:10128000122F05C00130110569F401E010E08B2D2B
:101290000E9460DB8017910709F4D0CE80E00E94A5
:1012A00034D4F5CF00E010E0F2CF0F94BF6FC6CE7C
:1012B0000F94CB5320E030E040E050EC0F94A57742
:1012C00087FD15C00F94CB5320E030E040E050E4A0
:1012D0000F940F8018162CF00F94CB536B017C01E8
:1012E0000BC0C12CD12CE12C40E4F42E05C0C12C44
:1012F000D12CE12C30ECF32E8091740A82FF18C0BF
:101300000091AA0B1091AB0B2091A00A3091A10A79
:101310004091A20A5091A30AC701B6010F940A781E
:101320000F94527F600F711F7093AB0B6093AA0BE9
:1013300080E50F94FE53882329F00F94BC53882333
:1013400009F47CCEA70196016091760A7091770A24
:101350008091780A9091790A0F94707E6093760A52
:101360007093770A8093780A9093790AE2E7F8EE0F
:10137000F4908F010F5F1F4FFF2041F08F2D0F94CE
:10138000F45F8F2D0F94ED5FF801F2CF4091760A54
:101390005091770A6091780A7091790A86E496E014
:1013A0000F946E2D8AE00F94F45F8AE00F94ED5F46
:1013B00045CE61E0812F0E94B6DB6E2D812F0E9409
:1013C00088DBF12CB701812F0F94AB44143009F066
:1013D00035CEF0926006E0925F0630CE4091D90B98
:1013E00062E081E00E94B2C8812C912C54017FCC34
:1013F000A9960FB6F894DEBF0FBECDBFDF91CF9197
:101400001F910F91FF90EF90DF90CF90BF90AF9022
:101410009F908F907F906F905F904F903F902F9014
:101420000895089580E090E008951F93CF93DF938F
:1014300083399240F1F0E3E4F8EE1491EF01219644
:10144000112341F0812F0F94F45F812F0F94ED5FF2
:10145000FE01F3CFE5ECF7E01491EF0121961123A3
:1014600051F0812F0F94F45F812F0F94ED5FFE01F7
:10147000F3CF80E001C081E0DF91CF911F9108950B
:101480008F929F92AF92BF92CF92DF92EF92FF9294
:101490000F93CF93DF931F92CDB7DEB77C015B0133
:1014A0006A0149018091D0038823E9F0F701808126
:1014B0009181C80ED91ED182C08222C001111DC0E7
:1014C000BE016F5F7F4FC4010F943F56F7018081CB
:1014D0009181019691838083FFEFAF1ABF0A81E06B
:1014E000C81AD10869F0F701808191810F94CC7DF1
:1014F00089839091A4039111E1CFF5018083E0CF1E
:101500000F90DF91CF910F91FF90EF90DF90CF90F0
:10151000BF90AF909F908F9008957F928F929F92EF
:10152000AF92BF92CF92DF92EF92FF920F931F93F1
:10153000CF93DF931F92CDB7DEB7E091D003EE23B8
:1015400041F0FC0120813181420F531F51834083C0
:1015500051C069017C015B018B01040F151FA016AE
:10156000B10609F447C0F70180809180F5017190C0
:101570005F017982C4010F94CC7D781671F1672DDB
:10158000C4010F94F57DC4010F94CC7D9981891716
:1015900021F1E2E7F8EEF4908F010F5F1F4FFF207B
:1015A00041F08F2D0F94F45F8F2D0F94ED5FF801B4
:1015B000F2CFEBEAF7E0F4908F010F5F1F4FFF20AF
:1015C00041F08F2D0F94F45F8F2D0F94ED5FF80194
:1015D000F2CF81E08093D0030DC0BE016F5F7F4FDB
:1015E000C6010F943F56F701808191810196918346
:1015F0008083B5CF0F90DF91CF911F910F91FF9016
:10160000EF90DF90CF90BF90AF909F908F907F90A2
:1016100008958F929F92AF92BF92CF92DF92EF92F6
:10162000FF920F931F93CF93DF93CDB7DEB7CA59C5
:10163000D1090FB6F894DEBF0FBECDBFE9961CAE40
:101640001DAE1EAE1FAEE99780913103909132031B
:10165000A0913303B0913403ED968CAF9DAFAEAF44
:10166000BFAFED97C557DF4F19821882CB58D040D6
:1016700084E690E0C357DF4F99838883CD58D040EC
:101680001092D0039E0125573F4F44E050E0BE0129
:1016900067587F4FCE0183579F4F3FDFC357DF4FC0
:1016A00088819981CD58D0400296C357DF4F9983E6
:1016B0008883CD58D040C557DF4F19821882CB5848
:1016C000D04081E0CD56DF4F8883C359D0409E0182
:1016D00025573F4F41E050E0BE016D567F4FCE0190
:1016E00083579F4F1ADF9E0125573F4F40E150E03F
:1016F00062EC74E0CE0183579F4F0FDF9E012557A8
:101700003F4F44E050E063E07BE0CE0183579F4FC2
:1017100004DF9E0125573F4F40E150E068E97AE041
:10172000CE0183579F4FF9DE9E0125573F4F40E181
:1017300050E063EF7AE0CE0183579F4FEEDE9E01CB
:1017400025573F4F44E050E06BEE7AE0CE018357DF
:101750009F4FE3DE9E0125573F4F44E050E06FEE80
:101760007AE0CE0183579F4FD8DE9E0125573F4F29
:1017700044E050E067EE7AE0CE0183579F4FCDDE24
:101780009E0125573F4F44E050E06BE07BE0CE01E7
:1017900083579F4FC2DE9E0125573F4F44E050E0E4
:1017A00067E07BE0CE0183579F4FB7DE9E01255750
:1017B0003F4F40E150E067ED7AE0CE0183579F4F05
:1017C000ACDE8AE097EDA3EABCE3E9968CAF9DAF6F
:1017D000AEAFBFAFE9979E0125573F4F44E050E0C1
:1017E000BE016B587F4FCE0183579F4F96DE9E01FF
:1017F00025573F4F4CE050E06BE475E0CE01835736
:101800009F4F8BDE80E090E0A0E2B1E4C358DF4F51
:1018100088839983AA83BB83CD57D0409E012557E7
:101820003F4F44E050E0BE0163587F4FCE018357E5
:101830009F4F73DEE9961CAE1DAE1EAE1FAEE9973C
:1018400083E0CC56DF4F8883C459D040CB56DF4F5E
:101850008883C559D0409E0125573F4F44E050E052
:10186000BE016B587F4FCE0183579F4F56DE9E01BE
:1018700025573F4F41E050E0BE016C567F4FCE01EF
:1018800083579F4F4ADE9E0125573F4F41E050E06E
:10189000BE016B567F4FCE0183579F4F3EDE1AE04D
:1018A00011509E0125573F4F44E050E0112341F075
:1018B000BE016B587F4FCE0183579F4F2EDEF0CF76
:1018C00066E77AE0CE0183579F4F27DE9E012557BA
:1018D0003F4F44E250E06AEB71E1CE0183579F4FE6
:1018E0001CDE83E0CA56DF4F8883C659D040C956F4
:1018F000DF4F8883C759D040CF57DF4F18821982F6
:101900001A821B82C158D040CB57DF4F18821982F0
:101910001A821B82C558D040E9961CAE1DAE1EAE81
:101920001FAEE9979E0125573F4F41E050E0BE01B1
:101930006A567F4FCE0183579F4FEFDD9E0125579B
:101940003F4F41E050E0BE0169567F4FCE018357C3
:101950009F4FE3DD9E0125573F4F44E050E0BE011D
:101960006B577F4FCE0183579F4FD7DD9E01255781
:101970003F4F44E050E0BE016F577F4FCE01835789
:101980009F4FCBDD0AE010E00150110969F09E0184
:1019900025573F4F44E050E0BE016B587F4FCE01CA
:1019A00083579F4FBADDF0CFC856DF4F1882C85912
:1019B000D0408FEFC756DF4F8883C959D0409E0172
:1019C00025573F4F41E050E0BE0168567F4FCE01A2
:1019D00083579F4FA2DD9E0125573F4F41E050E0C6
:1019E000BE0167567F4FCE0183579F4F96DD9E0104
:1019F00025573F4F44E050E060EA73E0CE01835743
:101A00009F4F8BDD9E0125573F4F44E050E067E636
:101A100071E1CE0183579F4F80DD9E0125573F4FD7
:101A200044E050E06CE973E0CE0183579F4F75DDD1
:101A300010E0C12C80E8D82E8BE3E82E85E4F82E48
:101A4000812C912C90E8A92E9FE3B92E111134C05E
:101A50009E0125573F4F44E050E064E37BE0CE0118
:101A600083579F4F5ADD9E0125573F4F44E050E07A
:101A700060E37BE0CE0183579F4F4FDD9E012557EA
:101A80003F4F44E050E068E37BE0CE0183579F4F37
:101A900044DDE9968CAE9DAEAEAEBFAEE9979E0139
:101AA00025573F4F44E050E0BE016B587F4FCE01B9
:101AB00083579F4F32DD28C0E996CCAEDDAEEEAE47
:101AC000FFAEE9979E0125573F4F44E050E0BE012D
:101AD0006B587F4FCE0183579F4F1FDDE9961CAE99
:101AE0001DAE1EAE1FAEE99704E0015069F09E01E5
:101AF00025573F4F44E050E0BE016B587F4FCE0169
:101B000083579F4F0ADDF1CF1F5F153009F09ECF3D
:101B100084E190E0C157DF4F99838883CF58D0404C
:101B20009E0125573F4F42E050E0BE0161577F4F75
:101B3000CE0183579F4FF1DC80E090E8ABE3B5E442
:101B4000E9968CAF9DAFAEAFBFAFE99714E01150EF
:101B500069F09E0125573F4F44E050E0BE016B58AD
:101B60007F4FCE0183579F4FD8DCF1CF80E290E0CA
:101B7000CF56DF4F99838883C159D0409E012557A6
:101B80003F4F42E050E0BE016F567F4FCE0183577A
:101B90009F4FC3DCC656DF4F1882CA59D04080E23F
:101BA000EAE5F2E0DE019D9601900D928A95E1F75B
:101BB0009E0125573F4F41E050E0BE0166567F4FE2
:101BC000CE0183579F4FA9DC9E0125573F4F40E22E
:101BD00050E0BE01635D7F4FCE0183579F4F9DDC78
:101BE0009E0125573F4F41E050E06FE07BE1CE0181
:101BF00083579F4F92DC10E011110EC08091101B93
:101C00009091111BA091121BB091131BE9968CAF00
